:020000040000FA
:40000000500AF500122A4E00956CE600A5BF3300F2DD35002F2E3C00EC24DB00DB121400C8EAC20015650700257C11003D94760026A3110075935B000E456F00EC7F280060
:4000400036711600CFCE2000B5217000B9B6B500490299001D14D400150E0A00DCC4EC00A5BEE200CF903000BB26FB00D29591002BF70800A3F0DE00B6A25D00D8F09B009F
:4000800033CA8800E943B800221F3F004DF23D00866E0A00EF63DB0020D01600F76BC000AB0ACF004CA56800A413EB007823210013547900EFCA8B000B9F33003279190088
:4000C0000D438C0085C38D009853EA000FB36800EFF905009313A9008D2B3A008B769B0050413A000B3F560082440000A3A66C00D1BD390080E3A200F215FB000481C60087
:4001000067D08F0053EA0B00D98FB100F0A72F00601CE200448AFD0092E6BA005F82B000A60B0300712AF8004860C5002FB41900A28A6300CD7C71002AA94F00C88CD300A4
:40014000D6676300E0B6D6006C4BE700CFEE8A0003DF850094604C00D0FBDA00A315BB00E6FB30005B642C0042AE1D008EFD73006303630017B25E004570980069C29900C7
:4001800033CA8800E943B800221F3F004DF23D00866E0A00EF63DB0020D01600F76BC000AB0ACF004CA56800A413EB007823210013547900EFCA8B000B9F33003279190087
:4001C0000D438C0085C38D009853EA000FB36800EFF905009313A9008D2B3A008B769B0050413A000B3F560082440000A3A66C00D1BD390080E3A200F215FB000481C60086
:40080000EC732200609DA400DD28270063800400B4CE1000D0B50E008DA94200A1586800CB450D005CA6C700B72A56002209AE000380D600506B6A0077E10D00C9B9B50075
:4008400045902C0036D94D008AAAF2003552D6005903AB0045F4DB003BB53900E4EA7800A55C19001BED7F007B937A00AEE20500C624AC00199F0D0079E2E70082D055000C
:40088000704110002F342900644F07002E4F6B00C0E22F00DD00350083BC37002F11DB008E4CBB00FA9C3B0032CD1900C12EDD0088E69D007481E700A0731B00FFC7BA00F6
:4008C0005B70AB00C0882B00340D9600B09114003A2C5F00F42B8100C896CE00E151C200ED5F410048AD9A002C693700DD9C5B002035ED0040FECA00220F9D006824EB0013
:400900009F5DAE0006CFB500AF946F00B6F30C002737BF0021ADDC000A9ABE0028B4EF004951DE00DA0B1B00B34D0B00CE51A700337BCF000F2D8600D5504E0071DC3C00A4
:400940003575180030C253008F45DC005D2C6E00A4229D0025581D003742E000C7718C007C3820000FBE70008B1004008E4E2700CBA0BF00847DDF009E86B100CA4AE40025
:40098000E876820004B1DE00533368007B5CA3001BD6D0005A69D500D3067F004630C60068839200C4A30F009495790003F2CA004CA66D001D8BA00002E97000263BAA000E
:4009C0008772EA008031AD00422598004CA1FD0080680F0014895E009D358A007F4E2600B480B1007226DF0060AB6F00B23C23006478E800A9F71C006C22DF00E593B00090
:400A000031592000E0786600110A7200364A1B006BBEA40048F72600B388890031F9270039223500A0E61B00EBAF3200C1B085007F8B7A002192C1005FB5FE0089FF9500C5
:400A4000DF0BB200F0C5AD000E727100B944FC005B74DC00818374001BB8BF00BFD2C500C21A2A0026186600220C9C00F1B49C00B5467C00637D6600B93B2C00C8BA64000B
:400A8000467FB3004FE70E00C521D7005FB062008230400073ED7F006778CC008A2183009A496C004D9571004738F3005EBD0700A52714009A9E5300CDBCA9006E6D3900BB
:400AC0002588E200044E4000C7B4850023251B00CA3AA3007877F200DD2F6C00D11D8500D7CABB00EE6087006A1013008BDA24008D4D25006DC17E0039F9130067FACE0099
:400B0000EC553300C0094800185F3A00957121005F1D120035B035003BBA9D005B44F40015B1D900E86B6B00AB476E0003B05B00BA78BA0041E2400053191400B009140024
:400B4000ABCDAD008C8B73006622A40087F212003E5A74003082A8009DAB1E008CF26B0024294A00E45A1600BDC59D008A71A00087E178005D8564007AF73700CCBD42001C
:400B800057AE33008201C60016301D00F2B687007636440067D5E400F75BBA005D304E008332D90053DD52005FC45800F3307900AA97E100B247A000F4F070008F2B5B00E0
:400BC0008980ED00764321005E2B0F00EED184001019F20092EE2E00F32CB5004357C700CC7ADA00467BE100F84ED300B2F21C00F6FCE700D622C100BD51620099F3E8003B
:400C0000E6C0F300222FCE0033E4BD00E027FC00DC66BB0084906C00619C8F00D00E95007A683E00388F31003D767B0040657B0028D8040041F996006FBC7000F75B290059
:400C400015E8D60090D751008786AE0086397700109CE900992E30006546EA00A4095B00981EB40073FBD900B6C6B1007DC0730008948400B4B18000C72BC000F0070E0085
:400C8000FECCC300D71C7400755E3800305AD900ADA18400906FAE007B16D8004ABDA00080E5AA0072420C00536F56002CF5A9004A6DC200930C4700436F7900FC278F0056
:400CC000FB465E00983371006188A900927DDC0044BBA3007555BE003C5AEB0009451700B2DD2A00DEACEC008FA36700B406080033E4AD00CB047B008992D2001058B600E9
:400D000075702F001237E100ADC58C009C690500CBA7C1006A6B6B004CA2C0002ACE1300A9A2440054E5010012EC3900F906110033398A002A70570065787E00DC32500091
:400D4000B05B8C007B727000D08FBC00BEF023004F810B00A350AC0006734E00DF04F70049D100009CD6B5008EEE0600B51AF50000F5610043164D007439DE0020B6B900DB
:400D8000099F6A0037A3BF0037214600239C0E0092FB2500083C2D002E1A970088099200EAEE6000BB4B5C00525CFB00FD06990043B8B400D753ED0072C5AF0035631600BF
:400DC000EA486C009100480012E872005CE20C00885D020055F1A300608F73001AE71E00D96737005240580060F52A001E929F00DDF20000E737D80037F6AE00A836EC00DC
:400E00009C839E0038E5C4008CC6D400CEB65500C7EC1F00E0ED89007CE8E200EC1502000370EB00FBCD390070AF190015CE63000E71D400F873E700A7AB1E0043C1A50009
:400E4000E79DDC00F8AFF7003198900038246D0026F9BE00C597AF007A2BAA00F4E7E500A9D52E009AB77200EA122A0068209500002DE400978DA300739975009862F7005F
:400E8000959AAA0023DBDA007D33D70053F432001FBE1B0046CA7600D871A900A0C9E600F5B4FA00E2FE2B00E91E940095A9CB00F6D2A4003F98DD0067AFE4001CF6AE0096
:400EC000CA7CCE009E74B800BD594B0060753300E172AD001E4B2D008D7D7700D47B2300671C970086EFC800575C120067BA780084E4CF0083F9630030D1D000C7AD2500ED
:400F0000C0E69400944E27007608CB004C2E8800DC5FA200275CED0003FC1A00FB68BC00D66EA70052B43400F6A814002CF8EE00504A540048387F00AA3F7C00C400F700A8
:400F40001C8AE2004B050900E06520006A1A470050BD2C006C63A8008E7D6E00EBF09C0060CFA20042C58D001A22730005C6AD00CD17CE0009CF4600D9BA5B003A99A600FD
:400F8000947547006690AC00AC2CF0000880BC00C900560072894600EA33840059563800CB727500929562009E262D00DDA4B9009C849D00722BAA005739E100DD796A00B0
:400FC000767E7B00EBA4D000EB8F3F0070E31C00694F320098E4F300B33B2600F24EF0005BC58E00F7193D0008724E00B2AC59005E231B005EE1F900EC97480020292B00D1
:4010000075476C00CC35B700698564000B240F005E5866006C5E160091DA390059C2FD0049C6130055B180005E9C13004F2F05001A515E00B4A5650034F2D4002ED59E002E
:40104000DD60470049F89B0036BE9B00001A6400EF96BC00D8863C0018DCA40007A0B4006FDC890041E3CD00A8D251003BF53400471C6B00217E8400E705F800D2392A0037
:401080008E569B00079DE400238AE7002812670056123F000AC9A5005C56C700B615FC00086D13007C52FD00F08305000673780095CF4600EFFD60008AF2940046DF850029
:4010C000E770CA00F3F2FA005F5A5F00D97A4400CED6F400F93B53004C685300DEAD96000C843900FC456200C06C67009DC96900E29D7700C15A18002F8E2F00DFCC0C0060
:4011000070A20400B9EF4800166BA600126F880058925D00DE262000FEB1030019073A00D4FE7800230E5C001E6EC50063448200D7C79800258F1E004C07CE007073250080
:4011400006FB47003DCAE700C78C8B004C57C30078A91500035AA600AA3B640092DADE0079146E0025CE9400920378008F045900BA1E1300DC4538001A9BE600CADB5A00D0
:401180001A82BC006D2D800084089B009BF56A00D10110002D0DA300D407E30009A1540068EB1D00D449040036861500F49D6E0007F6C80060A9180055AF34009BE3B6006E
:4011C000E29B89009D71C100E2087200840C89004BCFF200B2FA7C00E5635B00BD0A9700D7F0F40098CE4B007915890026C8BA00B1213B0049BCF900C56793008747A70006
:40120000C9B85600F7BCFC003A62A800D6565800BA39E1005C90B200733BDC0070B26D005572C400A8DB86007788E000BD2191002D595C00E7ABE10090BB25002A310200D1
:40124000D7C8CA00C0BE1600C644E7005B3EC6005069C900CC5236002CD46F007D53E9001150AD001827FD006E136C00A50C1B00CB7D0F00B29511008CAC4300902DE90050
:40128000ED920A00129FC10042AB56002D34D3007E4800006F15F400A49A2300757E8E00B0629200E97C2000C3143700DEDA770081A1320015314A00584D7900C3D3ED00B1
:4012C00097ABDC0083FD4E00077AAC002819DA0075FC6D00F935DA0057361C0019B5FE00C28335005D6BAF007D5E8500A9D7FD007B17D5002D76B000CA19F300C8125B00CC
:40130000A3C8C800587B3900A358760013930200F34C640009257B00E65E2B0037065700339C1C00DC4BF500EF627100D7631B0006D97900AA5B2B00933D8400AE8C1C00B6
:40134000E12C81002F6C6000294657005782000031AEB400741CE2000DE71000BE3D0100B91649004CDD220000ADE800D9029600731F690041639100563628005E257F00F1
:401380009D7364000131B7006E347B00D1008400D44B5B00D8B43F0006BF9900BB6190005A1D6A003533DF00B0188000B7A8EB00C50FC4002A910200DE83F8008535D40019
:4013C000697BF50011284F0024E5BD0087352D00AA04D400E9B82D002BE828009E9F2B002B922E000E58BD009D881A004C2F5800095308000BCC30007A245D00CD5EE70052
:4014000065CCF200456EE100D1A15D00E272BE0000063D0090D0330064A0C60091DCD60078D99400725EEE00AD7A5C007A53DE00685CB80016243E0045E1AF0008DF62004E
:40144000CBEF7100C2204800D5E1190091130A0036759600BC27F2004F2F2C0077E74400833F7500EC32D8003614C800D241000091024700AD4A2C00EC30DE00FE48700039
:40148000CC509200D684A000FE1B45001684B100A64FC200474BF000D2BAA30041B5A1007E1CC500ABCA9500F9F0A20079DB23006F601D00D9F29C001F655F00B6483A0003
:4014C000731A0200AEDF08008508A000F467D000CC88ED004FAC910097156300535EC800C75C19009BE3150031E8BB00C9849B0050EB400092CF7F002E359D00ACAA3A00A5
:401500002B144A007A66C30088F1060094CF33007EEA4900BA72EB00B5D8A500DD31CC00874B5E00BB6DCC00F4AC36006DDB770071A20B003C7E79007AEEEE00E2FC130045
:40154000A4E945005C47C700BA51AB006ACD5F00C60DBC003899B0009E58B400676B880031AD520085CDDB00ADFC73001AB97E00A31C41003D02CD00374011006BB1E30072
:401580000E5D590095549C00D027290012595A00E396C5000D0B55002BB7690014BE2B001E760F0012163D00A2877A004014020050C12600EC296F002647DD00898D2100CD
:4015C000534AFA00A531770015D52500A7BCD9005E5C5B00390E7E00039C6400EE6BF4003C34BF00BCF3D300E3F2CF00B5130600256F8B0010068800543C76001A515500EC
:40160000C1C373002B5B8B00E0AA0C0084B7B90013ACAC00E5CEE400EC41FB001FA28300B4E8E8002E149A003DB82400C697BF0007157F00DE21060071793A0095D63700AF
:401640006E531000AD19A3005E15F000CC5EF500D87D4F005B987F00FF196200D8C05D00FE73F60050ADD200F28F320067116D003E68BB00CE3D3200968C620031124C00AA
:40168000D1269F00BB904100F637960083545A0053A8CA00C7E8BB009F65B900722D5D00136F4500E1075C009BDFD100098B1B0044C5C500A104E300A01135008DCA78001C
:4016C0000E23DC0095B42A00EF16D60023977500E82C9F0003DA10001C55CA00A6ADFB004FD8A300E293B50010905F008E5BAE00DAFE7A00AE4C3C0070AFD100B095F700F9
:401700002B1F700024AE62005B46CD00AB1B69008AE2AB003A688B00F5F852008DB36300E72C05003CDDA20067FC2600549A82009F35F200204F9400BEF01500CF09EC00DC
:40174000C4C17700EF860F00D4352C00723192004DB72500D7640A00FD843500D71CB500D8E48900BA1BCC00AD992B0032D4D600A2DC850061E5D300C11BB200FEBFFB001E
:40178000D44E9B0037FBE800D760C500E1D7AF0089EF4800368C7A00BB5A5C00FDF51900E199970086C75B00985EBF00C3E6A300D3D9E500B6DA900083A4C2000C71AF00F7
:4017C000BA900B00D123E100E662000040172A006CCADB0067229400C51D6A00CF6BF300A6EF9D007A7021003DB879004D5595008BA80F00E5BFF600D72A48004826910049
:40180000D63A1300B9406B00FC0E22004E11C400913A3C00F0643C00EE7779001EE459009FFA530052E69200C283EF0090D568007C55AA00B4664F00FDB3BF001191E7006F
:401840007890AE00987BBD008C148800C0E27B00447BF000E5EDCF00D31AA100AC5612002504760061DA3E0011B65400C5C3680065E4FE000EF94E000301EE003C78C20084
:40188000031858006F020600D300F500E1314E005F973000F59F2F00B20ADE00B8A68D007903AD002BBF3B003E333F00531665003571A5002F71CE0087026500CA4B05001B
:4018C000620A8A00EF82820062093600CE1965009DFE44009121ED005DA132002B47510037C99800B54FF20076EE4D008BB355005294F200821C52003B3AEE00CAF00400E6
:401900007B117700C589BF008D003800C7AA5300E377AE00D9FFDA00D690FE002F2A41008B8ABC003801130080E2D3005777C1008D98C700EA7E1B009C17CC0050284600C9
:401940007BB91B00FBCCBF00C379A600020ABB00505D3B00FD7E1800B8790000CFD15200B475FC006B049900E6E92100C7E53A00B10F9A00488AD900AD314E00A3C9370074
:401980004AEC8C00560C0C004A094D001753AF00B1A56E00796EED000E797A00E97FC40014069F0096329000587AE00085F38300ABC6CD0073C72F00C7993C00EC2D370028
:4019C0005DB73900D165A70002C24B00DFC0C500B35B56003500C2008F1F440031E4530030B7A7006FF93800AB7E7E00CC35E9007176ED00C138AF009378BB005080E900DB
:401A0000BAA60900B7122C007EE51600103A0400797364005BBAC3001840130072690D00E843BC00DFECCB0000976300F24DE70035470F004D36740056A2400047A4900034
:401A400005429400CE6D400067376B007419FF00A6AFA600C4173600588FC80091C703006B3AEF0077D1700058AA8000D33E30007216D400F8DBEA0044708600DC8DED00AD
:401A80006A990F00FD1FB2001200E3006686CA00A7F8DC00001A5600F83A2A0056463D00E28707007DA6A300BF913100D149E6004194FA00999C2900AB158C00FBEC430021
:401AC00018B3EA00BD74D900CCE4A1002C15AA0095CF3A00B73F8100976757009096E8004A2A4A00B221F4006AFF44002FBD2400AF258F00E80CE400B2B800001E05C000A9
:401B00003BA763009AD067003A812900C52746004EAD81005C1834005A178100DFB9B900D9D8D8006E1DE600CC4F2100F0BB2F00AB5B1700A58BAA0072839D008CE8D8002D
:401B40002FB2FC008FD5A9005F7CFB00D7BD4300F3BED30032877A00BDD2F9002E2039005A1630002AD57600CB028E00F042BC0073927F00D30B58000FB7FB005C32DA00C7
:401B8000DCD41400A2403A00D2B9E20067474C006143570046C2A6008AA2CE005C280D00F4F06700CF714B003B531C00E0577100A0647F00A825F90098F863008836550033
:401BC000F4D55F008CA88D00F106A2007EFE0700F5791B000FA36C0069F5EB0098DB090069EC8D008EC7BE0053D8CE000D51EA008AB863004726FA00CFCB34006D95620000
:401C0000882DF20094A88800ED0AAB00D55EE300270C8800C4BAAB00624FA900965386003526F400B5798A00B8B82100DB04FD00CF04BA003485F200494B0600D9A16000B4
:401C40000409430083BE7000B746D20067882D00A01FF000C9A42C00DC5E6E00CA871100E0321B000E0AFF0079A51A001D06B70094EDF300688D2F001BF04200463E4B001C
:401C8000A8A25D00166A2A00DE48D800B687FE0056F578007DD0DF002A8625001B8B6C000C95B40082633D0085FF3900D044940087B63800E0CB5C00EF01BC0083DF060058
:401CC00016FFC600EDF58B008F1D2D00CCDF250099BAF10013427400A1AEB5009ECCA3000DBF1A00E2FDA4000BADC800538605003AE62D0067435B0078B11C00A264CE00A3
:401D00000672E7006DD0D300251CDE00766BDE003827BE0095882A009CA151001C1C6F00BA37AD0086C1A4004CC9E600DD9D390014324800A9CFF500F5747B003CFFF30079
:401D400031C6C400B0592F004CF23900451198006F9F7D00A56CF400A94CDB0036B7320017876C0081AEA60086B70B00981924001D6A0200252AEE0030BFB3007DD97A0058
:401D800027EFF000A32B5D0059BA650063B25E00C6EA3C00D2176B007C1193003739CF004AB172003F8DE4004433C200F8196200343FC500F711070019BC7C00A5D153003E
:401DC000980F790095776F0015A873000E582C005BD4E300FDBEFD000402CF0050867900E5AA7300EF953A0048E10500BB1D440099A17900BB3EB7001FAFB200F62F7E0008
:401E0000F91454005D08BA006BED6500CD308200D4C8FB008EAB3100FB931C00747E9600BC285900B86E8800914AB7001234CB004C2D0600AF3D8400ED85EB00615A160008
:401E4000ADB12F00879D4100FE7520009223E200DD6B2F00E64AF8000AABCA00FB4AE1003B173D009CE9CA00DA23EE003163CF0005B3AD00210E2E0039D1E9002955820021
:401E80009E446B00EFA85600D747E9000BE7B700DC44C5008B721B00D9345D00594E5200AA434E0005BCBB0092F04D00270C27002EC68E00F9789B00279DE6003814D8009C
:401EC0000927C40005BDBA0029741100A1829100413FC100B427FA0004BC700030C7B300F2A0D10043BD050028993C004D5AAA00E5B4B500FD0738007F3F6700939E8C00FE
:401F0000FD81D700357FF100A04FB4008664EC00957FBF00BD624F00409D3D002F8501002E95880010313500BC846F0049B0A9008CFD08006EF51500BE60F20012258F002D
:401F4000B4338D00287F690012D6B1001C16B900B4EA640030B73B00C925BE00CF0BA80008771000EA9A9B0036ADF4005B6A4000B19E1F00400E7C00C94B5D008E6E1C00BC
:401F8000237D1F00C6225600C13ADA0068406D008B315B00EEAEAB008C12A800ED9EC00010737E00E726A1003B929D002FDD63000CC8B900402AD2002B87710075AC1B009B
:401FC0006C3DBD002801C90084AE0C00CA9A4C007CA8CA0006CD0100D44E7C00659BB3005DA40B00CD9958005B6DB100BD1EC600C9060300D2D52C00CE6BDC005EFADD00B5
:402000006DFF6F00CF1BF80033A86600285EB90082952200CE6C9A0053241800BAA44100598CB70007FF720022069A00E2B56600E14EEA00C68C7E005BCBF200064C1800EA
:40204000B429FA00C683B300BC076A00CAA81F0071873B00257237005A8DB500A552BE005C84E20083D24D007BDEEE003709F80018A61A00DC00350068CBA500F8803B0026
:402080001E211B00D8F3490036F32200DD5470002C824E0046A3A2007BAB3600E41A5000964F2A00E34495009C4A39003701970028DE0D00ABB6770083465000BB90290064
:4020C000DACD89008609FC00B7CAD50013D4C200A4F21E00809AF400EFDD8D0033D885002C8F510096A6330074ACFF00747DB000D47D2000B9052300AAFB1D005FBCB2005F
:402100006C393F00F7975D00C47B84009CC2EF00A789030071293000998F2400A9C471006D9E1C0009CCFC007DC6670034240E00441DE200648E4B00956BD400E8B3290079
:40214000328EC100284C5400EB156E00FCEAF300EE43AB000DF9700042377C006A368B00F1C89F00CBA51E00845C7800197C9100D3EB5100A4351200CA59BE00A3953200B4
:4021800072366A00EAF0CB00304AC400F2527600FFADDB00CDD58F007040E000047D9D0038A8E6002F95C6005E6D230057C5F6009C02230083F38B005D1BA20017EA7D0060
:4021C00049434200DBBC6700E6DAC4004473440044C1590004761B00880C5500D0D83400739AAA007D99C90025E669005A6E1300B5B20300049A33008871D900EC98A900BD
:402200008BDB6A0040EB5D00FE0ADB009AF6680042704000DC9AD400D7C6A600CFE50500414D12004A17230094F4E9008965FA0080CA2C0006C46200379E36001BD1B80065
:402240009912F500E1735100B661B000C44CF000B1B8AE00CF5F5A001B0699004EC3810053C30C003E438B00E84E32008E6E43007FA3F9008EBA090005217B00F41EED0086
:40228000FF78E900B8077D0032213900727C7D0005243F00EA1DEB00B6425B00AEE3A9000E4A1E0077650B00806A610009EE1F00A45D2900830B78004F6BD00023690C0094
:4022C000563120009B0A3A00642CFB00AF81970075A8490078950E000629C20076091C00611C7000E0A30400BFA47A008B6CBC00E3854700C6AD81003DAD2000351D1100E5
:40230000857164007FC98B009689DD00D9478600F3A9E0003DDEFF007955E40079060700766FC4007D5A200039073A00332E7C00FCC4570028D91D00B1B46B0014D7820097
:40234000CB797300F1110D00FC9FFF00D7C79600E2228A007F4C4C0002883F002F28C5004ADAC300B899FD004140B800693BE6007F0D1600A7C75400886CC700AF973B00A7
:40238000B5FB8000F72ADA0068C897003BDC11003FE8F7004DF7A1001472E10073E68B00D5CEB500856F40008CA9A300E9EA7B0038896300B64B44009E27580038256800B8
:4023C000FFE93500047C3900769759004F0AB9009DE4C0007AFCF40021ADB200BAA08F006B875300B9BE03003030C600A5EA8A00965C8900A66C9E00D9D9C900DD51AD00FC
:4024000087B36800C604F50030E4E7001D92DF00AFD876008B238900FA23D5003E3028005213AD003A5C9100F1AFAF00D1160800B61172004F17BB001179280061A05E0014
:40244000862121002D265700A170060074EAB50017DC9200E70CD200093062003729B0008B766D0000081D00F49C8200E4B27000176BE600E6994A00545E6A00665AC9004A
:40248000CC9A3F002CCB6F008B49C10005874600D8622A005C972700D04EF900466F81003ADF3100518919001A4A40001A9D0800932A86005FDCD50097746E00972E3D0071
:4024C0002244C7009E2835008F2E1600D4CFA100973F8E007465D80023F50C0039AC67000FA0090074946500C6D99700E5E03F00E686C1008E382E0032CDB30074F49100ED
:402500005E989500BEA69E00F0DAC000503E5600457CAC0034B5FA00E3758300716F25000FECAA005DF7A2001170180008A7350051D868006811DC00D46823003165EA0093
:40254000CFB67E001924E3005A26730076BB4E00BBC86B00B822A100922D440080E82500F83E3D00EEFD2C009E7E3600C984A9008C2B62002E7397004F0DA0000C39C600A3
:40258000FC29BA00C0FE4900FC9B7C002B23D0004CA1E800AF65DA002196F70038476600B195FC00445A15002E863100CFA64C00B6C20F00519C8F0086ABD9004AD072007A
:4025C000AEF7EE006122300033483000BE82F800F000D70095F20100C6C0F2009BE3E300ACB30F00A558F700612DE000FF688600C24B9C001B387F007D365700EE3E1A0002
:402600009FECB200A20C3000DE2DED00B774240039B78300B6BD0400CE7A5E00714E6A009BD5B800E0F3240047D6C70090E7C100A02A6F003AA2000035B76D0044EB0200A5
:402640002594E000262FA20052C5F500E7BFCB001B4B5F00C0964300CECCE000A440E200DC630300CDAAD200D36B1D000C2D0500F07437005A8D7700EAFE0100A452DA00D9
:4026800003FD7800D538210007B249007CDD26003727F4003FE612004BFB4F00A38B6000E2FB0900DD64C100442285003996DB00056B140030E21D00260BA300C96C82008C
:4026C000E5C38600AB09BD005E063E00EDB7180046E29E0086CBCC0061E78800E7EC4200F415C600F37C5F007C397B00EB86DC00595080003C9C8A004C3CEF009ECFCD00BF
:40270000FDDE730090A1DE001B2297008ED9730033457A009DE33F00FAB1BF0079B900007A1D8C00EDB62D005855C9004ADB5200735FAA00CF592E009C49D700EA9A9A00B5
:40274000E1362C0016AF150041797200524A1D00AEB13800A41C9B008DA50000EE4A43000228B00002392A003F3F17009F49D800B7A1D7006D713900F58F75007529F9004E
:40278000018BEF0062C4AF0025A8D50064E0D900FFF51B0012A37A00EC0D51003AB6E2002104D4004E8D4400A2875B0062816B0009D838000A52B6002129A300C4BC3500F9
:4027C000A43D630014C7A400C4C890006A4470009654F8007681AC0010331800078D6600A213E00078A54A0028CB9F0071CCFF0060FE3A002CD46700BB080F003AF6BB007C
:40280000B208B100C36BCE002417120007027F00DF7DA10078C6200089BCDF00830B8600D140FE0034CE8B00F6A63F00332ACB003FC7AB00CC5F8C004347C100F0D398001C
:40284000DD869F00DADA0F008451F600CF156600FA620E000B5AC1001C9CBB00DDB5B1002F2B4B007F7BAA00AE1783006992D200B5C22B000C03D100CC60F500674C66001E
:40288000D79280007151F000D4E23900D499FC006183AE00EB682500E269BB007CCC40002D575200FF98C7000636AB008E927B00F4B254001C1E5E00D7A725001273890094
:4028C000879285007FAA4F00DE21B10088A8C800B498280009CB0900BC22DC00C1E24C002E797100D5065600D8A14D0040348800B3DC06001EC3BB0080729E009CE42300B1
:402900008517DA0087D5900001F9C4005A5A1B00C9196000A68CF9004A85CA00E058EA00FF7AC900A9BA0E001D0654007F914C003B0E16007A466300918C09004CA2E9007B
:4029400010190E005C0D8400AD99260019E76E00A45ED3008B7B64000162C900FA0AB20025305A003F599C0076075600EBB7E600E95CE000F0938B001B582700431536009F
:402980002F74C90019B6CD00F7C3C6001E604100EAA38A00C0F90A0041E61000814FB70063E2E2003E834900895CF200D38C5000ED739100E889BC000A226F0061092E0030
:4029C000AA348E00994F6C00B7ACDF00F572190087FDD60007E1DF00A56BB4004C3C08004F48FC00016FF10067EE930072BEF20014C7480060062500ABBC0800F3C7CA0041
:402A0000DE80AE00EB3E9800B3465300A759A000BA505B00C71B9E004763F8002655A50025DF4600B9BEA400FC720F0069586300251DB700679F120035D14B00500BF20081
:402A400036AE52008DB69500712BE00027BB2100DFCF4500CCAF5D00573C2200FFF33D007B389900EBB6780037BF5800B56408009B87B200A35502008D273C009D6953002F
:402A8000DBD86700849FC50067698400BF65EC000705650033245000657BF8003957D200B01C690073B75000F5F84300B7A5E0002F262D007A737400312593008E00880061
:402AC00061377000AF226C002757A500B9B98F009F1DF80039287E005DF91D00D9DF590060A34C00D7D16F009B95C2003AD60F00A305B4002B05EC00E58B70006D525D006B
:402B0000978546007426CE0003221900D251AA00EC4DF600E4A2BD0083A52100821A500075E44800DEB55500CF1172008D61B600E7BBDF0070FD14003DA49F008DDDFA00B4
:402B4000E8087C009A884F003129A00063696B0082A41700343D8000AA7C15001D3E4800A995BB004574FC005A0A15001F3E94002D8F0C00A8FABE00E4155600BAA9C80081
:402B8000096B3300332706005E4BE900B53B7600A7E28200B2372600DFB166002FE166003384F900FB123D0034B8C100A6997E008B26A2009ACCDC0044CEFF0035116400DC
:402BC00082FE5B0062D776008A6C0600A0F42700F3E3DA001845A600D0583300364BF0005164D800CC630500009C0900FC2D1E00053DB300DAB5D100A01657008D93660080
:402C000009B9B8000B681300F8443D007A6AC10026BF13000661BF000B049400DA690A0049C21500D30D7D0071B3FB0026554B0070A8CC006D449D00AF1D7200FB04A200F5
:402C4000AA85E7009B91530036B6B600D775C3007A9C3B00D5E0A700C4A057006CF736009C52CD00478AEE00D514D90026CB5C00FFA91A00D9F934007DCE990016F23D0093
:402C800056CC6500BE8EFA008D16B800116DCA0078184200862E240064EEA6001C73E600DBEA4B0086655A00180B8A0028764A00D08B790065ADC4004C19BC00C6D24200FE
:402CC000DF4F0A0020685D00A51CA9009AF78800495A290069387D004DE5AE00E735830007589400B2C7BE00622F52005EF8CD0055FEB200F0D497001ECFDB00C781230008
:402D00000A289D004FE91C00C0823E00738F61008897F100ED15B1008C1CA00041244700BC798300EF445F00DDB30A00C93D6200C1716000EFDCF600637C8500A2731300AB
:402D4000C872780095C18400028DFC00CAC7B800D7BC4F00F3CF6100DDD400002F7F7000BB310D00B10EAD009072E100AB8AD7001C3507009FEF5A006011BD000792C900FB
:402D800012BD7B00C6288800B9126D00596E5F006AB36D002FC44F00B3419A00B12F9600C4DEDF005F21780077CA31007796B300B74BDE00BA636900404EA0009CFCAE00A0
:402DC000FCE2BF0003157D00B46FD10093614B0012412E0031718C001F6F23009E8FB80023CFA900A8B8D2004EA488002C481F008C02FF009086DE0010A7B600A15A1D0049
:402E000024C4FB006894E700068781009B0E4C00B5ED3700A1AFA4009E191400C96E3000417C6F00B4A1190031E10B0079E750005F10CD00048AF000F2F07B000E19920093
:402E400076D3E10003FAAF00AF7B990081E8DA00CE7BE600FACFFE00E41B9B0076817000C6348E00C4791A0037DFEF009A2779007DA0C600F938EC00D022C600A384B100D1
:402E8000FCF22C000B9F99003EF30F00CB2DB700C7D70700D5C76900BB9F3B00AB4A3500DE58C200FABA320092286700582B04006BA47D004DBBA500504F06007C29FF0055
:402EC00088679200264B450084430800FFCC460001A87500B6D02A00527ABE002604A700B1DFD600B2FAF4001C680C00FFBC98005A6CA200FCFBF50058F47D005B45970055
:402F00001F478C00EFDC9500D827510094518700BCC6FB00DD8070006D37E900388B2800253A2500336F85008D321500E0D4F000C2F7E100427E2400A464CC00E3E516006E
:402F40002335E1007F0DD7002E81A000976F5B00B54AC6007009EE006F2E89004207A300EB298500BDCDE100BE790A009885DC00803ED6001ACEDC00EC1EDD000F32980071
:402F8000628A360097CD3500C47B820018472300C0F07F009AE61600D3ED0A00F7CE8400588045009180500057B30D0002C551002EF6B4006667FB005C3119004EA6020052
:402FC000165653005A9E1D0055C74400A41F4800FB4ADF002BDBE800225C00007815670073E727008E020600E4E288008D1BDD00A5053600C67E030051E555005F4950007A
:40300000B0DAAE00C73AF200C9BE3C008F250A006BBC6300BC890B0065E25300C975B5009D40C5003B0D740007653E00039A58002A2CE500F9A16F00F436D1008A49070067
:40304000575AD3002F948800D882FB0009232F00A2CC24000863D7007A4C8B00B7C725003D1F77004674760019754A003912E000125FBD0076B4EA001A8F7C0083C827002A
:403080002ADF000012F3100066FAAF00019EAC002AE998005C905300A3EE47002A78F90099436900DB76D600B3004000A93A3E008DC28C0049EBAA004583A0006E373E00B7
:4030C0004BAAF900C2524600ED6D8E00B17ECE005A7E55004847EA003FB27800D8B77C007290C00024BB1800D83B8500283333002C8A5800556AE4003A6C6D00133ACC00CD
:40310000E4BBBA008BEE4C006BE45100A69B170005ADDD000F284B00D29810001AA7BD00F4F79B0024090E0048DDDA00FDBCA80040543700D0CBC500C7020900CE44B4008C
:4031400007D720008B97AC00BB96BC00387A8E00A2E1BC00A1DA6400B76E2600AC416300B1CC0B0055A7F7003DE39E00E4D9F4007E2819005879CC00CA7BE200120B720081
:403180005786BA00DE2A6F0091BDF40040A3440097D6E800037C7900145CD7005550E7006D6FFC000858AE00671B37000CC998009C58EE00181B4A0051EAD900FB918D00E0
:4031C0009D08C700930032002143440018C700006E5B250058084000995C8F004AD1C800BD19FA00FA05D40092BDB700497DA9003AD13400D0103600F59B270093FB2B0045
:40320000D247D100BF903C00A0719B00FBAE2C00EEB3DE00DB89F5001ACA15001FC5E900AB7E900097D11C0084E74100D458B000A3EED3003081B4000A89070024E40B00BF
:40324000C4B0500037E31B002536AF0050B9090072FC4300B1633400E4A50300EEEC0F0095430F00D1BCF100FE52950002B02000F5FAE300449CF0004D3C6F00C11DAF0088
:403280009C7495005DD73B0034011400BCDA0300F428FA001DE84B0021E1CC005B1C7300EFE79300804D7F0023D27B00EBBC2F00415BFD0091605D00A4B9090085FB990099
:4032C000C6776200DFBFEA003CB3AC006461CD00BB8A32003DDFEB00D4C3E5000C0F8F00CB36CC0012ACCD00AFC74E00D0FAC100EAE07A0061A96500BE0A57009C7EBE0085
:40330000B25F54007B7A410017303500958CB400D1A75700E0C051007F417C00E1BFA600BE0E6D00442855005563ED008ED85E0016CAB300E37B0B00BFF37900A75A1800BC
:403340004B199D00ED8B9300399DA40088CF7B00AB73A20082FE4D005ABD4B00AEC4BB009E687A00F462F10075980600E2AA6A00C39A1100B02F7200369D3D0075FBAF001B
:4033800010C05B008E658000BC93A600BC8C1F00C568F6002E966B00C7D59A00E1982C0078F149004EE8B8002F41FC00C06AD9002B94A400202D910012BF8500E84688008A
:4033C00032702300F313CC00708D1800C606C40007DA7D0095EB8100A46D5C00EE3EC900B951CD00FB736C007BEE9200A9767500A0C23B00BD66680058869400E52A7E0069
:403400001FE2F00004933200AFED4B0063F13300841BC800EE5BA400A70650001F7B230022920B0031614B001FCA1C0079145600DC87BD00372E0C00297769006D0EC300FA
:40344000E3C308004D37FC009A751300E35DE200EE0A7900AAA02C00599FD40065F1F800E03A080045977C008F96380005D1AA0015E14A00A4360C001A526800EBDA700053
:40348000B1BFFC00CBC5B60066194B009CECD2003069630064D4830007D055009D5904008F51B90062605600668CAC006856B60040039D0010266400CD633A007AE6110041
:4034C000E91713000DE58C00A095F10093A9EC0042703C001477E9005A219C00B3A99000570EFA0024246400E98C2800BAE1AB0041C262000CEA9B0059CBC400057FF80040
:403500003C62EB00ACE31400D0E5F200E0503C000F168D00838C3D00EF18FB00B9EC650022C576004BB04E004B8F2000EA6A0F005D8DBF00BF0AD9002FEF4A00D7F4790048
:4035400048D9F0005C7BD000E3831B00BA164A0014F374003999E000337DE500CB31D800CB03FF00BC600500F904BA00A10CDF00BF72B6004DA080006611AA000547CF00A1
:4035800066F27000DAF7790084E2860019D99B007A4D1C00947AD6007EABAD0064076C005DDC8400CCB1DA00613E8900FA4327001E0290005DF758003A995200FE613E004E
:4035C000F2AA6900C0A6800035CA3A003FD27D000661E7003264840050BC2C007B2EFC007800EF006BF6F2004EB90800054B690084977200BFFCD80022E66B0076C4000085
:4036000050C1AB00CBBEFB002F9B8A0072270000D45FB70088F7A2000F785E00E4DC3E0040787200BAD76700B5EA14000F0B540053852300A84D95001BA028005228F20058
:403640002681A4004A038F0082A52100F32BE700B2B24000EA846D00BFF32B005D8AA7004A089700E4A15D008FE3530074FE46007DCDBA005A0C030094F7DD007CD29C00E5
:4036800038605C00AB382000F8972200AC697300FB8F9D007029F900079E030078ECCC009129BF0078BD50008E32EC00C5972400D28E9100BCA8A40047BDC20028374100C0
:4036C0006712D700DEFA2500E2003C00695363009FF251005D3389001F6769008AC4C800A77206009C18880046B6CF00A1CCFB006A8FB80044536C00E8166C0070D01B0039
:40370000381A220013845700A4381400A8998300ED34A10054A82300CF7986006446D5004FA7E4009C884D00C8C3D600124BE600000CE500D027F300F82EB200D71A190099
:403740002B697600DCA75E00B07C86005992BB0078325900BA48AF007271BE005BF3A90083F6320040AEBC004B3A010072E65A0049606F00AEE7C200E116ED00A769880042
:403780001D55B7002FE7CC00A1B0F20012A4D9005A2F620060F3B7003262D4009E5C3100F1C924007C26B6000E4A1A00DACF6700A2336100FFA76F00EC4167001C040F00DE
:4037C000A69FE6006F62FA0059FD63007FA00E00B6A06900CC4B7900B0CA03002E162000D3450D008598D500283D8700D0521D004EC8B9001B52EC002116C8004F4BD100E9
:403800000F9F0800849BF7003AB4C3003C7C5000BF412D0009244A002F6006000B0A25006C895E004753800002C12A0073A5190063A6150022616D00CE5EC9009D898D004F
:403840003A55D8004C6C49001AF7A5005EAE8700ADED070039D63500C28F5900F637060023EBCE009276E9008B4BDD00EC0B7000EED534000104A600C8765A00C5BD8F00A3
:403880002E14C600238A70000769A2009B0FCE00B9C44E0009F8D80044A5A50068111B00D566BC0048A2D3003AE3EC00E14E0F00EF1A140027A9E400D991030069D9B10067
:4038C000FD80D0005D696200736211007F13D000D5AE610052BC5200C21DBA0001EA2D00199C6500EADCEF00581FE300750FCA00AA911900A7D08C00188E8100DC3B8D007D
:4039000004D36900F9C6F300FF600F004D7F0800E24D9000E611890008380100D230F2007F92A3000D196900791AB7005C824500A6973800DCF0030082E6E8007BB88400E4
:4039400073AF5C007CCA310016924C00932E1E00EB6DC800ADB63B00FC794C000631C500122AE600753EE5000E6559007E4B670042D29900BEB63D003C725E004EFAAA00F2
:40398000D5304500BB548C00F25E34007A72E900C9651C002656DF00343F8400196B3A000433BC00AF0D8C00D622B9007FED1F00F61A3400C79B9400FC13BF00C3311600E6
:4039C000304FBF009BED3000E685D100793019001535AB00BDBBC8001F0CEA00AB4C0A00D066F400D2D04100E8275000EC2EDB007F65C70019647A002CD091002B74A100B8
:403A00001E5615000018C4003BCC3300C9D703000403370062328E007925DA00763DB600D68453008D55EF004AFFEE00C7934E00A89D6E00511456002D43D1005206F900A6
:403A400074D677006FF4630061CB6B0082FE6500B1176F000E569000F97F8A0001E83A002C4691008F9F1F00A238DB0016F3BA007D7BBE00A2AA4700D628300051737B0075
:403A80001D934700301CB5001ED4A8003F915600408F2F000A6EE700A90D80002A05E600868B67008A23D400A35C5A0053966F001C14CC009FC910004D64F900E85941005C
:403AC0002EB833006B34B600ACE69F00EDA17F00C336EB0063B8D1009F5FBE00FA0D3B00B198A8006D46010029284000FFB108009FC9FA0046A5C700F1786300349D0E009F
:403B0000E9ABA300FE7E0C009FF98F00DB139200148431008F5FB900C0D5E0002799DA009460C400794E1F00DE309500BE1587009551670072CE85006261F9008A622F001C
:403B400061BB060023FF6E0083F4B6003AC779006F52CE0033842F00BD1B0E006FCA6400D0786800D8387200C0E11400AC770400EBCD3500F1461F0034722F00B9FAFD001E
:403B8000D66A1D006EF06A00C2A2440037CE3A008D519400D593EC0048D0D3002D23A90025C9020051C4B400EB56B90027329A0097674400324C85007C5926004723FE0001
:403BC000CC040D006CC655001DFE1E000FA5CC007FB75800902C3700D0AEEF0051E32E000494F300EA3E6200DCECE900671FA20037501900E0CF40006DDC3D008330E200C0
:403C000067EF1A0052997900AF3E560021F4C6006A60D50040390500FEB42B000E4FBB005E85DC00BD557C0056C44F00950B4900297380006B0C2F002C435F003C10D8002D
:403C40007639240079F70C0006B9BF00576C6E0006FE0B00823B4100384F6D00AE07F60008DF4D00EFDEBF00418E4A002A864B00E42E0D002F1EAC00D22FC500F36C0E007B
:403C8000690841007426E700DBE64B00B998AA00D4C2DE00B9C1EE00F0ABF8002E581700C6CAD100DA7DD0006085880022164F007169BF00DF8B7E00B06E1E007571590046
:403CC00097966D008116C0009CF43500D5DB6C00C73C870032E64900C7DBD700216AE80069157E00598827009C5B9000935A5D004C0AC40057646500A42B3C00A41B6A00D8
:403D00006E8DE300D310A9009E56150062F3B5009CACF500A901AD005D6D95004DECD000237716009E5EED004B3B1600BFDA7900B3C8FB005CD458000505070061612200D0
:403D400080768600A1974300EA864F00B4DA2C00457266002C0F8100180FA800668A5D00E15033003D566000C72AFA0005C5060035E59A0035AECE0096FD0200099E040027
:403D80002C64A80062C63F007B7CFE00507705008FB6380058BF4A00EB1B19002E33130001D1E7006030E80030A4FD006AEEA100E8AFF60000298600B802AF00CB9CD30058
:403DC000AD1F64001DA3FB0084B9070023905F00F9944400FD7F6B00FF7CCE00D9BED2000B5EB80074816B00CA83B60002E8560043038E0056531A0055B9B40075E19A000B
:403E00003EEB5D00AA6ADE0097E64C001253CC0053A704009235E3008F3ECC008FF97900F6B3F90058E594004387680037173600423F3300553346003C06F6002E618000DC
:403E4000AE619A00F3B44B003F6BFA00053A8300AA76A7004EBD8300A36D640040F4940009CBF700F8670900A70F560036C9B3002DFBE900489D7900E6AEED0081B5B800E1
:403E80007D1BBD002E91E4006B4144005AF63100B6FB26004A358E00D16B110092F38900858482000882D900780C5500A2452500EF9E8300B9F35300BE183900101F140026
:403EC00077ECA700D7ED4D00B4EAEB008970BD0060EC0500E34D2100432A4A00D4C45A00CF229C00ECA5D50050E887004239520021949300D267B9003F4598001A09240001
:403F00006ECBEB0048DFAF0065BFF300E414670034E1D6007F2A2E005BA34500C99ADE0018033B00AD27CB008183DE00D73868006F7E0E00FC592C00317C820018B85F00A3
:403F4000FFCC5200A7727F007B463A008C5778005248A90083AEDC003A463F00328990000B6C7F000EDA6A00148E9000E406C500A299B6005040E100C0486F009B0918001E
:403F800038820F00EEAF1D003DD49700121848000CB594004E846D003AE51100314DDB005E5A170013BC3A008F89990002441D00728E34001C179900B8C3870018122D0002
:403FC0008F08B8004DD2E8006270C800A1BC1200BB85AA00C2089200C9896C00AD516700488AEE00DA58DE0022D02000F2A18A000E572B0025DE6D009E159600F8C74900A9
:404000001A1A3C002EE98A00BF25D2002B4EEE00ABA2CE00B49F0E009B24C3008193B10059A8F200B3CB31007FD94300CF01E4002B47C500AE90F7001CD13000E85837009E
:4040400017D03E0097C42B00EAEC8E009D673A00A23B810000938700FEB30C001416B000DA8D2B004146940087FD91003BE42800524C56009FBD9C005AEAF8003354BE006E
:4040800014223C00D377490034EF1A00A81A25004EDA5300F1835100BC6677002F45D5006771CC004CF3C3000F7D97006A15B7008D918100863B98003BF7D100F5EF7E0059
:4040C000D0F433002AE14400A8F05E001F7179003E2B51009EBEE1001D947100BE2CEC00E7F7EB004B3CA700A3025E008296930076442B001650990054FF03007A9BB800E0
:40410000FF32940015021A0005CD1600837839006D1282002772A9007FEE78000218EC002FAC570002B356003928D500B2DEB700FEAC7800CEBA800071CC83003280990050
:40414000952613009BC00D0086288F00FE4D5300770B2300B6010E00843B2300835B3C001A09E200F1CAD000340D160071E43900E1A4E100861E56006FDD4A0068429F0014
:40418000472E0400D0943300BC299600C856C00044DE3000C26812006B04D300E9B644003484CD009091C7004A301E008655D100A700140097D0BF0085867C002CED24008D
:4041C0005C32E4003244090031EDE400F718E0003665430038E81500116E68007AA80500AAB67C00DEAA2F0088AD40002225920007DF6600CB87E700D29DC600CE56DD0020
:4042000033942800B2B7FF00C21969002E36C800E38489003783DD0005A4F6006A0D4F00C4475A00C053A7005BDF9C0094DD3900F193D5005254B300A59469007246070019
:40424000F033F400DC574500CB05A30073AEC7007842980053611D004D2F4700BE066E00EFD5E500E6BB2900C4480500ECEF2A006EF2D700AE4BE400ACE1EF005039AD00ED
:4042800013ECAD0009C7A100E05F4900A6F55F00D9DE74009FAFD20072E2BF0099AF58003C51240085E0990067EE6C0044EB8B0023CE1000C1A3110048B1C8005AD5A90028
:4042C000A9CBF5001D4C3F0074F1EF0068319B0026897100A5E89600374E6D00DAAF7B0050BF1D00CE784700074C62004CA9D7005D0DC600279C75000D1DB4001214110035
:40430000DF121200FAA81D00CAFC3E004703620047A2BB0052B0290031533200BF6F5F007C8BD2002A046F00D367D4001796310028175000DF997500EF5BF8002567CF007E
:40434000EA15EB0000FEA900C393130007F01400B2048100D2C9910098A2A00064863100EBB2C600F8BBB900BA92A2008521D5009B694700FE02D300C3DDCC00B68F930046
:40438000C1EE2F009BDEAB00FB709A00EF5DD20089DB5C0099B548008DDD6F0061E5800050606C003181E1005C30070021040D0028E6F000641D1800E3AE1F0097764A00D1
:4043C00041A2BB00A2690C00AB2C6400E84F6E009ACD4600A3B29E008A287A00FEC37B002DE16200C3E8ED009AF13C001122360042D6F10051D2EE005226EA00E9E2880019
:40440000150E330022108300C70AB700F1D9B100836CA10086784C00F01C910056E6770047A416006914E4007AA20400577E2500E86C800059E2E800B7D7DD00B2A15200C1
:40444000CF92C100CACDD7006E5F770057686E00B08E2D0087A97A005FEA57009C798A00747F35009FCBA4009A862C0061ADCB001E03C00066EDEA0077C76C00A0D6DB0073
:40448000EEA77800C6CB0900A5E3C0009D377F004DC39300CBAB63006507840031D177004ED54A00030CCC00F4E63100F1BF6700AD111E00E6D36E00B0021000F614EC00B0
:4044C000BA1F5B0088B4990025C8380015710E00F06A1F00BCD4880078A6DC0090BBDC00001F6700CE792600E6F021006C248400A40694003D9D7E001FD4F400EE52EF009E
:404500009C381600494322008FCEC5005B106900706800007BA23900B05E0100A9A64600F6642900CBC15500D868BD00E3242A0021B04300B3D0D400B2DCAD0086EB510021
:40454000538103005449F100EC0D1400D6A76B00CC63A100F2DE4A002A165800ABD05800A9C6900021DEEC00A8D6530016FFF8000195E3004BF9B900FAE3D400730D2400F9
:404580006F516B00A345C9003757020097A7D0003BCE1D00E061AF007B570800F244E000C675A300C2A77600DC1315008D00820089D09F005666DE00565D87006C26DD0070
:4045C0000CC960009809DF00F05F3A00F384C000604DE300F2EDE400ED431C00A93D6500C1C94700E25B3100E1938900F18F5D006789830037C58400CEBC7300C8330D004B
:404600008B01CF00A3535D00714A1C00AC925E0059009500D5F57900B9F59E00BC849C0050875C00AF654200CAAAD300976339009FE59600AA707F0069982000F06FA80022
:40464000B4DE2F002BDA2E006EC6E4004B5DB300572E0C00694D56005811030063B4F1007FA58800D7A61C001507660043924200A157FF00C6F55700D7E08900A4368B0036
:40468000CA3BFE00D1886D00153C3400810F5B00C8D03A00E3E6CD0081E90600F13E1600B1A53B0062D1FA005CEF04006637D7003BF827008A4F9B00495F74006905FA00D1
:4046C0001CCAFF00EC61FF0070AF8B00B4BC4A005F01BF0003328C0019D4F9009C7E97005E3E2F00DB45F4008D44320079F2CE008A2E6500677AF6005251690096B7D30073
:404700007BC87B0048FE8C00815171009B2D28001EB3D700DE91A700AE288B00FD5FDD006DBCFC008C5F1E00906B97009EC66B0078688000AB397A00B9FB78001DA6E4003E
:40474000DB8D06006F9A5E00A682120070D604000F45840082078D0014DDBA002CC3BE001025A1008CA1BB006E762B00FABFCD000C5D6600B5CF1A001AC77A0040C0BE00C1
:40478000475A55000EDECA00A6C6FB00A08A74004021A50098C34A00453EA40085731900CF1B59007324DF00AF6DC50072047E0068C3910060A76000F3CE840088EB0300F9
:4047C000D4E7DF0090193100BFE65900B1F465003E2A9500AA0B8800C77177001D010300486CE90015DE750017572A003612F5009C08430093E39C0029B1410053FA0F00E9
:404800003F75F9000688430024CE4800ED2A7B0088EC5300DA68B100C95BBC00266C9500AC33AD009FBFAD002205A0008EF255000034D60065506D000C0451007E170E000A
:404840008CF5540022AF46007D62290096E20E008388F7008C726600BE744D00A7B239006E89B4003AAB5A006BCF590067108F0049F50C005A4FB7000A2B6700D5324A002D
:404880003B00F500321C5700E188C20054E33F00FC0DF50000B85B0092DB13008BC0BA0065C225008EA0550049A2F900CAA602003E427900CD69D200A0223000B31E2200E1
:4048C000FCCD7900938D4300BF32B0000566EA000A78A800D3E0CC00398B8600C2AD26007D506900ACD2B80017AD7B0058F54B009546F800B90D0A00F7AAA300C684B80069
:404900000DB61E00A105CA002B7BDE0087324500D94B00007407DA00DE8E940026A104004E33AF00BAD84A0083BF150066301B000EA02900437411007E20CE00CA524100E4
:4049400091C09800338D39009021220045AED000998465003D1E5100F8A4E600D2026A00D44AB900C54E8C0097DE4200F42D1600707A6A0003D1C1005D2977001759E8002F
:40498000B1174A0037EE6800DC65D6003E4DCC004CD4BE009D0A17009E1CDA00F04DFD00AA7C160005B7F300133534005EB0B000338595004F71B3006DB2AE003E81E70028
:4049C0001B6A690033A6C400B2902F0003324700C9D64A00BBB22A00C75952009BDBF90080B343000BCB0F00FAA2B800E205B300BE940C003375F400FCEBDD00D0033B00C9
:404A00006A478200CBC0B90081F8E7000F646B00890A3B00993D3A003AFE550045375100F2706900EF8C970096398600112B8000023C1200571011003BE6A9000FAA33001D
:404A4000E9B97B00B1C098003AB1E000CEB5FF00D88031006167F000463AB300F1774900B8544F0027F9E1002E951C0056A4A000BD25600071E8FF003A08BD002741A70021
:404A80004BE1B300CF873C00FA30EB00D53344007CF8F4007645EE009B67800005C481004D1A70005B30340010C4B500BA0D7F00419CEB00C3B3D400DAEF83007CE42700FD
:404AC000B4AC4000FFE6870068935600A45273005581860090D949005DE9AC00EDEDCB002B4DEF00DF8277009604D200275017004EB6D100E47FBD0084FD750082979E0070
:404B0000970D0000C0DB550096274A0090EB69008C2E1800627EF900488BE5003BFC340063F747008D1B1D0064F28C00A7060800032ED400C6D4F3004A4C3600F2B77100B3
:404B4000AB62B90029193D00CA3BFB00AC6C5D00ECE73600F23DA300034D4F0063EFA0006F5CA90021CA64003131CF0072814F004F2B800016142F00AE4A3100FD07EA006F
:404B8000730E450025A04500EB2F4400D6071D00EB34FE009A84F100F51DD3004CE0CE004F3B960040161D00605E7C00B6D73B00058F6A00BF3ABC008250360002C9C100E6
:404BC000FD232900BAB56400C28A9B005922BF0084AF47008C4B3200D88F4E0072B495005629E100C0F39F00D472BF00D2126B0061239D007DC97B0025B99A00440EEF00E4
:404C00004F3826008C3EEB00DD79CA00C7F19B000AE729003E65C80031863C001A3DDE00EEE44400EE476500F3035A00B8B35A00A529830060A55200D065D0005805C9005A
:404C40009AC4C900C5E1320072F29C00D4B237008BD6EB00FAB2EC00D1810200F868BD00CFC5C900CF26CB00CF9C75002EAB5900E2A01200AB7E6B008B628F002737C6002C
:404C80006EEC090043C4C800766DA60077670E00A3D1AA00056722001C1BFF005AD1D90043BF9D0035B2DC0044628100EBEE3E004411250057161C00E92EEC00EE9D6A00CC
:404CC00060C8360022928F00F8B6B1001B7C380042785100E25F1A0087786C0050E3F60091376000DB1C37004A1DBE0067B2680026B7810029CC7400EE4FE900B7642000C7
:404D0000B8EBB2009654C3009C83DE002A7FCA0068B6AE00DF0D0500B47801005DBBCB007AD0EB002C0AAE0016E8C50010B64300968BB600EFD3B00053BC0B00CC2C3600BE
:404D4000703837004DBCE500F48E8400702E6D000AF1C8006B788D007E4FC1006DB743003F036500FB7A7D00EFC0CF006FEB8B00A6784C00BD74F70081D0370053D42200CE
:404D800001C5BB002A783F005781F300BA797C0061246A007E652900BA55BF00D3A60E00F947D200CE8067005949D700EF30F00033B72D00236BBF008F2EB00043FC7A00EE
:404DC00063F5BC00338BE500AF60E30034FBC400484CB8001564990043B487001E0D8B000731F600CDCBB80012A3DA0070976900A2D65B0024CFC500B3BB85001AFE7700FB
:404E0000935CA7009D651D004D253E0022B559007CB1FD0052D94B009441B800CAAA1B009F491F0090C16700F9396800FD8F57009290C10011E58E00ECA0540067DC21003A
:404E4000A26D6700A5CDE200AD653E0051898F001854A700A160B4009EACB70056956500CBAF4500AC309400339DC8001D059100E7519D0002A13400DB3D37006F85E70046
:404E80002E25030030BAF000AACF66000D875000E5ABBD000304D500362653005EA342005BED66000100D20002A11500E29A9500E0DB4200A0A5860050E4800072CF1B00C2
:404EC0004916DA00A862D90017C6C90092BBF40081962C0000614C005355B600770D2900F84642004AE32500797C20007D28C2006E311900D25D04002E5EB4007A89140024
:404F00008E853400C6DB1E000460220028D673007032D6008F7C53004520840054BAC000FB037200C1BE910012EF7C00284809003ADE0E00AA66D1007C0751006E4B850058
:404F40004560CF0047D99D00133ACC008A4D6200C486F600F46CF700E25401009E9ACD002E6EBD00EC2299007E5B0400688A2D003F561A00451F830024F9500018E95E007D
:404F8000709A9600E62DB8002D70AF0059320E00E90C9A001A5F8F008CB18C0023CC46000387F400F799F300F7F763002F906B003C1D030044C60F001CD72900A57C6D0071
:404FC0005A56980048C62C00A5C3DA00261C230054A15C0084725B0055E18A00317CC300DCCECD009F0F7900232B4E00B6499600C0D5AF003D70CA00C0A0B3009FF6EC0098
:40500000707EBD0024E14A002BE359002C66B500AF718A0015C809009D75BE0070D4BD00AE1C3B00498E8A00798DE4001BE06300E345E600615AE2008F202500FE8BAA0007
:405040000492A600869AB300F7674A00E9C96E004FA061004CF699000012EA00D8BD4600683BE20083804900EDA14D000EC45600CDC5F8003D5E7A003F4C3C003ECBE7002D
:405080004330C000BAD37E007077B0007E9E3D00A21804002E973600EB79AD00D50EA2002755E000EF7ADF00AC9A730039047B0031198E00DBB98200625ACE009E1A3600F8
:4050C000605D4C00B7E74300BE1340007DA14F0094B9AF003DC89800868D4F002B3E370005A5C300115565000F3D12003193090017B015008117320092598700B6600B0011
:40510000E93FD100ED655100BCD0F900DC785A00D20E4D00FF55E4007280CD00EC1B06001713590051235A006A8C1800248508009BFC6D0034EE99007B93CB0032740D0014
:405140006B8FB600C611DC00B65CD400DBA165007749690038219C006112D6003F7F16009125FD00FA45D100DA514600E08A09001315BC003EC919008426B70061E6E40093
:405180006626F4004666D9008802B5008486B000E4D36F0041BEAE001036E2000476D200A8A556008B0E6F00B541BF00D75640005EC4E100AA940B00746AE400F3526F001B
:4051C0006E93FC009AFAA200A275A700E16C9F0026F5B1008C900D00FB6EA300F54744000E36B4009A8182002C965A00DE26A100F1418600E16E0A00C9A57000D9924B0056
:4052000022143000675D9A0056D7AD00ABA8FD00A4958900F1EA5F009B2E3C00AA24D2006C6CDF005096B400EA0006002C0A15009779070078BABD00367CFA00E6D33D00AB
:4052400050689D009E34AD00F1C4E40068223900C15B6400B8FED20024EA9F002CD6F8006D24D00054FA5400EE2690009EEFD000EF058800B2DB1A00CF068500BF091000F6
:405280002493CE00189FFC00C13E61002AF3A600E2240500A7065C00D14E1400631D8C007A1B7C00D113D100291D0A006F60210016AF1A00552DCA007EAF7D00E2586900C2
:4052C000B7AA2200F686A300C8370D0052DBA9005C86FD009F74D6000F26B300851C58004595A8002FFA1700F99367000282BD00616FC50010D7F60060185E00D69D1C00B4
:405300009505AC00C8B87200F72E570039226D00D1B5AD00BAF51300F02D9100142E35002E3A4F00EEE1AD00BC7B36001B007E00A13DE4003A71DF004378EB0087E65700E8
:40534000533EC900ADDBC400E79B94000664AD002808700082229F0030CB0200A70F8600558635005924E300E5DD6E00B269FF0005E42D00B225F4000D9688003B7EAE0011
:40538000AF39D6005DDE3D00863C89006CBE0600BFDEE300683E4800568FF7002AB20500D3394500C1B78C00E58EDD00EAAFBF005084AF002DC34D00263BA8005CDBC40050
:4053C000E1D3AB005D2C3400AD7D1E0049416700791ECF00C8DAC700304E3600F935C400F49FE500564100009ABE7D00E27A0100AC74B1003202BF00C18A04009095410029
:40540000DC19A100164BBD00E1026300104C44003E6BC90073D4CA00AC0095004518AA005F424700C64B6E002E2E7500987031008290C0006442A2001B689000969ADD005C
:40544000709F70002E4081007FBD070096446600835C1D00F2B37300579E3B0075F2A100029D9A003277F2003D4291009D8BE50060183800564807009D9496003AAE9B005F
:40548000550BA300D2609F001433E200E3DFB1005609FD004F64FA004D799F00AA44A300197FDC007329C300F8B439003ED97300F73C160013607B00B45FE200F3F27A00B0
:4054C000F9C5AE006FF5C4000855850032782E002D2AA700CAC0B1005C31F400DF9D5200CA35F400A9D1F5009C4C0C00E03BE400E019DB006E8355003B8AA600DCF01F0011
:405500004AE5B8001A353100FD7BE500D21590003AF53200B9ACC300FAEC6500BF856D009F8F90006AA59B00C5331D00ADCFAD00721F2700D05DC500F4ACA900049B030070
:40554000855882005B55CC0019A87C00BFF7F3003F4DF200168C5A00349CEF0002A1E5009E0ECC00F639D000ADA265005AC8E90020DCA400C2A76A00C5E15F00C0E66200F3
:40558000AE52950006842400CC6F4C00E0121B008C97EB00A1E866002EFF08006E8029008AD1340022E955002B97C700D3892A00AF43F100F38CDC008920BC00689C5800CE
:4055C000007822009DBB860050A60800F63FAA00CD59DE00A5F5C100AC1D2D0067D16200D61D9D005CF76400618FFE00CEF7610085892B0098B1410054FFC800EEC2F70087
:4056000013F2CC008F19960087812C0010EC1A00580B2700FEF7FA00557CE6002C86DD009A5D8B00C20641008F5C1400B793DA00069DB30019E5560026D56B009D7B360046
:40564000F8E0A200B1FCB1003F2F21005B324D00FBAE6800A4D82300F25C5100A6ECEE002372BB00E268440076BC2F00A99892005605B900989160000FEC6F008FBF29008A
:40568000BCE5AE0057E0A3007EFB79006BF3700037CC340066677200B2D5010035412F00EC8CA0006A2B1F00BA50EE00B0E36C0021F2F800CF332F00176F4F0092CEBB006F
:4056C000BFE7AA007AB3A500C375140026B7D70076C5A6009ED76C009070D700C673B100F27560003F887C00A9948B0092030E00F6AAEA002A5F9E00FCC82900AF38C1004A
:405700007BC67A000B37E400060A6F001466BE00C487F1000DF2D4004E44F70082DED100D2DD45001E594400B1754D006817D700887DB4000726D30001AABC00D6104C003E
:4057400095DD1400F41B1A00155DBC0081210E0077BE710061B5B800DBDD6700A0E2F100DB628300E7EEEB0000328400CE690E009919E6006E94BC00C8768D0079D959004F
:405780008E832F00CF16DF00B2C27D00552CDF00EBDC44000414E20065A97F00C179DC005F129400EAAFF10049DDA50098CA8D008980830058AD6D00E09E04006542170065
:4057C00076910000A86ACD00DDA35E00EF5B13007269A90080E626007DAC0E0057722300F8DD4A00BEBDA200923D6F00FA44AF00239F3400FE3D3B006E99BA005A217500D1
:4058000034F14F0082B29100B35EB100C0558A0002223F00FE5A88007146BB00BBD75100119DAE0049AAD700D7CAEC00225A7500F3793200902680007EEEEA00BDA61700EE
:40584000B3388200FD190500B5C52C00E9F18400DF8A1F00FE5F9F005FA64800D4200500EC948D006F583F00E74A960074EA1A004BA67600D8D670004AC922008FC5510021
:405880000F0904007E691F0019995B0053712800DE8C46009A3C96001D7A6A00A3209B009C22F800CD4E870088904A0094BA93007A833700F151F6000834D500905ABE0092
:4058C00094BEC800DC7C0E00B42AA1000C6F51000A64BE00CE2F9D00AC6FA9009D223B0002E15000FB666F00F0EFD6004D93E500A82FC90064934600E84C4800F20DF7008D
:405900007776AF00A089190074A50B003571D600EC62CF0046150000DBA11500C286D10074B94F00B789A300C2675B00704208004AFF5900BB7C7A0064BBBE0041982B00F6
:40594000E00442008635720079693F007F6931000310E400C7EB6900E6AC5F00683F3A00EA785A00993CEB0039142400A067C500C3B390004E6B4900F25DC50015B65200C4
:40598000CD85C2000F4E95006ED2AD00C795EF0023A0800046D00000026F9E008B1B49000F615A005DD49600ADCD0500C9C9D00069153800FCD7C4006C18CB009C91AE0069
:4059C00019B41600DF9CCA007C58CC000871910070D611005A834600FC70BF005D6FD100BD4313000C1426003CFC7300FD142000BB2AF500B01ED900CCB3F800BFE8A70018
:405A0000372750009ED14200EC1759005ADE1700B4E04100E9C86A00293E480086B53C00942FCA0093183E00AA9580003DFA060046AC5400034FD500DA1E0800702B840048
:405A4000D0F587009701F1002EE5EE00D26E150058BABA00632E2800FF58EE0037CCCE0058F3ED00C1544100B385C6002E3B8A001A7F6B0080A0FB005B2F8800E787CD0075
:405A8000EED0A800EFCCA5006D46AE00BAB48100FACA04009AF6240004E90D00C7D56100814AF100207B3E000046A0009071A900C0F66B0071464700A6719100FA2C090042
:405AC0006F136B0055D94C00273F9A0086DBFC001F88EA00F575A400AF6B8800AB51AB00A8DC4C008D95130021791300146CC300BF3A650030AD2D008F0BA300DC1B7500F4
:405B0000692BE60036B11500F039C10042E86F00E820D800339DDE00EC250000FFB90B00896AC00070CBD6009E65760058A875000D6B940035913A0099CE6100A2DC2E00D8
:405B4000AD4F8100EE6C3000BB383F004CF40B004CA8D7002D99B900BBA1C600DDC6ED00D005FC003AF435009B971700ABAAC5006DBDBA00B13C5600583F6B00F3FF3900BA
:405B8000EF9150002C47580002596C00AA882900F4CD34008DACF200A9B67F0023CE1A005CBAF400CFD27F004253AE00BF0AED002C089E00A66A0E00DB3A59008B6233007E
:405BC000C591900011BB4C0070E57700925FE900B148B900BCD09D0043F0990028994D0076E3F40025EEC9007021C700D19D0C0006096A0034D5590070C256003B67340018
:405C00001F31DC0053CE750085F858004D1D9600507779002201A60002FD4F00F97FA30059BAAE0026945F0037162C0038EA9A006F17B100C1F0A000CA1F180027886200B2
:405C4000CDD63A00907342003B9FB900494CD900D82E09007328D500572CB20033066D001249290060C2C000F9A5CF002BAF7F005C68420089B66B0045B7A500D0B7CD00D6
:405C8000472C6F00232031000A165500A25E1700FA5F6500ADEE7D0028555400DD1F0500E723910056BC770082CE750030EF2F0061F3310091C5D60095B0A200DDE9EF00D6
:405CC00007CAC9005D287B00D0522D00414E88004FA0D40052B03C00338F23001FF2EB000D8471004DE38600EBCE270046206E00765A380038B4CC000799FC000487B400BB
:405D00007A60B400DDDC0D009AE4FC000845320092F54C000933DC00B5D261007D7550005E9D0D008892EE008552B00024E4D800C5B3F500A87E3C0065C76800386E14006D
:405D40003586E70000A3D6007194D50020940F002393A000C6185B00FF2A1A00F36247007E94BC003E1C0F00F6C1B0000FD4510081E96500399F1100CD0823003F24870091
:405D8000CBC39400EE8D7000CB0A880067240A0020677B00E050B2000BF82A00E5B5E0002B4DF9009E085F0076DFF700A1E0EB00E178BF00135FBC009D493A0024CB8B004B
:405DC000C4AC240073B487004A38770052A6E800B898A300163FC800574C3900E55B1400A9396D008CC5910025D12F001F154A002F5871008BA647003BC0F800F8ADE0008C
:405E0000BE5AD0009826AA001A1533009F441A00F86AD5001BF7C500F03461001C562600A25FA200111E970012BE0E00C72CDA007AD52400E1189D00792012003B089300EA
:405E400045B619005238D100E7932200E210F500AE255800BE3152008E9A0500A9156D00B2E31C0077E6030097D0C9007D2C4F00624FA800BFB39C000C9205005CBF3100DD
:405E800092EC180048A62900D0CA8600280733001854BC003022E800134437007DA0FF00A1033C00CC8ADE00F3806000E88D9000C0C9F500BA07D000027B1100A3F8210062
:405EC000E728DD00AD73E6004DCD760079370A00A22C97009DB21000E05C5700DF8F2200EEF02500D52D4800C43EA900C740590049F78F004A89A0004F3BD5006FB97E00E0
:405F000097BEDC00614AAF0003BB910060D02A00F91F5900C68E3F008FC43700C1B092009D4AC300070D5800F9B8E4004C100B00AB6DA200F80B0C00BA716400A3ED83001F
:405F4000CE69BD00A92346002208F70082E86E009EE3A300B3F87300111FF700213D52009F04A50006CF3700E2FA660003939900F2FF06006CBE68009F7D470022465A0096
:405F80004373DE00F02F6200B6B25C0071F52F0074486A00E7876000AE372700973299007BE60A008FECE300FE19D400B05DD400FB0BD40019704D006666D2002F7DE90099
:405FC000C389E500B34A5400F0BC0600A38FC500E44E180010635D003F84C400A5097100E0FEF60006040A00B2580300DE5E3A00F49A18009A4EFB00149A440063903E009F
:40600000A7EF220051B39C003EE58B00D5A7D70022E77B00182F4300326BEF00D053940091D6040066F98600F807A400CD585500C501E200E2A9F400DFBBEB00C033D400D6
:406040004BE4DA0071F8EE00B1B998005471CC001BB203006FE44F00FF9615007C708E00290A8700552F0C0058A33E00597F3A00F6B0E8008CFBA90021A99800C95B480076
:406080009913BB00F5200400B91EC500623324001F34360054471500E465A9005CD9E700D58F9C000C00EB0036C73900DA5AF7008AB4B4007E33B8000B252200435A5100D1
:4060C0007010400014790E00E5DAB400D45A4100B0F6340079D2E50009E57D00AAA69B00FF840000CF32A200742A4000235D82005A0D98004CB9D6003C63AC00FDC3EB002D
:4061000080606400E7F05F001B707500935277005B05F100E14737007C6D580057E7C400803B390009F7C0003638C700974DFE00D0223100FC00E1004A1D5500B5E49900DD
:406140006009D5004E1FE600AC0D1600D1D55100C7F71300C058BC004589AC000D64E00062B4390072CA8200BDD99E00F778D9000FFC6400FCBAB6006240B40092493E0085
:40618000E1F2C200F87A4000C651C400E758B7008560AB009F947C00F5F4A300652F8A00E727C6006572360089ED7D0009A53700B165ED0065BB2A00627DB400C0500E0027
:4061C00076809C00F5971300C57CA1002FFE2C00AA4F21009D31660027104100C0EAD60005CA2E00BFE53400785DFA006A369800DF88D300290D0F00747280005C63ED0080
:40620000F44F18009F406300FA8806009DB1F10093809D003A35330056608000919150004EE592004B4B5E00597C2D00C999C9002117B9008948580019CC1A002AA416001D
:4062400087618000197292003A879B0032762500D7BF17002A9DB70033D1420088A495005961D500762E8B00A8E2150046BB6C00203B84004CDA0800CBCC1200F66E180042
:40628000F152A9008D6B8900E0684000BE227A00720D7A001F10E4000B122C00C95118000512D4005F3C9400B645D200B47AF6005C5B460023CD1E00CADB8900DF679100ED
:4062C00085BEB400F982F200C67BCB001B42FA003BCB18000B503C0072CEF40009D4E1004475500058A3030026A7A500EB2E2000FBD52B00F80BA500E70EDB006F688900AB
:406300006E12DE00864C0700B163E1001D7A3000D1AE25000EE65800A76BF3008711A50090FC280047813A005CA31C00DD1E0D00D8DBDB000A91250089197300277FCF0087
:40634000B9D43B0059B0F800A756A4000F66F100BEE3D2009A18B500462E4B00C5030500507A4700584B0B0048715500ABFB3700E0451F00C3BCB100842AF200E73D86007F
:406380009C041700B1C61C005C8F3700EA447300C25911006FD4DF006C8B74003F7AB80015FD1E005A199600FD35DC0023A6EC00BECB3800A959E400A52FAD0025581900EC
:4063C000C6007E00AB17E50099C75000FC205E000B4E370064FDAC00FC1E7000D0CB3B00C123130035DCE500D10F6600E17B9C00003A7B00D6B7A6007F4B88009EDB490064
:406400004B21E900063B4800FF79280046BC4F00F67A1D004D3DC800B78CC800622B1D009661E500C9B0F300C67F75006B70E0001C8D2A00BC56FF00FBE1D900C10C8D0049
:40644000DAAC920013FD5E00811C11004FD67A009F2DCE00D3E4E6002B5EDF00931FE700A88D9600072827002607DE00507B8600AEDB6D00AAB8350037A954000DEF99003E
:4064800086880B0090666D00A99BD6007AD3A9009BEAB0004F1398001B0058005EFEEA0023B143004C917E0024108900C9CB9A00C0119D00D334B20003B1FC00C0CEE300C3
:4064C000EC1CC2000FA7890065B36500E132CD00B603BF0046986100D73D4F0013B6850000D42E008871B0007A4F16003EFA0A0037CD8C0034A99D008CD25C00F46478006E
:406500001392EC00C1A4A800E4425400EC33F50034FD5200D5D32400C3937C00A3467900C1739A0039B36900CED400005668CF00FE7F0600E0F70C0064376000A03B4C00D2
:40654000F236CA0040CE9E00318B2400ACDE3600CCF14900276DB90044CB2F007E163400E521FB00F7C3E60024D9C7008470A90065165400629356009F84FA00DC705600A9
:406580000A2A4E00B0D1F80094A50C005FC6A1009723E4008758E700E385E200F01D840048B6D900A682C40027588F0051CF4800B7B3D400D73D270010E2F6009AC03E0064
:4065C000BACE5B0031B46C0013B1C1009837630077710900FD0F1D00AFBA7500FA44FD0083E45A006ABA4F00E741CC003AEC730014F5BA00A3A95700535D05008378DC00CA
:40660000A5429600C71D59001D581E00680EEC003FF6AC002FC53700EE9C3A00BC652900D60B390049DD30003CC9A500747AE20031736A00DDC41B0084007400DE50A8000F
:40664000C3DA6600147CF1000655EC0076BFC70038FCF700FE724900343B6E004550E90034115000E2592600506E1500460B2E004233910014A981007E61FE0088186000AB
:4066800016EBDA002EFDBE00AE497100605C0D00AF02A900025D74003DB2100083806600FD77AB00BEC65A00DCC3FE0099B05300755CEA00BDAC2E00C0D9F700528A6E00EE
:4066C00036683800167E6800917DF4000788880054E63A008529BF0065E612001FC9210040551200697F980085BCAD0025066F005B11D000E480DB009046D60012AAE000F6
:4067000042021D00BBEE470050005700D3BB0300C6780400AA341B00FCD1390082B7A000D9EC6700EEA4B600338B2E00BE3F1700081C5E005D03A400FA3A270083B2140018
:406740002867CB0043095E000BBE6C007BE48200D7A72600E48528007F21CA0091511600B14D370038BD4700A4181F00D4E440003484AC00C5ACFC00FA09B500CD17E200D5
:40678000DC3E6000E26B3000BC397400E69F2D0070E628008E8EF2005E27D700DF2BD1003BF8BD00AE25A8007EB15D00964F9E008B2F0D000735340041033B006DA9980026
:4067C00081856F008E5F7E0063CE96003789FF003EE4E7001AAB93004EEFA200BEEFA500ACECEC00A4552800DB7ACD0050F85F0043BE7D0003D5D800DADEA5009A8141004C
:406800005A869200016E16000FB47100FEE25F00AEEF2D0026E53600C6BF7E004BC40A002130DF0071DD1300A0D57A006CE91700CB024B00B2C66500FE7A7C00B079480081
:40684000195D4C00D5286A008180F7001869DB0010EAB600694C2A0092A6E100DAB66F00EA089400CFCD6C00E88378003A37C10091151200F8636E008139EA002904DD0022
:406880008A84C6007ABD8E007100E20079BB5400766BA90074109C0067B1E50051CB5B00206FBC0000E0EC0024E30100F3B81F00FC12C0003B253600DDD33D00190BBD002B
:4068C000851F7E00FDA70E00C0443300DC62FA00CDB59300AC6FD200D66F4000DF8DA700F9F98400122F830004E24000A90DEF009F96C9006B4F0E00E15E3700A0EA4200AE
:40690000F52C7E00B627F400504E090065CD64009458EE00527D4600F3735400E0943B001F8B9100A3AE590052A2F300B6EA5900DD56CC0034B64E001B03AF00C0C23F00C8
:4069400067F79000275BBA0031F34600289CBC002CD55400A0028A005C139F0093444D00637B1B007F0CF700DF527600AC7D1C008310C800D759C000851EDE00D8E68000DF
:40698000A00154002ADDF7009823560051196D00B28DEA00EA746200FDFFDB0050107A00A9AE7D00D72B14002C1489000F71F2005BECA000784C260059721D00D2851D0010
:4069C000998B650019B27A00CF9BAA001AC01C00B6623F00C782DB00B598C100FD1FCA00081D25008774E300540F77008D88A000AE5EA9000F03BD00D3605100D4340A007F
:406A0000310FFB0000C0C400DB848200221D5300AA575F00145ECD009B68F60070FA4A001354A8009C2F1300CE1B290015F59700D0FABE000102D100F07703000C231B0028
:406A4000E627C7009C44860050F9CE00FE0D800012FAA7005BC8DE00ACBC6100AAD5C700936CE300EEC477001EB71E005F996D000B800D00572A8A00E75BB7004897F900A0
:406A80006EA1D300F31E2300DB670900551FFA002CF8840069F79700E955B200813B0400C1409F00EC6E49008B9CC800E3DF5B0057DB8600C0A5730092C2A40024B75200B4
:406AC000BF341D00387B940040A397007CC4C30094B8EC00C97A6D009BEDA800CC669E006B133000EDD71E0046DD9300280EE7009736C00004E0E40097D5AA00483D870000
:406B000066006200B69277000604AC00E13C0D005357E7002102F10004745E00899A04006154500073D3BF00FC5426007D6B2B00BF6062003558F000F35D2A00D6888C0057
:406B4000C9F40200893FEE0050B3C6007C8A2F0087733700FD78990001DE7100886F4500CB690800A8C15600099CCF0043499100DAEF75005CCCAD00C60E7F000D8FC90080
:406B8000ED824C00A0320800C006460060F2D500512955001584E20004859E0088A4D7001A325F00FB1823009796F500AFDD5A0054CE8600B2124F00C8698600A7EB670045
:406BC0000C9CF800E43C8F001F19DE00D84F1C00F9F7560089870E0094217900EA9EB30065D8660044F68D00D3885400662CB20052402100593CEF00EACC9900A5706C00BC
:406C00009DF5DA0094B63600339E5300BB9454002DE3BD0078BB6E009E73BB005C422E0061A4CF009256CD00B44C1700D9DE0400C5F3830062628800857CF0002699FA000F
:406C4000F45239005E049700C3397000D3183A00DEE758000085BC00CF5612004F370400C6718D0052AC7F006C977F005B82EC00239E03006EB9A300BCD26300BD581800B4
:406C80005BFB35008EA1B5001E034C00EAB0E2001C3770000680DE00CC0C05008CA8B500F6553F0060628900E1E041000FF4A200E2464400B537B0005FB1DE0075F1670050
:406CC00025A284008284A8000BA6C600163EEE0019C09000FFC1AE00EE635D000B08CA008FBA5E002E175A00811BFD00CBAEA80009C3E000DA762D009AC89A006B70A100DF
:406D000077F20800CEDE4F00970F60004DA9890004A00C00E286E2006B0F8800E0E7D000A068470020084D0000AE7A00EAAD5A00D5ABC800ABA9A5002E2168009286F400EE
:406D4000C8BE5300886A950044E1F700BFD81F007AC15C007F6D6C00F51F19004B003300061956001CA76000E4B0BB004A2A5B00B3A7FF0020992A00DF0455009454F10044
:406D8000984E9C005C6D6B00C8B84A00742D2B0094626C006E256F0047E6D60083D9C10023219500242FB7008BE49F0099D10800B4020B009D1794005F454700AF3D35008B
:406DC0008B740B003D9DBF00F1DDFF00597A1700F8E01A00BACB9E005DC32200BC1FE80039DDDB0084B36700A567EE00F7D362001DFAE4002E0BE3001130E300AAC8DC00E1
:406E0000A6C724007418BC00BCDA9E00DFF52F00967A1C0095737F005A35840032623A00D82A230024BBB100E55C8100B4F2070036576500764D60003FFFDF007EAA3E00F2
:406E4000AE0C880087847C00DDD02F00679E5A00DD60AF007AFE6200B3C7E900252032004F06F5000E951500195D06008764EF00469407009E4B8D00FC4CCF0065C73D003F
:406E8000DA593200EC8A4100C222DC0066668C0065173F00EAD2D7003BA026001CB4820057AE67009EB54D0095095300188E8E00B52C2B0036642000E95944000C176D00F0
:406EC000FC7D2B00E9BF98000630E400881212001FA68D0036369600C296E100F8E4E000059E37007D3275001F787000FAE232007F474D00F04FCE0021E8B900E9C364009A
:406F00003A7C770016ED050027C03E00871566006E66F700219255002F9AF100CCB68B0089A7B000B2F36D00929A5400E9206C00235416005CC45B00CCF9B40087EA790009
:406F40009E5C9000935174004AB7C000FA693600FF3F5B0071B5060057C9B20092C2B200946CAE00152CD600FAB1C200EB99D100403540009C3B28009C5EC400B3647B00AD
:406F80007A2778006E36A700ECCE54007BFCB70098F46000F9575D0036017500A3733F00E96CE500FC18A7006BD41100098B4200730E6700576AE500CD1F9900FD0DEA0075
:406FC0008CCEB2008258EE00F24F0F009D44A800091B830088C4AD0071548C0093ED0B004015BF00F415C40067AB71009E03DC000F7372001309C1002157D300E8FB2C005C
:40700000D9C29100C54D8200A8BBE4007D739A0064281000BD6094007B873B008DA0DE00F4153500BD5885006DE40F0027312B008780E20052984F00ECDA640089BFBB0020
:40704000AD0C9D0017037000E44D4400B927C40004F8B100B752A100AFFB8900CBD7E8002C935500A805C800D363DE0018DD9200304AEA0029D405007EC2E400C7F2940008
:40708000B444B700258091004781F7006FECE400378F1900E9188300C2A7E2004B46C7005D8B9700545EC600BA5B68001DC65C00E4F9830088A8C400B1F7FA0053014800A2
:4070C000E40B7700561C1F001AEFBC0059567A008F8AEC00130F5900F835FC00E0416100B4C63200FB8415005A1FF8003312D600E33AA6000985DE00BC667C0025AB79009E
:40710000F402F90038AC3800B3BBB5005C5BA500015BC3006478D900191DB400E2C03600A224FC00F5D6DA00256D900007C940005647DA006FAE090012C7B400B0D5FC00EB
:407140003100890075BEE6007A110300A693F000540C3F00AD585E0051F39C00561FB9005C27B200C37D1D009ECDC600D810B80099A1E7004FECA0004D5A2400F38773005E
:4071800002DED300E2DF9F00A06D510020B69900ED065800C0DDE800F8037C00B8218A00ECBBCC0058909A00E310450076A879000C6E1A0063FCEB0042DB640049D8C5003C
:4071C0009D39A800883421007A394000D7256300452CC500EB58970085C54800C3A2840024D8E40001EAD7003DC569005BC263000867D20042278C00A7A3730099BD8A00F7
:4072000030F982006CBCD300D18AB20093BD3C00F665880056871D00CC118600BB75E6001F5AEC008E348700CB5DC300B6DCDA002000B1005F952800F0EDB9001C020B0008
:40724000102F9D009CCEC10000446D00271F13008A012B00CEB84600DC86E300B152DF004D773300C54F4E005BA22C00666EFB0029F550008F049F0039F76A00F8C203000C
:407280005FF85100A4FBB500411BB900BECBD200981AA80059DD2400F25941001E6F3B00A0BB3900CB0BD800D9E6BD000FE2C20099C10000180C0A002762B800BA236E00D5
:4072C000D0EE89006B299400E2AB03008906620017F9800072F40300A9E614008F0B92002B1102008C35BE00C4B458006318810067A24F00189A5B00A47D450065085B00BA
:4073000023760800675E5200AD40C000CCB8CC008AA6A10030CD5F0045F52C006321F20037D1580067AF7400B53E9B0019EBA6004ABE93001BFAE30067F49F002A748B00B7
:40734000597A320006017200DF2C8700499638000F6FBC00D4A9BC0015468E00AB401D005B678800E05E5D003EEB0400757CDA003E02270063C0BA00171A9E00F2D18B0044
:407380009C586F00E560DF00E78B25003D308400B7C3F1009A067700FDBCFF00ACC413009DA1FE00F9D89100EB9D3100651DC80077093D007481B900229D0B00FD3E8C0064
:4073C000D767F200638C8A00D11EEF002C256200CA4A4F0057AF2700B8D1C9004CCC44009D425800A57CD000B3E22500C61A93008092AD006278750028C06A008833E700BE
:40740000FE5BE00056A54E00B96F4D001057520080F96C004867930015BF530001752900C7B5DB00E7884B00386A2000A2396700AF1DCF00D65C6800D1046B000BA45F0017
:40744000C8D8D80021DE4900D762550081C2EE007BC1E9008F76F2007084DB001FDDA5005257CC00F1056100E8F8DA002E5A2600B67F0E0066F9500036107A004280D40085
:40748000EEAFD300BDB63C0019905500BCF6160080243700B2BD0900807ACE0009DD3D00F9B95B005BD302000F21070059E8A200FEED9E0071540100EA3BF8002B4D31003D
:4074C00049FC120031BF9D007EBE28005C291000D2F31A0060854E009BE90D00B968F900DEC8EC00A99D350022D27D002E67F400FBF1540094E8A20083B88D0096F2A90094
:4075000030C1A900A5368400E63C3600F642FF00CDFF7C0027BA15003579CC00FB90A3004D87D1004F3D200015EF6600203FE7005F975800DBCEA100165A0E00F916820035
:407540009B4E9400A8999C00390EFC00C7EEF300B669AD00149B76006F793600268C48004C7C45001356C700DFD5FE001F6FDF00DBB78500E4D683005A493B006B0B760043
:4075800096CE500094D9CA00E6A8DD00751A7700429C9800B118CD00F1186E009A1D690065A31700D000C200002E7D00202FFA005A867800F9730100C6B2AC00F411080031
:4075C000A1EF8D0050C70600890F9B008F561D00AD3571008A227C008595B400EB9426006C021F007FE2DE00031951005366040061E98F00118BC100A6FB11006F6F3F0033
:40760000AB168700750DE300778C3000757B8F00B4734E000DCE6000EC24B200A5B14B0015146600F458A200BF697400A4164700A8387B0076781400D98BD700DDC2330054
:407640003D40530086E314005E725B00FFCA4800E14F6100A0156000CC7F8800A70A3700F5D12000218E0F00F05D7E008B1A910010C83800FA406600FCF14F00D038000087
:4076800063F60C00F0842500EF53AF003AA3EA0038125000559FAA00CA13070082DB1000DBD9990057539C00882207004B989600E77CBF00C4CD9F00CB7D2C00BA7CA00032
:4076C0001B360600CB9EE900C705F70013365E002822AB0078929E00D53F39005FD656007AA8C000A0EDAD0061305D00FFF7C7001023AC00DCBF5B00B68CFE0031A97700D5
:407700009A656B00902A5A00A9EB5E00BE67A5006AF5E5002FF9A5009C765C006F1C6A00A804BF0037DA43009282D400647A63004E0D3000C87D48009B12E200DCD6360024
:40774000C5C71D002D9ED6005B454800F0204400678C7700D1CF110036FCA4000EC5DC00FB26A70032B5DB009903D600B38170002C310E0047F4A9001AF3F400DC7E640035
:40778000B4637D0092388800334EED00AB60690078BB6300A7E83700E59BF900571AC60081FF4C0090D78C00D23E6C006204D400A735E10069B37C0039113F00DF60E00083
:4077C000F1AFA100E044FB0086067B000B52DA00AFF7D0007A5ADD00260B2C00D5DE2C006904F900E50302009D01A100C1CFB6005CB40300F8D96500DF9AFF00528EA4006E
:40780000D91B1B009643FB00C1A5C8001B40B5002D54AD0056A8D900C12BAD0079228E00A3698C009A779000974C66001C5B7E00719A550003F638003B3B40004D8D670061
:40784000675C7900078296003782A800FF194C007FD36C00D7BA87005EF32B00C40C93009A8109008D0F5600894821009D5268002F79F300EE9A9D0084D399005B199E0012
:407880004CD59F00B97D7E00F11A980013DFA60012E8B100F71B24007A37FC00851DA800A8607100F8D0310073482D002A4D08009A49C100CF90C80039112100ED5CA40045
:4078C000F948C6000213B20037AEC6002119A800EBA6FE000C6DE2007D33EA00B9348700301242006F0897000F6C66006CB9E700C056240052AAEE005896ED0081167600AA
:407900008FFD29004D2124001BB18400A0B1F10014C6EC00A008340071DC3000CF16F4002F4A7B00786CE500F88A440020E5090033F2100073FEC000AAACF100413E7C003D
:40794000043D6800809CAD00FBA5B5007DFABD0003555E00D442B400085DE900ACFBEF00C6FC1F009E772A00AAC28000899CFC00065030008C92FF00A9265C00B37C52002C
:40798000A89AAD0014399900306C3600421E220013EB4400DF3A9400B5722E00434E05009AB0BB00841CFB003E5F01007B4079001584540063CEEE005CF93F00772B6C00A4
:4079C00076766A005643C4005E8A8B00410F4000920BEF00876C1A003285ED0015C35A005342FA001C494500D6DA2A00AC8E2700AE251A00CF963100EF92C1006201FE00C8
:407A00008C4085005BCDD80057931D00B072FA00DB154C00FF187E00B5EDE0008297340048B33800D626B50093056E000406F000E355C90006996600EF7D4600D5A99E007A
:407A40006995DD00CDB3C30048C11D001329D500054623006C9BEC0008D33F00406DF300E71A4C00D606A9003AC87300670F4C008B50D00092E7F7001F6CC80065EE6B0061
:407A80000367B700853BBD002B5963008394F40018D1C500D6F68E00B06FB400A5DFBC00C0994A00E9A4B2008E9B1B00E6BED80000CE82004D2DAD0012B9AC0044443C00C7
:407AC000018FD900FD823800B14DE700E36F950074A44900F27B1700DC30F00083AFD3007DFB590095628700CFDEA30086F1D600E8C72F001D4E7E001586CF006EFA8F00A0
:407B000093038300D64D5C00B361B80055BD960068B10900B2B6DF007A39A300927D1C00717F6D005AA1720080A8B3001B28D8001E0E4900A90C1300784EBC0018D71C00C5
:407B4000613161008A65E10086AB760037BA6300283A400052B7E400279F9C00FB32BB005076CF00CA15AE002BFE98008DD8760042D74B0000FE4600203638006CC9CD0078
:407B800039FF0600496BD800E39650008B4F14008A7B63009E4AF300059DBC00E5B84D001CEAAA003C75EB00208E8200DF12D20083DB5B005EE44E00C61F1100508E260037
:407BC000592C6C00717B0A00CBB6BD001B252E001474E700AC84100065ABCE00852AEC008171E10052FAE0007E11E2000C5EAF00BF674B00B72846004A3CF600E07F880048
:407C00007A45CF00BE82A200AD18A300534F21000CD96B0064F600005C14400063580F004A4523002A105300DA1E8A004B7F3C003F6B500068FC14008AB60C00AD23290007
:407C40007E7E4100BB1BBD002E1A13004E791E0039BA4400A8F1430048D6F500DF2D1F00B1CB5D0001B3EC001813AC006FE4EB00F6DF3D0099190F0098D9F0003B1DA900E0
:407C8000DF30D300CB3E3700ECED6F002FF3FC00F61792002739DE00DFE192002C807B00E780D300202E14007D31CF002DBEF600AF77E20053C8BB009CDFC90058EF710012
:407CC0004AF67100B8AB49003DA46800DCEE5D001821EB0013E66C007D43F300D9F1690043009E00359A7A00834C1500C2D43300AE80FF007120DE00AEDD0300BE1607006C
:407D0000E7C8780021C57B00D67EE5004425630054A847007E266C009B1A5400B1F61F0015B79400F7C66A001AA187001CD50B00A28504008459A8004EB5A80080EF4800BD
:407D4000F4E4090000D17B00B911C800E1199600EA0E410013A30B00BB3B4B00137F3A002E20D3005E29B600F5F07800A43B280056622E004BEFAF00528BC5009805B40029
:407D8000C6419600A911F000C194C10016CE6A00E90F650051D184005596E500648E09000D140D0029D0290004B9BA00533A2C00CE530D00FACE8700D28129003B78E70037
:407DC0007B63B300F67F0B00BBF68A00E50E5E00E0AC7F002C148D0092669E0031FAC40082152F0048CBF700737ED1000C492A00CB11F30044DA7E004C2857001AF83E00F2
:407E00004775F000627F4E00A47D0800BF15CF0023A815009971B4002D7BF00073176100DBED8000477E1100181E370005041E005FB0F800DDB35100E5610600FAB4C60020
:407E4000E8569A00B8AABD0043D109009C47AE00193318008B556600D7B18700C41DEF00DE00FD00D275A7009736F5004DF3B9007AF3C8003D4A7800E13A900075E93200E1
:407E8000D8001600542CD400D31F9900AA7B6900B5095700EB13F400222EB900859E26002B5EEB00F19D130009A5E30057725300D1259A005FE868000154A500815F5F00D4
:407EC00026466F007D08DA0041A1E900F152EC00149AC5008594430025FEBF005F1F3900CE9ABA00E9D3AA0096AF4500907EC3000F422C001E639C0057E977001E714300E0
:407F0000298B0F00242A60009D8BBC00B0A92E0074711500313C860016465700DBB32C002E9F9B007D023D00F05A0B00BC335100B6FC1D001BBB6A0063EC3D00E4020D00C4
:407F4000B0E612001AD0ED004C168100F78E6C00CCBE81005776D8002EE2F9001578030055B38E00AF6D7000E17F9800E9DAF6004E8157005826C3003AEDBE001C0AFD0023
:407F8000A173EC0080BD8F00A05C37002E10E40063FCBE00C25C7000F9CAEA00F958EB0062668600598E6D00CE387C00EACD1300757D55000BDE2500CBA26500BF6EEB00DF
:407FC000082E8C0071C30E006D2A2500F6DB1300295A34006A354000BB7D1500B8F28700DF17FC0033BC7E0067B32A001F56C7008D116500603DF900EA789E0053D23100FB
:40800000ADAE0C00E9558A002AA51500EC70B2007358F500EDDDA500B557A700F47275008C1B72000B69F800141EDE00AA967C00B359EF00C58CB5000A44430059AF600017
:408040006AB6E600B2DE8E003B65BB005C4DF700460CFE00E2288A00DD82340026807700DCC72C0085829800399CF5005A7CC50058E2F40053EE22004A7E8E00807CE900AE
:40808000F789BD00AFC5C500AC089D00EE8BC0000F81110015AE2F003314A70082131E0067AE900059742D00DBD870006684310027BA66000387DF00A689B8002F4C980005
:4080C000A26D04001013840023A917003E65B6008FEE2200CCF98A009544CA008A9CAC003407D7003FE0300064047A00F26047008E8AC9003D1EB900CCAFF200F857440056
:40810000A49962005BED5F003EA25100FCBC2600EDF4DB00805B6A00588454003F68830003E0DB00E5604600DC3891009EDC9C0026C53E00EB33280025515B005F0E860058
:4081400075F18400D82ACD00093A8D006BF57B00F3E59600C730E10050B45100C71EE200A2EDEA00D6EF2200E2D17D0095919100C5A508003D76A600B4C60900DFF2D10002
:4081800096324900FBFA7D00E0C3A000493F1500259146005FA8B200B0FBF500E65BC600925BBD002EEC7300CF29BB0005D4620080EF3E00906C8A00B5D5C1007B1E86003E
:4081C00062C2E90080F77000C64D430043101C0057DEC400BA44D500E3EA3000E0258E00B7579300883006003A570A00CB6EE900A0B8F8002DE64B0082633F007130B90022
:40820000DEF06E008EC6CA00E6CA64000C4E6E0031691A000980B50095735B00EB63F2005516E300CE954E0073D9C40010E64C00E800F400734DCB003A576600EB3EAC00EF
:408240003E23FE00D44E8D00142469002CD04800EBE8C700E9F1540008D59900B7C113005A27B800BC8F96000A37450018340600AC850A00B1E5BA00D74357001DC25B001A
:408280001804BA00800150005F4469007B6BA500A7016500B2BA7C002A238500E0AE2400C565240014965B0064A003002283160099872B00F4773600019DDE00855B720038
:4082C00044241800F34D630071407100F4C5A600725046009D4CF500CD4E5100B3732C00D5867500402AAF00904DA1007FD6FB00358F42004988FC000C9D8F0018F29500D5
:4083000065B75C00FBE04E0088211500E760A600BACD17000A2CC400B83D1B0035B5570048963B0082569200D09351007576EA006D152A0075E31000F91D1D00D353D000BF
:40834000CF9E1700DB19F500EC41C500248D7F003339E700D28AF700F34BB000E5D8CB006FEA5C0007064C002B4F6200904F1C0072270D00542CB400DF6D97004CB70000AD
:4083800050E34F00CDF134000C29F60095B2540083553000A5C6A3006A271C00FCB9EA00C1569D00B48CC100D127E4002E31CE00DE2ADE005D486E000EDA980089B74C005E
:4083C000D1910900CED90D00FFB8C800F4B60B00E066440046FD4A0037394B00DA48D000907B340064C1CD007B6F26007D8E4B0087D577004E7DF800310FA00005B76B0032
:408400004498DD00E7BC110063E00000754B0E00285B2900F4788E002E08B200CB489700929F400056223A00371C22008CB48F0053373A003E063200D97FF400D3A06600C0
:408440003FDD2E00BF860700ECDF9500C3669A00F7C53800C881C5002C52B800831F0F00F4094600AEE4BD0062E07400CDCD9000761D7C000DA003005DA35B00C09C27004B
:40848000D1256600776EF5002ABE7200203FC900E4E7EF002F637E00D25BA000342B03004472C5003BDFED0077084200E3F8F40006FB5C0041E4DC00C17C4F00AF92AE0020
:4084C0008540A200D049A10098516400F0B82700287D3800CDC9D00038DD3D00B0651D000107410022194500C909B9006BE84B00275AF200A1E50400DD75840014D330009C
:4085000001634D00AC6D5600E8292E0094ECB200AA582200D9BD380061233D005D682F00CDAE96004CFD9F00EE70B9009C2F9200B5B835009DFEA500A001DD0045927B00E4
:40854000F5AFB6004449860011EF7E00E30EC8002AA8EB00E5760700CD912A00719B7C0053875F00FFD7B00077F025006DFCBC002010CB00BB4AD2001332F500B4C05700E1
:40858000294E1200A16909005404E2009A263100E4EBEB009CAC6400DD8ED80003D23F00997B1300A00807009F634B00186CDB00A736DD00FA607500079C5B0002DA2A0028
:4085C00081BA7600E41F1D007F88AE0024F775007FE7DB00AD27FC004359920019D4FE00226B1E0095C23A0095338C00F2DF0100F4FE9F003271850087389C0002D7840068
:4086000028E627000A16FC0080DF3500BCB77A00FA379700917FB4009F048C0031E46E003EEAA9006437F7009E7D0800F2B747004E916200EF4C43008DFAC60028BC1A00AA
:40864000C76A0A0058CF6D009C206F001C6BA300411F8900E2E28B007BA4F900800C60002F843B00739CB800E6153300931C0400CCB7100099C8FB00BEF6D80072AA670006
:40868000B9857100BECB0100E4034F0039889100B0D78900E7F781002FDD37004F2AD500F267220052F62800E1B21F00FC5D310003A3B700BCF57E00EB768800010E9C00B2
:4086C000F1E3E60048B1A7007F46C20052648F00D81A99004854A8003AF7D5005C071500D57EEB00A8BE5C00A113BE00938CEF003D57C200BDF59600649B3E0052A718009B
:408700006A9E8C00F71B8A00442F0A00834B720076EB680033A75B005B30EE00AA005B00B6581B0047C891001537C300350F220022D5940061F95100F1368800FDC472007A
:4087400092110B0004AAF900FADE1B007423F200480D6900ED535400F89A5300C59FC3004E010C0080BA02003E91FA00E48956007A854C001EBF4000E95FFD00533E030066
:40878000B9C01700FD5EB90035FDF900FEE4BA0043CDA300E1027B00B60AE3006B3EA60081B032008882BE00DFF03A00201A24006B3ADE00EB77660028D45C00216D7F0009
:4087C0001D63A30011EDA100145F5400FBFFF5006196E000598B68009F39A20067E7DB00E4C5FE00E7C7EC0045FF49004AF38C009FC92F005C3BA600E44E960061FCFE00AD
:408800003BD2CA0059D6F6006632AD005419F30084BAE40032AFE300B2C85B00777E7A005D48CE00CA5F520013881A00596AF1006672B500F8E06600ED810C00ED42D800CA
:4088400004055900ABF8CF0030CE1A000F75FA0048131B0047BCB500A010AA0041E98200BDB4F7008F7F9A00E3B1FF00EC5C5600681E5D004F45CA00096F9500BDB1470016
:40888000F0DB4800D00EC200479A0900BD4FD8001A5152006DF7DC00706157006A382A00F2080500A375D4007EC28B00ED83B4005E0A6800A4A4A20034BA210019EDD300CA
:4088C000998D4D00522C5C00D7841B0008572200855DAA00621390002515AE00AA5DE700663FF5003D50D5007190B300DC1B1E008D769900C07FFB001F89D8009017770094
:40890000F1EE8300AE6B56008A1BE700CDAAF400A3B0B8009E8A28003D1D74005AF057007F268C00801B45008A9E2300442B7500E4B71700315BB100A932650053F9FD00ED
:408940001B9CCB007D29410039F2FF000D64B700583CDE0078D64500D07E4A00687D3B00FA96EF0005E23900C8228000F773900040DB2B00383BFA008FA661005A0FCD00FD
:4089800040970600B21EB800E386B200C684A8002E989000E8E344006986DC00E52CD200BD34DD00295647006AABDA00A7D00B00802F40001D381F0083849300CBF1B000C4
:4089C000B246DA009D62CC00F7113400106C4D0037AAA200F479F000E0929D007B261B0022F11C0080F86D0046EA76008CE16000B1E69C00DE301400907B6E0067DB88000B
:408A0000A4B49100EB9E4E0098D237001BC26C004FF60300A635F1006B7D4B008A9BE20035579E00F981D200882F6B007287D90020436D00311A5800A80C0E00FC4DB9009D
:408A40001116D10012DEC500A92E8E001C84480019DFA30098AA730086E360000B1DFF00852EFD0063E71C0046925E00019C7D003FC521004C643800DF785700CCF4F800E3
:408A800043B40200F822A9002E083700892D240031CAE2008E400900080E3700A6C9AB00B24CDB0050BC20003149870086B8B400F1050100C28D8500932D5C00011A190085
:408AC0006700C000C6CF6F00783C9A00D58C9900C5D0CA004AA3F300DBA6E8000FCDE00086AFDF00133A5A00952CEF00A15E4600C0843500BC7DF40067A602005CE5D90020
:408B00009D418600A37A23007BC46400968CAD0084C817007C58C500F8971600326C2E0001207C00E5449400F9E69F008D80F200774648004FCFFB00C71F760059094200BD
:408B4000C5DF5C0091F17C00E8640C00152BCC00D3AAE900A9E2450098103D007235A0001B9C2500C5E9EC0017B9D300AE368200D262610047A84C006148DF0076159C0033
:408B8000134291000B865800647DFB001AD70E00A5C42A00F7A36C004829C600555B2A005919D200BA44CC00E1505F007E8C950092369100B321C700CD12EE00A41281002C
:408BC0007C325C0066FE4000787910008A53B00034B361004B4877001D9A00002D43E5004645FD00568DE7006771B600402F5B003EBF4400D1553F00BBCBFB001195F7006D
:408C0000A1EC5300DFC58300F96D820081593400E8A57D008F81E900041A790076B00A00E93F500029C49F0044BFD0006F260300D5FC050086E18900DB8CA100F3E031002C
:408C4000C85A7B0037F3C300EB70FD00265AC6000238C50078E66A00BE80F700FCFAB200DF8447008536580075950E00FF09BE0083915100D9BC14008659F40001A45800AF
:408C80009C35A400217D8F005DD88500121D1C00101FA70073A83600E626D700D9A3B9008DBC6400182A13002B03FD00FD6EF7008C598B0085C37A00DF386A006092810019
:408CC000EBCDF400C13B340004BAD3002C817B0069FE6900E516670096105E00DAE34F00B445E1000177F2009D6789001788C100DDD3C30006CDBC00DF005D00615ABF00B4
:408D00009B6FE200FA21DD00CC8327005EB5C200918D0C00E15BF50081D29400ECC8CA00C50CD600EF284100E1B2780071803100C55B7C001C59E700D49254004825BF003A
:408D4000F76A240095672200F56AC100207D0200EAA869008A2B90006A569500E6B46D0001136800E0B4890057D81A00B5E10E007C9CC400801F2B004A33FC002283180093
:408D80006A44D4007BB09F0009478700C7C3FC0083D5810046477C00270892005E1FB300A7857F00E9DA58002B1C4600F0764E00C3D3B40060B63D00E50932007362FC00A2
:408DC0008886B400E3674400DCF4F20018DB4800CDC68500DAF99200C0205700F685F600E3EE680045032800E7E49F00ACF37500E8E3820016F28700B17F6800B639E00097
:408E0000A6FCAB00D2C32300948343004F1673005214D400CEFA8400DFF3D000D0F74600A55EBE00F368110022B968003EEDBF00AF027000AC5B9000B3A05100F2D57C00CD
:408E400042B19C00AD47C900E3236C0060A323005FC60F009DFCCD009E12D2007D8D240040337000E328D60079A1050074AB4F0045B586005418FA0038FA1F00FC84CE00EE
:408E80005E33E60041CA2E00E26100003D2A6A00FA7DAB00FEFCC700CA66C10010C6B70096BACF00AE067D00A878E400D5874C004C3B9E00C286D800F978F9001EE5CC0013
:408EC000EB574A00DB949000AF818400334B7F00A167EB00354DB0003EB1BC00F1F13600D43DB500CBCF1900E00E3700732A4800B02B20001115DD009AEEC700DE81E0003F
:408F0000B82E6A0054573D004779C7000C92E70013D4CD006722E9000BE3C800F0263500538AE7002AB5FA00AF99D000E7223F00EBF52A0009BE7300E9BA6B009B728900E1
:408F400080019000A0C6FF00E7A7D500A954D900AE0AF600E3C5BF00923ACF00A4049300B9376C00146709008CDDAE00671CAE00AC77FB009E3C860029FF51001099B000DF
:408F8000102088008C126900BB23C400287287009F484F009E16DB002C97B400AEE8BD00960E3800F6FADF00039DE0006464FE008E726200EB935000E424FD00F4518C00A9
:408FC0005A3F1A0035E0750060F6FD00F494B500AB0A370032DDF300CFDA1B00222B620005F36900CC1E2800970A5B00D0B640002634F9002126B3005C22740017A05600C2
:40900000BD8F4000DA38C500F6D9DB00D85DA600E3A6B700BA6FE6006450FA00F710400062BBDE00EA7E4E000D167900FC1B8500BD65660000E0210061794B000A07A400B8
:40904000B066500005399C004C5D2700E256E500D8540300E43A8F0045E0C40047EEA3000604690017D336005CD874003E09B200C0F0AF00A1DA4F00AF401F00F44FC900AF
:4090800014E58200CD157600D4888C00BDFFDB0082A207004DFC4400F09328004586490021012500331A220087B39300A0823A00F3549800B69A840032013900EA1B3800AC
:4090C00048667400B623ED00C5B42A0026A02D00A4ED3700BB338000EF5C470081D07F00088EFF0006F8EA0099F734007811200041451A00F64F010004445300CA40B7002E
:4091000002142900B7853800B8807A000284DC0061FC3E007F0D7400770BAF0015065600535DBF00A26DA600AC517B0044D89E00CBB1E2003EA6220066A2200088339400FA
:40914000CB60E10087FB17004322B20037433A00943B4500479B4600A36836003D441700F3AA5500F16FC0009C5DAA00938E5700AB2D3C009A6E0F0069DF06009DDF5500F3
:40918000C62B6700090F0D00B51FE5008F723E00897E060095D1F200EE8EE50033BFAE00B15293001495B8001D5E6400357E9F000AFC3A00138735000429290048298D0049
:4091C00054E05B0099585A002535780069244300D450F90061276900F92AAD00D1491B002B8CFF00AA997100B6DACA00A973DA00C12C5E0033FFAB008172ED00088AAE00DE
:40920000D3705C005CE10600378FD0008B199800B39BFF00CEAE0900BA8EE00000CD1C00B8F7F600C8194C0024F9D600A7F9B9000A21FD006C281500E025370063C7100032
:409240008DEE30005B154800DDD1D8006E2D4D00C264F8004B474300DA63E30085727000A18E40002E2837008D8A8C001F01520085EF3C00E20B3900B2B6DE0094D077009B
:40928000532E6500AC474B00A3B1EC007D767300641E820044A5C6004832FB00FCE0F00058667A00234FC800546AA200745F23004F9A4200670D3300ACF8BB005ABCD6000B
:4092C00024905B0015041800E52E2A00D5961D00FF69CA00FF668D00D96F4D00CD817D008A04CB0042606E00FB2BBA00C694B500BD953400F8C112006EB86E00D78244000B
:40930000CE9D6900FE423600A56F0D00F245F8002BDCD200AD49420049DDCA0091D5FA00945F8300CA316000AC8AA900CCBA2F00E592940009DA350027A5A3000E147100A8
:40934000D5170300DF8FD600D1DC0F002405260055759500E3F016001669EA00FE59840029F89A00CCC7A4001174F600445179000B365A004B692300F3785700F386C0003B
:4093800047D4B900E617B1007763C40033141700B320FC009CDE0800FA7260002DCF9E00F76DF900674B7A006AF668002C2C4D0070438B00609DC800D1CC7A0060D30F0026
:4093C0000CD8ED0040C58F0073999D008CC0720007DE3D00A69D000097C281009356400057285600A702C100456806003FA49500C88C0A000D6F6600675DF200196BFA005B
:4094000079F8C3005CAD2C000AD53F00E63DB600F89F65000B532C0086E0F3008204F5009F4F4100BB1F4C00938FA5007D0B9200A6130200BEB57B0039CEA80004DEB00052
:409440000EEBD500BEF891005D33DE00C5B95C001B490F00B142D9000D5430008340C00069133400A789AB00B12B3400AEEAC900D6F4D9006BBDAD003E97FA0011287C0044
:40948000FB8E1C006204BA00834C980080C51F00ECE5D9005EFD8400A29E9D003B2230003668740036722500BCE44E001D6C09008B8A70007BDE7000D6CAE30040369200F1
:4094C0003FEA37008EDB41003E80D10099918C00AD2F89004447A60050CE9200C8921A006B00F40022795E0073ACF500BC10DD003765B9004183C000B66E69003319390063
:4095000026ADB700107E4A00DF21CB00A83BE600E8325D00FC4184005F0050002ADDE10048A90E00633A0500C4126900D582A9002ACF8E0089348E00C4BA46007998AB0034
:409540003C96DA0027F73C000ACA5A00F5CF4700E3D13F005FF75A003A2D070073FC4B009E317D00783AE500658002007D171F00496E93008791FC0003542800E19E1E00EA
:409580003A0AAE004C40E3008C5F5100994FCC00299C6800DB76A600803C8200AF91E700A62F7200A82F82007D0D08001E8D7700342696009F9EA8002FB0240014E96A003E
:4095C000DC8B57009DFD1A008065B900DE3F0200B5A0FC0042B9E90046828300D6EE7500D978FE001FE2CB003E2855003F714F00A7566100787CC600990A8700AE4A69000B
:409600005FCD1800D9AF72009C902100E883DA00C2BC4800ECE1A900F479F2007B7593006766090090C512006BE5A300290B7A0055C0230049D77700AAA52E00DBA467002C
:40964000F7B7D200C15043006D8CDC0011DDC500FAB77E00E0DC2F0096A4220054C5DD00004FA200810AB20030DCDA0090E77D002427DB00BE214300D6889800C550540073
:40968000F8E4D80088E81A004585D8009396F20076091200E83641003B092C009067AA00A6818F00B2C6A0005E203D00732A8200BA0A6C001AADD500936E5E0073347000C4
:4096C000DA8F0F00E19ED5006A649700E6076C00AFE03D001C33F700C836D400EC35BF00E12BDE002FFDD400B81D2900467E7E00D7E1F100F5162100A11650008DC8E900D8
:40970000CEAD9E003DC12E001B0CE900BE78B600C7F7CD001AE1EF0034021C00B410610010897900D1244000637ECA0050282300F6EBB300C67D770069EB6B007D66EB0094
:40974000069111002BB7DE00203ABE00C1E11A00AE2D0800CC6530000C000D00BD026400C9CFF7002652F600AE128600C7FA8E0060214E00A68C0700CFEA6700ECB3D700FD
:40978000454EBE008CEA0100524AAC00E3BB6E006569B50097FFF400D4CB190063F2D9000E629E0048438B001821B800057862009BB6B20028ED9C00E72E550033AD510057
:4097C000FB1ACE0076723A004191CB003993F30048788D0056554700B7DBA700A4264300F38CE000DAB3FF003881D8002D00DF00E4D82400B87B6B00FA1A45003DB5120020
:409800001A2D71005218FF006ACB450080354200159730008F87F400719A3600C13FF800E40CD2006127570005F82A006C796B000C80D20045405F00A3593B00AC4A54009C
:40984000A4E80D0073D1C1000525780083B21C00A8DAAC004C4E590098851200D50DE700F58D4100FD2D1B006D877800D9653E00F3E55200EE63CC00EC8B7D00809EB40041
:40988000792DB200E93AE000E8FF7700252432006E42A30062CD9400768E200084116200EF9B510025C3D1005B3FC7006783890069CD6C00AE627200ED778E001114B400EC
:4098C000BD0EF60007CF11003DA56C005D928100CFAF3D00056F440016B1DD007CC97E006BA8B500066A6D003EABA1001A6040004682250065AA5600E46EF0001CE5850025
:40990000C63BB2006A6575003461E100335715008E55A500DBE3BB005DA03A0050EB36009A5DA0005ADD7B009230730024B2930003556200A7FBC700DC02A200EAFA0800FC
:40994000D23A8F004952EC0022E9BC00B6E8070015E836009772C00066E71A00709A0C0030DAA1007091540094099C00A5661D00AEBC5400067CCC003F1EC500C0A8B50034
:409980000B8321002070810052105C0091D64300E36FF1005D85EF002B1A5A0039DA9E002BD595003FCEAF00E49A1E00CA6C0F00581A4C0013B94F005B093000F10EB900C4
:4099C00068417F00C5526F00AB49F400D2346900F960C00020832400223643000FD1AC009A9A0F00BAB66100FFE7F60060A0CE00C1DA4A00F47C17004B7FDE00E90BE000B5
:409A0000880B690058EEDB00BFDEB700C3030E006309C8008399EF0075203C00FD4F610070B79B00DAF8590064899A00C5905200E5C409004DF5BF00AA83AC00899059000B
:409A4000E969AD00406D3900D44B9100CCE8DC00089B7700A086F600E7208B004CD89A007ECB460070D882008B4A410041905D0074CB850038FC69000A706400B1F0FC00C2
:409A8000EAD70400D0B6C3006EA010007AA847006A2A9400654B870029DA510021F77D00A9568C00563E0600049A3A004EA98B00E2E60A00EAFFB200EC717B00A0A2B4000F
:409AC000F8B1E90055D9B700260AF500E6B4AB0092EC90004A966B003669AF00DC8FC70069869800231DFE000E075B001719B80037966C00AEC4FF000BF43F00373DCB0068
:409B0000F22853007FD7C10004524E008C4F1700501B7800E68FA60078A0DB00DC1C0D00A6D2A3000D7CCA00F9396600A3A87300EFA7FE008D50DE00A2BD890020F5C00045
:409B40000BD7BB00B8304E00AAA22B00B0C18F00E5E16B00169B4A00BAB06E00C58894000BA3810024A8B1001B9E72002790DB00A97C3A00BC5862008FC5D100A5E4C60004
:409B8000B7F45800D5DA6900D3302400C6BCCE00F96AC90020BC0500910F24002A026900D30F4F00658DC500B9D23500893E100089188C00E49D4B00512A8B001E67A0000A
:409BC00082E1B000D952C3005DFB65006502870011056900AD286E0060A06600AA4F4800AAB4C200048F3F006D6F290046538B006E0D3C002CCC7F00FDC6C500D005D700D3
:409C00004C4DC200312AA30053177A0016507000421BC5002CC8CC0055DA4500CF97FA00814A360047613A001CD5CB00E0A83D007642D50076787600CA62ED00D3E38500B2
:409C400005A45A0075121B00637F530033A7BB00972384005960C00034A29C00A2D67C00E6D28E005C4C90005C743F0035D89E003F911B008C3FFD008EFC8B003477540059
:409C80003C58FB006E52C3002B1C4700A5ADDA00543E3D00CC71BF001E8B57005E4C72004D289600F0E9A600ED3A6900DD963F001EA4FC009DE59600D181300059BF340081
:409CC00059D29100743BCF0062D689007C53920051BA1100E7800F00906663005CC08300E0B535009A62A60001C5C30092AF1B00108DD0002AB83D00D2289800ABEBC900B0
:409D0000B6DD3C007827C90000B8F60066D61400D51AF80032E25A006B8E1B003A81C900F2297B001F77FB00E17A8F00B3FA6000CC5C760054B072004737C4007F12EA0012
:409D4000A79A3100CCBCC500BCA683001BB48200049C8C003DFCC90066AAB1005DAA1800DA75FD003702EF0070505D004A9E7E00148DC6005942D4004C503E00444612009D
:409D80002CF90F009F096100E9459000F4707000D00EE4006DC850000DF8AF00168A6100325D3E008C4EB800FF554800FA4CEA008A1A0900ED68F400D3F6D3007F4907004C
:409DC000F278030054B248008F624B00FA591000EFE9D200515AE50020CFA80056341300CACA5100DB0E8400D4D34200B46F4B00FD9BA50088E0E100A8AFC3003EE3ED0044
:409E0000842739001B70BB009BF2E8004EC5720001A34D000B22B70072B7CD0013314E006D9F8E00CFA7DD003DCC73007974910038BF1800B4222E006EA90B004CFDF0004C
:409E4000652EA9000574AD0060FB53008710430089BFF600E20BD300785160000CF9430030088E0099297800A6FD31000E6BF80064BAA30088765B00EC5D5E0089A2B9009F
:409E800008ECEF00128B1C004E064100D415850082169700B7C914005F252C000251F00077893D00DD8E18006EC4BB003DA21A0070A76D0013C7C9006334DE00E8A1C000C2
:409EC000416EB700BCA1F7005F0C6F00AD58220035E7EF00376976002DD82E00DB5C8600FA5ECE00CC66CE008B2CFA00CEDFEB000F486E00178539003DE2FA001A14ED0059
:409F000022A29C00A5EB8200904BFB00515595009FF0E700019DC2001215CD005225D10049780600281704009974D0005BD2BC00845D2E006D95CC00E2C18D00866F20009A
:409F400019C86800204FBC008B52E500AB1176003FAC47006977690057B0DA009D094E00EC6C8600DB54700015F7D400B5D0190092DD1000C764310055039700E3813900C7
:409F800023A08D00F8E722003B897B001AC30000F16E6A0060DC81001A446D00E358BC002FF40500B157E90078A73800124ECD00AFAA7A00CDCBCC007BB18800D11CBC00BB
:409FC0001A768F009C5A2900A61994009AF5F80011C90F0004091D00FFB673001A29350046878800EE48FE00014E6E009C0E4A009AD00C000A7E2B00BBB139000C59BA006F
:40A00000E1743300A6A8F300C220AB001C809200B2EE410055DFD4007ED7AE00BC8481000E12D600BBE761004D0FD70005AA910095504300C6E482009094D00064EF1D00CB
:40A04000AE78F900404B0C0096C0370010580F00AC697B0005CB3500D70526008DEE6700E33F3800D3A355008758F200BBC50C009DA13F00C35EAA00F53A3C00CF4EBE009D
:40A080001488A0009FB2CD00C099DD0039A30D00F370EC00A15F1A0002D15A00AD9612007D85220050A98C007B666100B1DB2C00C0B16F0033A6E80068517D000260DA0086
:40A0C000FCF32F00A2D9F800E4ED87000CBF1800B5721500534B5200CB4B100021834200CFCC37008B005800C5B448007662D000ABA9ED00C142710005599100BC12330099
:40A10000259B3D00A3FE8F00BD5E8000943B48008B8894008C705D007E82B700A73A0F0042D42B00D6F7A1004E062300287E25009223BE00F30C2A00DD719200EA1B960091
:40A1400052A27B00BC06FE00E4BD7A009CF6E300A9542E005D403C003F931100259C6B00C0D37500B2B10900A6D895005AEFC8004A1AFD00005FCF00C300590084BFAB00DC
:40A180003054F50046CA7D004EFB9B00FBEE8A0026D3DB00511097009C8359000429CB00FBCB2E00EB55D20009FBC7005B281900729D3D0038A9C600E9EE2400D555690018
:40A1C00099F38B0082D4A600F7784800BB24CC00DCE9A6005B2F35008EF9A20070A18D009E6BCD0030321600C9D8AA00708BBB00F0F35C00FD6E0A007615EA00F530370025
:40A200000B45B500240B6A00505D6D001C0D380085333200E86D1E0039243800F9986D0010746E008F2B86006753340070A2E300E9EB8B0000A1690020E8C00051BDC700FA
:40A24000B61B8E00BC68D100EA66D000D7410800A951FE00CBCE01009C661F00182C8500642FFB00F02CC500275864003D7AF9004735CC0018445A0007C1AE00F6A7720049
:40A28000C13F260020B89A00058F5500B0BF9100CDCAAE00AA601300ABE645007115720063330700FE83600053FBB8003A9A7B00D180FB00F712A700A63C2200FF66F300C2
:40A2C0007D8F1500E12C23005DB23D00188EB100A5CE07000EDD4B00B347590064C9BB00F9F89800B1F61E0036BE8F00A4F4EC00A537C300550DA700E4C5EB00A2444C00BC
:40A30000C860ED00D81CA700C3F1AD0009E47E0041EF15005A9AB600C9AF8100DD15EF0013B59400FF4D8F004F0BAD002713B200827C0400B9273C0073F71B00ACC3A500F7
:40A3400077D9B100016590005E917400E77D930036DFE800B19465005950FC00854D3E0022E5CA00C1074600FB976C003B5A8E00096D9B001AF5BF00BD255D004F6CC8008F
:40A380006DD53900E2C07400ECCEC7005076060075136000275695002CD892004BE610004254C900493006009C294B00CE69B20073A6520000B1780012D20C00D594FE002C
:40A3C0004D472A00CC392D006D0CC600FCC52200F4F51E00A6B2A30024557D009785E8001724A50024F2B7000F5E99007EC21C00DCA6950058D496009B8A320091A72400B4
:40A4000064A0B3000FDCCE00AEECD100422C2E00230E62006DCC2300695C08004A33E1000320E300EB048E0000098200F714FD00A0D2FF00A31DB1006ED428008F124C003C
:40A44000D666A9000879F100E24678008DEC0200A6D2A600AF6F1A0072A6B300EDB8DE008508DE003C826800BC5A620060F30100B2B0B700583F53008435D40018B3AD0061
:40A48000EC931C00AE380500A6706B008EB8370021B01000274B37002EFAAC008C065C00AB966F00BD7FC300E5C11100162EBB006B77F300E5165D00436E8B00F6053900CA
:40A4C0001BD016005E7994009E4913008DC1CA003CC93B0048E70C0009C84F00B89917002C5291001AF667005FD7FE003BEF4200131A6C00BA97D200A3906400ABBD690091
:40A50000421FC400E181A900AF4A630072DBDF0002501C00607B79002C0C2D0032898700F49AB100F35D1B008E9388002251270012E4460072AFC50053E02200F97A8F0094
:40A54000E8D63D00FA71DA00D75E9F005671190035B76900578A2B00EF776E00171EA600A59BDA008D925200ACF28F00D6851200621E2B00E539EA00745906004A92B80098
:40A58000C01DD6007C82B400F4558200B8E6AB0031A12100221C05007D92A2002218D800AA243200A46E8E00080BB100B7E93500099751003D5D1F00B459FE007155C100B4
:40A5C0003579E700FD6DA10060E8940061CD680012D50B00485B890014B42600043CD0004021D200AC588E00B9650900C641E6005FBDE00028A92100E7127D004D142E0061
:40A6000016DD77006C9FB800298ED000E0F5B000B3E139004940E4006DB5920085647F0054F54400632C4500427D0500445E0F0094F7AD004A34CB00FAC24D00C0134F0009
:40A6400063384E006A1A5800D98FC500AAF7D000503A82003F1F65006C2FE700BC9C3100312DDC0064EF9F0044B0F80013435400ED9899007D0970009693850084ACE50004
:40A680008C16190094D43300123DC80094F510007042D100EF020D001F5A840079DC9600AE453700B2BE70004C8540001DD2310031135400F11D7D00D849F400B2A7FA0065
:40A6C0008A9264000CD03100249ADB009F2B6F00EF305E005DADFF0065EA0C007735970079346900AC5B89003A961B00F73875001C5B2700882D5900494DE6004F043700F0
:40A70000601E990072C35F00C6CB9000C78DC300CFF3200076B3DE003F914400317FE800E8C3A0007A60F600EDDCEB0052B65900C0466B00D7EC6400B9393B00BB80D3009E
:40A74000BEF47800E711F600605D0600EF9DFE00CE84640078A9B400510B5500BBFD9900FFAFC70036D78A00CF3CA200F53DCD00FE531C002F6EBB000C86C900478E20001A
:40A7800039157C00B3BC7500B7131000E0DF230062C33F0044EBF0003A8D8000EE7DFF00EDF545003A56DB00A8EC670054AD4400FC44F9004F20F2002AF10A00475BA40024
:40A7C000E35BC2007382510087849200D400E0006A66220062E8A7000C851E00BF85E600DC4A4400A9190F00BC624D00B9567C00E26B3C007E5EBF001F5010003EF5C1003E
:40A800007D219F006DC67500A2533100E8B2010053D463000AB82D00092ED400E98D1A0076815500D393EC008AA2A1000E392900CD2E3E00BD27D30045ADE70095218C0078
:40A84000785B93009F1E2C0026D4E5007DF668004961040084A7F2005E1888004CCE7500B212C500A2074E00AC00F700FB5E6600B5BD4200A321F0008A0C1A001DABB10004
:40A880001982810073F2B9005DE71E00F25B97003451DF0040D6EC005066DE00272E2D0085BB07000D866000EF68430021DF9600625DBE002DF3FB00F876D700D4BE36008D
:40A8C0007FF05D00E549970053C83100D44720007B880A00CC8F2B002B2DA200CBA644002EC43100F2063500F9B4C9001952B700E7BBE400DE5B99007DE0280043CF7600B1
:40A90000AAB4FA005D50BA00322A71000753D0006E374F0012263E008B41D100AF4E7500E7FFBC00DE8B9B0070AA1A004B40790050D41000ED835400E0DAE1003657CF001B
:40A94000F010B600C78C9200ED804F0078BDC3006FCB710067200200C71CDB00724E11000E44A600627D6700108BA6007AC6280089C5FD008E7CCF0006DFA900E0FFC0008D
:40A98000BDBF7100CFD2870051F0160082E61A00D37B8B00AC4ABA00451E73005F61E200037E3900782A8500FDFA6F00BBBDD6009F38BF002DE12B00D9BDC3009EC7E600A0
:40A9C000695DD100DC58C1009FA1B100A202E400AB9C0B00E9F0BD00DD2DBE0087C21500E6FD5900E139FB0098296B00B02EAC00685AB700BF6D3200E1DCC000100489004C
:40AA0000697146006E08880080B63A00B87CFC0000671C009DA37B005F026800654C2F00D44CEA0049BF66002EDD1B00FDE64A004EB3BD006061600047430D004FF7840066
:40AA400028C5F400BDF9EE005E792B00D7661B0036C73000B4ADDE00C9C96A00E602CB00D78408007A7714002D2A380061BB2F003C031E006D47AC00BEC600000444FC0015
:40AA8000971DD300D3DA0800A922640079672E00C46DD500FF99D900A4B41500F11E3C00AC042C0017F07900B5EB7100316F8800EC05A300CD6BC700C359620099A9C50041
:40AAC000EF05520096651C00E5894C008246DA0021E68E0029EDA8007CF1C4007D58940085CB37005160880093069D00CFD1E9003AF3A100FE881A00919DE400606EBC0027
:40AB000099B31200E6B51D007A85C2000A8C4900674C14004C190400785D6A00D715EC0005CC940058E83C009F8E3700A6A4C900552588008BBF2E00E49561000579A60048
:40AB4000A1FFE90067E25700475DAF0012D01400A0EBC50076289B0063E5AE00ED3D50007DB86C007C0C10009CF79300DAF67300481D0C00087A520004EC6C00B03FAB008D
:40AB8000FF7FDC00EC2C37001A6030001A2F6200A648C400152D79006C0C54005C911200A619C500EACD5D00B79E9400D05B18009C68F200271AC30075C63B000E509D0030
:40ABC0005B8E7800D34FE600B04AB700E8978900FB6C64007BF16C0034907400B71955000EB0E400F2B2290003B1C3002699150067F1DA00D250D700E36D7100C188DC0068
:40AC0000DCF0FD00F7B1D300CA99390001005600153C670040B053006DA8FB0008CCCD0077CEB7007DB8B000B29E0000928E3900B59C1D0078E1A1005CCF42007AC85E0032
:40AC40006002340070557D00095E54005B4D0300CA6A69002C61770034AFCD00A925CE00929D7000F589950049CCF200D8C2F20082DE3D00D62FF700ED790500BAF952005B
:40AC8000EA3EEA008682F90001ADC200289ADB00621C7900BC0CA800D84E4100E4653A0096A63300DD444800B4A7A30014F1D5005A01BA00691C1D003069DC001B73D000E9
:40ACC000AA9F410084B58E00BB1B6300B6270100BC8D37007768100013275A009D4DD5007BE7C300C87D25007AF24500D9A919005C20A5009A5F220012569D00168DB100BA
:40AD000093B17600E3963000786EC500EA954300FD807D00963ADE00F433A400F2D6DE00AB746E00101B830052CCA300E6E07F00326AE100B2C6790024150F00347E4A0037
:40AD40002957B1007A80880012C2D3004C9A5300F236F000B121760052A39F0031C9A0000E0024001683F40028BC6A00E231D0008FF23700B4CF3300602ACA00FBD0220013
:40AD8000A11A810018D51500007D2400BD2223007428C50049DDBF001426D8002A560D00F30B99005ABF0900E80F7400D0ACA400825B040075F27C00D69AB2001FEC160082
:40ADC000726F6A00BDD7F30079BF9000C9F74A006865AE00474C6D00DAB879002391F300FDF7E7001E86E4001553040057DF7500C67BF80036A1FA00AB073E001051E800C5
:40AE00000965FE00F22EFA0050E784009C96E800BFC44C0054D99500698E7B00E17E360013176300C14FCA005BA16400B4A413008446A500F160A400DB66D7000D8A870053
:40AE4000F3D28200B391DA00BDDB7200E11B9B00503CCF00A9AF24009A29F0001CBFA4009691E600351048008BFC0300EF15AF00EB7D7000BB65710057D7B10048A4D500E3
:40AE80005A03510092D581003757320030262500FE83EE008C29A000C2A8A500123B000046BB310043552800EA8884007EA01C0067B6BD00CA086C00495B66003766990027
:40AEC00046CA0A009CCE1700D4CFE500F6094000F6876400808EE50042FD0300EE2698004C68E400B5687F0049EEB300F7F5C500633DD7009669AB007EB0A600CCAB3A00B9
:40AF0000026B7F007167870036B415002B1EB9003FFC360028533A004A28E9008602E9006888C600328D8400ECE663008F8C5F00425A0A00C07B1300A5FC4E0011682A00A5
:40AF4000D4921E00E60EF300574901004EFDAF00BD889E0010F91100BE9D0100FC163E009554370017A66000A7769300BF0CAA0065932C00A9D98400485B13008367F30003
:40AF8000026AD800327CF6009E0C7400DC6F6F009747CD0040C75E001F835200E030D500DD4F95001076BD0039A5D400F96E3E0057002F0024D27500B3525300ADACE40007
:40AFC000E8D2EF00C6FD7200B973D7008EF17E009FC31B005E102700549A4900353A2600AD90E700062CF00034A6CF00399FD9004E867C008C836500D6DDF900B38C6C00DA
:40B000006547E10046DFD000795691003B5B2600DE9AC8002C87A3008FF6A00029E52C007214E50057453E003F15DA00A472680015077D00EF26DA00F67D6F008E18A700D5
:40B040002AF44B00B0877000EA5CF500CF188C002208C0009CBAE0006FB21900EC8E5F0011852B00D2B2850049095300D9CCB0001DF0B10015A8DE005AE3DB00D547450049
:40B08000F34DE100AF0553002184E800667863005A718B00CCBB7B0032FD220044F00900DA3683000E79CE00CEFE200043BA7700F07ACD0025BC41007ECADE00AE65FB00DF
:40B0C0006E4E3200AC914B00D68093002D146F0041FD1700BF837700D516890077FA2300D997B30071F66900F54A7000C24EAC00257DA7005229D3006FFA7B0060D09E0084
:40B1000058CD7100F6474100119064009E79CC0075DDDC000C445300CBE6570066F9AC006308AD005D0C2500A12CEC00CB3E3400E2221200CD60800054D3FB00FCEDFB00CA
:40B14000E6015B00A42A0700BCA8C5008C320C0096913D003F9CF200217BDD002ED36F006BE5980000E6F70073AC2D004797CE00D9A23300279DA60068AF8C00EAB9D700B9
:40B18000246EE2006A41470011F01300487BEF00765ABA0077B46C00F6F2D9006FA0CD00BAF1690099576B00649D8B00DB731F0042A77600B0A0B200FAE4C000F0A0480066
:40B1C00083333000580B2900C0DE7C00A2E16900F1B2E700FD8CCE00A3C5F70045568800EE00AF00B90BFD0090F01F003F271000B9F6BD00793FA100FB4F6B0010CEE900C0
:40B20000BD9A2A00E748B40093AF3500E22A3500BA5BDD00884E210043E519004D524300BB4E5A00C1BBD50083D7DB00E7642F000E2B800007A9C4002E5C02006437990096
:40B24000FCD6850095C00500AFAE6900D2F62100C05DCE00D08A4400EF51340073A3C500FD6BB0005CBA5E00313BEE000631F900F03DA500A06FFD0063E22B008DD5EC00E4
:40B280005988AC00CE534200544CDA00FEDB5D00EAD2F30045C11100D3244900A87530000D7B8A0045A4E90077409D004D4FC000CF6C0D002CA5C300C5366400762A7D00AF
:40B2C000036B9800B33D13007C16F400390DE900983858001DDF130086A1200006720200712F7500803803008F10C7000E809E0065F89100560354000BC134001A0CC700AE
:40B30000AC5C9D008C8ACF00F46B1E0013C4E80068C70F009B0BD100623ED5002A05CE0054F6C2004F4DA1006F5195004FAC2800D1DFAD004FF92F006BFB780014AD2000CC
:40B3400017994E002AC98B00BE564600B25B0800713FD100786CCD00796532008C4C86002C92C50086E7B600856C9C00A0AF050081A9520045E6D300C6852E00096BFB0059
:40B38000337AFA00314985002DB2DB003B6C3800EDD8F6001500B1005E037100E6657900B87E5700FB9DCE0002B45200AF45DA00F9485900E40C59007F38020027030100A7
:40B3C0006EEED20059D3B700B08E5700D1D2C300618E220059178F0085B6F200833C36008CC07F004AFD8500DC99F000C460AF009D33E60094747C0028C6630045D3FF009E
:40B4000047CCCF008EF255008197DA00EC049C0099801F00E72665007B0C25005385BE0035EF4400E1E285004777D5007F47780048BF37000FEB5700AF3C890088570F0079
:40B44000C74EC3007DAC59007D804E00C8FD3200A71C5D00E0D38300C7859900D087DF0056682000BF3F6D0030FBF500A04EAF00C1776100F7CEC000CE622F00E844090007
:40B48000BCE5D8004BDCC000103C3100AE38FE00BF2A84001B4069002DF332009435EE0072A66B0056FA060091C929000ED4FB0098B4AB007DE67900C7341400A1AF5B00CB
:40B4C0009EEA880012039B00FE146F005F681E00B5B57A0018C415001C9E3E001D5A1400CD923000053FC000EE82DB0010D55E00A4E89100853A0500733F3800E792320037
:40B50000A19947008C9523000391B9002428310071A37F0076B01000D7A1C000167C460008A2E200B3478D00BA3AAA001F90290090754400724E2A008BB56F009448F2006A
:40B5400032E0C40097EC2C000FE33A0000CCCA00828470003700FA001AC4F6001DA92A002CBA1A002369B8004A339100903CCE0064EC5A002494220049D35900ED1C6000CB
:40B58000472EF000FC3C790067E2A4005838DE006DD66200E59A4F00FCAB3900850FB00016CEF700FA526C0023C4430047AAD40061E9290089F8FA0019BA5300FCCDAD0077
:40B5C00003BE0000B82B7E00286E0D00F62F79005B9DDA002B975100DEC2E00007AC3400D141E200A41149008FBE5E005A5190008E94ED00FC71CB00D62191001D7A00005E
:40B6000077D17C00CF3A1E002EEA2100DE564000DA822100069F5600C0148F0089BF0400A5EADE00F341BE0069A3DB00328E5A00CD0B34000B79DE00A2C67C006FB43A003C
:40B640002216F3001BFDB100E5115B0066440D0089BE0F005101ED00CC2BA700A59B83004A52E0000390E6002A50C10076EA370046F1AE006ABEDD009C6C97001E31F00049
:40B6800027784900779FCE00C312670047D5A000FC580900560290002EDD4E00E55E0200E87D5B000383F8008C46850097FA3300D9DBBA00CF0F5000EE633300D9E9C000E8
:40B6C000998C850082789D00C4D9AA00EB802300426C56001961CC00049D34005ACB9C00A13EA2002E604D00CE4520002A6F72005BF41500BC7129005D767100A7B19700CD
:40B70000091D5D0065ED0000D05E67004587F2001889E2009355AA00252E8B00A7716D001A897200CD70EB005B2FF60067BA8B0086FE5D007A00E600A020C800D3D8690023
:40B74000994999005DECDA002052260060C4B2005F319200A5E3AF001721D3009520FB002DD12D00022B5000B2552800B180EA00DE8F5E006E0669006A77F300AFB23D009D
:40B780006B6F9C00DE288C00FE8AFD0023BE0B001DC8AC006E654100F52FCB005B6A340018D10900CDAD2C00EAB78E0057FE7C00A7735F00C7C48A00C59D7400FE39E3006D
:40B7C0004EC05E00DA02E700882B9700ACD0030043D2FA00DD08E8002DB7210015097500D927A900E63E8600F60AB0000CE67600DD985A00FF735500E55FA300F131C4000F
:40B80000163FCA00B1D1B300E8B4590030C5FE006F92860051971800638C9300324F2600B98CB400014C96003E9FFB0067C9B20046068C00CBF32400F66C1B004FEF9A0077
:40B840008AD32000A9D1C600183CF600BF3632004827BF0063CC4900AD2B56006A8B98005C039400BFE72E004E6C0500117A4200A715F300169C43004AC837007CF7E400A2
:40B8800082AF7E00AC240E002B74EC00FBC3970016B34C00BEB3880005DE98005C7539007D232B00046E4A00578F2600212FDB00C9F53B007D7D6700F7964C00F2D5E900E7
:40B8C000929CDB009FFD51001E380C0069610B00CD616E00DDA39D00A62B690029AEEE00263E5A005AB6BD0084005200EC6405007060AE0069A65800041682006F50C900A4
:40B9000089BEEB00BE415F00E9F26E00A247E70078A3FD00C8C25A001F36240076EF6200F3BB5E0023DCA100A9C68D004CC24400CC058E0079773600B1F85500EE8D190011
:40B940004BD4F5008FB7A6006D0F7E00D5CB1300BF8C3D006A6D0900F012C8001EFE4A001759F2002660F000ED5CC900475527003033150072108F006377B000CC6FAF00D8
:40B980005015B300B0584800EDE0E30085ED1F008BCEA900108157006D369200719B2F00BA6EE600DDCFA900C97F6500A892FA005A3E9C003F43D600360B55007E3155001A
:40B9C0002CFB0E0002611B005B756A0022A899007D5C1300F9A00400D607B50047A6B4001D48B70004222100E6CA460030714600E41D0A00813DD00012306C002F302B002A
:40BA000008EDCD00483CFE00E3B26400EBE9FF00729C2A00C356A600349BD4003B8C07008DB54700B075A9004FF52E00464C4100080C6E00B5D1B800EC9FB80098D1510035
:40BA40001D5EF700C9E29000B06C6400E5784F006FB8AB0006073700F7911200EAA6FF00349DA3000BC432003E317600254D1400D4D59300370D2B006B5C6500853B0A002D
:40BA8000806F4C00C61B6C00E7623300E7E111003AE74C00F5DA1600645B3B00BBFCC70058748B000606FF00A7E8E2008E491300E4134900E227720058046900FC65A2009F
:40BAC000AE83C20004068700512CD2007C263000BCF4B0003A79F10074F3190098225800512C7900B7EEBC00798439009132E700D25F9800EE3BEB00478863001368390011
:40BB00003B85F800AE3E44006311F1006B3CBA0009425D00C3D71100730A7B00552F3100CCEC2000AFA593001996240098D3DE0043C7440073FB2900EF3C6C0020CA6100B5
:40BB4000747AF10063EC3D005E8358007B72930025DD5100F05A1900DAF7C000581FF9000A8CF000D719FE00DA451100342C2C0003A9270067283B00D1B1BA0055771600FF
:40BB80003E15DF00801D5F007DB5E3005B09F000C0E9F400807ED80012F8E10086B04100D273CC0080C7D700DF347E005F1FD000142BA400E95BD7009ECE78008AEC220091
:40BBC0007507A70017BFB00014B5BB0020E307003C9E6C009ECE1600C315320078D3D700E38FA100C6E04700DAA35D006C3892001A773B001B401400DC10A8004FE76C0099
:40BC0000A34E4B0035BFDA00AC2BA0009767A100FB6B2C00343E9B00FCF24300AE3F6C002AFF3A006E86FD00AEAEEB005AB407002B593A003A638A00FCBE9E0029886400B9
:40BC4000AF489500F4329300736A98004EEBE500B939F200DA953300B47B7E001B2BA40009FCAC006CE57B003C239A00378A87000B385B00F5D80300DF2701009D6F7E0012
:40BC80004120ED005BD76100266EE4009F0EFB00ADB2650087BCE600F2AE08006366DC0011FDEC003C93AA0059900600E6959B00C5061F00805F700042AD9D0046889B00A3
:40BCC000DF07A90014482800F092A600BFF3FA007EA4D900643819001FF10600B9D370009634DC00F0564E0022389400BB607A001C092200D3C88700F2D1E10043FFF90096
:40BD00000FB78A0076DAB800E53EFD009F78F0008BC03E00986DC30066F53C008F3794005C94B800FE926600574292005EBDFE0021D9130053B016007CCA320056535800C1
:40BD400011743900E1891A00236EBA00D31FEB009A2EBC00179766009215C8003748B40038823C0080CE3400CB1A6000515E8000E6285B00FBC00A008464E300EA0F2B0016
:40BD8000CF38C1004C8DED00439BD80019FC17006F2A5200E55F7F0004306B00FBEDAF00F2101F0087D1970049DFB000EB4C79000CDFAA00DAD5ED00804EF20023ECB800DF
:40BDC000A4A0FD001A19C600C81B6400F0241C00410DAF00B585ED0081095700C14D9200FAED50005C143600337B8E00598C430023985300CCFC8F001F67E20057FF0C007D
:40BE0000413EC9008FFA06001E003C00A7188000651C3E004BFF890016312D00113A4300A5353F0018515D00141D2A00EA004C00C077640028370200683FF700FC9C7100EB
:40BE400017795A00B07E9B0053F3CE00A02BF000B4558C00D2B485003676B800473A07007C31F1001FE39D001885D7001F74260052326C0035575D00B6375B00D8606C0085
:40BE8000F35BEE008024F900A2A416005A30AA00A1E43500E918E4001D729900B838190008B5A700943FFA00C707BD000653E700E2745E00152669003435F200CD42370054
:40BEC0006CDB0500A4B380007BB4EF0066A1B200C3710700BC789100FB80DB0056E6730014912600BACDF2008EC9A600060C640063FCE200461E71006FA8F90025BBC100C5
:40BF0000142D0300A4D9A0000FDBB2005146AC008E370D00C45B3E005E5D0C00A9B5FE00467A41005BE21F005B61FD00E704C30062F23600C477E800C92310006DA15200A2
:40BF40002D4E2D00FAF5AD007A5A5000FE46B800B151DB00FA1A39005C333A00D5A08A006444F30019D58200A7AB8F0022E3A1006D2C250070FB76002D51D400FA31B0000D
:40BF8000AA462B001C0BF600842E0E00FBF490001FA73600755FC9000EEC3700E088CB007E293800B30CD10007105C001C111C003281F400736B0700D51FE000F33D0D0045
:40BFC0000141F40038E5D700AB74EE008CA4690007F22B000877300069900E00B46A63002B6417001B47E300684806002678A50059AC5E00B20EE9008B53B50031C8940006
:40C0000073EAC100E7DC8D00683737008DB673006990E400D6567F00A244FF00D246EF00BB14FA0012C05A00D054B10091030D002A3D6500CDC576003628DA000EDE2D0002
:40C04000D01DEE007D3A3C0070DFC900FA3AB40044A0DA0028448300D0B52D0080264B00E6C4EE008E222D0067795800F2E8B3006CEAC000599F5C00E4CC2D00F3E76100E6
:40C08000B450CD006B798D00B4E91C00FD9C16008C754F0009AB2900FCB90E0095B1EE0025BC040095DF71001AD87F008690F6001C4F61007F55A0006B5F3B00967BEB002A
:40C0C00073A88700D4018C008822B40088FF1000091F950010A38C00FEEA830053D21B00B7DE5500FF7B7B00C2D3C500BC6F8200A756AF00FE8AC70053812F006E491F00E7
:40C10000D4F4F100B1183500E08B97001FF67200B5939B0011309D00BB35FC0031C14000CCF16C00E087930035462B00CBE403002272650015B6B5003A7C5800E58C9000DD
:40C14000E5CD9F007DE91B00DCE94200D4E3C6004B546400B231CC00577F24005CE83400FABFB400FC1AAE0017BA50004A60F5000081C700E8964800BD95810028F2D90080
:40C18000E1BC7500A560020035C14B00B50D6B00DBE8A500873A2F0050EA7F00415A0500A966B60059298C007ABACB00FC98C8004EA9ED006FDD9C006BBA9400B014F100DF
:40C1C00046860F0003AC6400B2B1C400C8523A00684EA200CDEFB7008E10D200B97234007C855B00C36BF100A635120049AB640066CA0500BF7BB000F45D870063073200E9
:40C200004E1BD6007D628800C42E7000D983CC00573A8D00549A6700A8179E00AB356D0026558A009F7BFD009FAC0D008EA36B001BDBCD00E65CD8007FD36F002DEA2300C9
:40C24000CB2101008B7F2700560FEE00528A9B008FCAF80088DE6A00484EFA0026D715001296E5003043F300187CFD00FF0E7600E7DB93006C72B50049B0B700E8D839007B
:40C28000405AAF00D43FE900FAD2B9001DD76E007E73DE001DF17E00E1BDC800192CAE00FF18E5007690D400571ACA00A2A4960018B5D70009C97B00DF72F700F0910800EF
:40C2C00032A0530022551A0082AED600C9596400E05332009C532900D6A49600573769000F666700C6BE090006627500AF1A8B00ADD32D0062D96D003C03EB00E303B500C4
:40C300000BE4FA00E31CB400B9635900576D3A0012032E00202ED200733AFD00CAC1E500922AD400CB308000102B5E0067723100C586D8007C181100F8C18100B3770E0089
:40C34000222CCF00ED662F00F6256E0099E6910041F37A00644ABF003BEC9F0021860400ADA1EC005A13BF0048638F0040AF1500B9ED1D005A2D8D00A9ABD300A21EC000D7
:40C3800066F591007F9FF200192D0E00DCD6CC002A08DB000DB269004C462B00ABDE7F0021118A0070E4150022497600700286007525A900E34CC900F2D4AD0086314D0005
:40C3C000763A9C00E7E80700CBFF0B0012F8B9001C098200C3966D0041E6F70016B1F500DA021A00BB8D0B00B4640A005C1DE900894BE40017B8C7000DADC7004CB015008F
:40C400008E55A300810EAD007AC00800BB8417009AB1FC009B696A002B29910096363500F211830046A17000ADDF6800D3242E00A55FB300C854C30038FD22002303E60018
:40C440008D3FE400927B5100AB9FFD003F94D2000ED9F30063D518001F6ABD00885D760019404200AD85A00036282A00C422D5008EE7240070B10C00E00DFD00F7EB250090
:40C48000699E3B0095CE5600B63995004F0AFB001D17F000E09AA00027C1920013914500BE1A4100058CBB001A15C100F5419C001F962100C7B07500B4A8C70058C7DE00FF
:40C4C0005043FF008B414A00297B9E007E68B3001E67AD005588D9009DE5C700D51CC3001C68FE0030C5BE00BCFA1E00D4642000F1AD2B00D4186300567CFD0033F2360031
:40C500003264850051C119006CC21D009EEC700028F859007565F700B9E7E400F6FB7600F54DEC0045648A0030F33F008F719500FBD8DD00E6236E001DB10F00DBBB7F00CA
:40C54000E7C25F00F1AE99006F4157005C11EF0072155F0036110300DC0485008C9959005B9895002316E400FF60DC00DF3663008BF788004A4E0E0026D9A2004B2E7B0068
:40C580007DA85E0011E6C800E3EDD1002117F0000BD3DF0043DAB6009370ED00459FE6004A3B2500ED7F530046806000EADB5A0060590A00CFA92A00844F7300A1A25E002C
:40C5C000A62B9F007BCB1A0009D7180018529900C8442F00011F1C0091A3B800DD453900A64C30008A5A3D00234E280059946E0094641100DE14A1003011060040E2D8009E
:40C60000B26C7200FF32E300174C5000D92A0800036693006B8D0400CD5F2300D330DE00ACF21900B30EC0004A76A7003AF39A00284BEC00AA00E900AC7776003544B30053
:40C640009C4C6000DBE36A0006AD9C00AE2A6600B2DA8000AED870003D265F0013C41400B9356A00B23CA400EFCADE00A60A4A00EFED44002EAA4200C58D2400AF1F6100B4
:40C68000EAEF2E0056CAC700FEF900001F9C2600B8C6230060CA840047E79B009849E400DA30AD0052607300618D9A009E299D00A2EE8700751DB80089B4DD000DDBDB00D1
:40C6C000ED47D30019C5B600821C910059F7CE007E726900D2228C00BFD87300A5348F00C3DF4100C11EFA00F94F3600C37CC0007AE5F400E23C570021573B001CBEBE00BB
:40C70000AE50BB0033FCDE00C7EAC0008866AA00B5E30700ADDEBF00F7208C0028CF2100BE5F4B009A390100C1B5EC0072662B00E43A7A00202E1A001824E900A34DE900E7
:40C740002C26C1000C3D2000A8F19900FC9DB10001012E00B96F5B00108CB400385C3000ECFB2100862B1100A919AC00A9071200FBBD6000D74DF6007B3679002A546800BE
:40C78000F5F0ED009CE78D00EB5E5F009BDCD200541DEE00915E7F009732E60024C1DA001CDAED000DA5D4003D611100DFD8E300CD065700E85D250022EB2600C25E2700AB
:40C7C0005F74E000DDB4E4005AD41B0017C4FD007DC54300AD1DD50038C19600E4DDF800C17077008E3C0E000A98E2008ADB2E0070FCDC008EA25A0019937000AB28EF003D
:40C8000050632F007763C5007626C8002ADC5700662306008643DD0026C93900245603008F7AB10000528F006A076700926EC000A2716D000F0079005AB4B500A3C75B0019
:40C8400066ACFF00B17A7600F56CBD003EDAC7009BC02C002BBE680089D967003818CE008FB74900D9BB59001BBD1500F9FEEA00FFB8B200149EA3002496E200A6B5CC007F
:40C88000AB16EE00AB4CCF0099435300A6FA2700F2E5BE00779A6600567EFB0070265000A37D92005D3F1400EAE58B00ADEBC700F95D53008F44050057DD5200D43CE40036
:40C8C000A28D7900AD712600A61A4900F6A1AF0055125A0080A81F0092C58000EEF7B0008B1C85001CDB330098EAC900C0C265008C4D2000B91BEB0074E29100A6736200E7
:40C90000BB42DD0068372E00D0172100F33D7A00F52C4200BC0FAD00B743BC00447ED10078F46400C870D0009DF56F00BF2C7800D7FF340036B98C003C0F51006FCA930051
:40C94000E481E40033735000A1806300BE251A0009A2BA001D1C4600591C7700BC12F70036F8E7000E784100E4464800A9D6B50035491400CED390006CCD4C00754B500088
:40C980003C81FA008F796F00679F4700C01B6A00F16B3100F6BD63002D45180084B12500A2746200EA124600E8EE2800F3A94B00E6FC42001C3D2D004390C8006F728A00E1
:40C9C0004B3693005B6DCF00E1B9D400DB95FE006B1DFE0036DEAA00E64E9500A9E18C00FA26BD007D44F2004B5A1A00F4295A00945AB8000CA0DE002777F00019918300DC
:40CA00001C1730001D0E9E00B36219007DF01E0021787D001D8997002FA62E00F06A4100704D6E00E841E8008437B300B18C920020F98100E9FEE50091D3120077274700E6
:40CA40001174B200449C8400271E9D004169030060104D003B13DA0085D1C8001EF30F00860B730047130800CCFC5C003312CF00705ABC004883EE0012EF8600629D9E0068
:40CA8000AC81A1008E7096003108990032214800DC4C1700F0301200D5FA070023D22100633F32001F0A8E00B677960079360B002295AC00977FB900E4E86C005BB747007F
:40CAC00098118E00C8FDF700C2E2AC0051DF12006DD7DE0085F07400A7ABC5005D6D6200124B52003CF6180099D32600FEA25A00C356F300354DAD00A98784007BD72C0071
:40CB000001250C00A6D2380044F8BD00D59428007D34F10030700E00D27165007C264F00F18D9800C8823100AA18890059ED4800FC74B00019E41F0016C183001E2A7A00DE
:40CB40007AF60E00B366A900AE2205004A8CCF003D389E00F75A990079A12D006CB86900BF86B700D15E2700C49D1400A005B800901C2D00F4A718006F320700F20AD50001
:40CB8000F9B1D1003923DB0013CA8D00E2FD0300DF0D04001093CF00BB567400F4AF240045C94300EEF85C00C7DFB000B64F3100D647B800B69DB000DDAD7B009B87AD00FE
:40CBC000F9D35A00F0CAB000DF391600EA60FF000F3F9A0098B86600FF0B3E00A6E7F100210BC800E7953F0067E08B00C473F6000D274300A393A400743947007D6887006B
:40CC0000033E6200EFC21500300E3000A64E9300C28625003A155B0026122A00626FF700AD20F3009515EF00AE4FFA00A02C2200E6BABE004D89CD0071E4DC000B9F6700D4
:40CC4000954B160004894D00D6B0DE003716E300C6125E00CC936800038551009CDC7D008290F7001DD238000A7DAD002C13F300BF0F210075C5B900662C7F003EC84700AF
:40CC80002358FE00F3B7F400A45AA8002CAC9F00A5E02B006AD4C800363BBF0014F29500A0932A0077FACE0041BC0C0075D31F004FF60500A63746007ED32300BB1E3700C2
:40CCC0006CE4290071634B0063086300BEEFC600CD5EA000F878C900C67D4200D4D0D400936BFD00DC4266008CEF4A00ABC8590041A31500BA436C008A1F7200A1970B008A
:40CD000052223C0087EABF00B0E4F100FAD88C00325FFE002BDF780031403B00D01F61002628C3006F94A10054052B00678D6E003727430079F7DB0095B2C700B26E8800E6
:40CD40004F1A010072865E0094AC8C00B3CF220018BFBC00B6BBA8005F9DED0089A665004E35480092E7270031AEE2009C6DE3009F9EDB0035A19200F4C4DF00FF855C004B
:40CD800097E38500F26DEB00B7999B00E0D6FC00B370A3001FA5D800567EEF00CD1ED5003DC7670068A8000016201B00E2E451002FDE9900E6440900258A7C00D268FE0089
:40CDC00065CDB4008B2635006C62EF003F575600F7A384009A9572000E8D7A00D74EB70019455C0057C9DB004B9A21005579DB00B6018400DDFFC9003E318200D9E54200D9
:40CE0000F120B0002397D200BABAD600402CE90001668E0076C334008B7984007A208E00F5BC8F000CE17F00FFFCF300C5F6F9003137470042F66300CF227200909AB60019
:40CE4000A5BB97008AD3A2008C93B30092021700D855B100AE5DF9005138A500C458D3003F13A1001E97F300B1E6C300436B39007C0806009B024600EC6D05008D1AF900F9
:40CE80009092EF00E6E9DC0043A4EC001848BA00074E6C004A3CE500E117510003BBC90031D63F0023FB7100D70CE400EC1D7D00D69D5F00465E9A00A9F9920051324400A0
:40CEC00052C6C90024548D00EEFE5D00CD87EB0083DEE50041856E00782DC400233F5A00D7C56600669BE8001CC688001BF0E600E5FC8100E6366200BD46B2008324F000B3
:40CF00006763230065B2E600A7208E00F23EF600C20D360090915900386F550004517C001AB1810022FB71006E34E000C505850034C0790081BFC20004A96D00C63E9C006C
:40CF40009D58920078DC4B00CA837700B3590700F1BA2A0040D0610069EE1E0024C4960012B35E0019E7E800FA17D200BC2C5E0079294900C9DE1D0039632300DC887F00F6
:40CF8000354EEB00C0411B00FCACAE009A698E00C18817008AFB1C00AF095B00BD1FCF00A14FAF008DEBB300B0279E00C1AAC700BDE2C200E1F47E0047CDBE001BFB7900BB
:40CFC000EFB77F00D67923007E31FA009F95C700CA98D300F61D3900F69BA200AE56680076BDC1006904B1003DBDBC008906A7006F3517007D759C007A2C4C00DB7C100036
:40D0000065BF980010EBE600BF1C7C00273A160092FBE2002B785900D444F7002996AE00F7B09F000E94E30044BF9E00B675A40049F92D001F8B0D00DBB1C70028A27200AE
:40D040009EDE5F006A5C0100B805F800C09327004EAA900098C29D001FFC5E00017C2E00177A910029D3B80024E9A0000DFFA60078E63C00DDF068005DB3F200E3B5760028
:40D0800041FDFE00B4D73D00D6757700929A8B00D863610014ED8600B98E7600AE9A49003537B600952D2200E420DE000034CF00EE4EBD005F68FD00479EFA0012AB6900D5
:40D0C0009CCE3E0050B489003832BF00F6460100D2EAFC0067638F00F976D6008BC53C006E8C9900050A9E003FAA950060224C00402ED300591ED9003A755500AFFDEB00FB
:40D10000508F74008520E7000DFF650052F0490062DEA10047D796008739E800713836008C7D0D0013E2920091631E0087E570002C5F3800394AAB002613F4008AC1C9003B
:40D14000E4CA340048029900D71DF800A1EE30008C3EAB001F10ED00EA9EE6006976A100EFA96F001BEE7A0084C5BD005D07E700621561008736A00079E23D00C32B8100A9
:40D18000C8B5690045EAE8006AB0C700DBB57E002EF47400B2824E0078A77A00FE033F001B071400766F7F000F3D6C00D0FFFD00463461009D97D8008B8091004AE0A70020
:40D1C000279B1B00AB6A0D00FB93B6006ECBFC00AD36FB007D127100E9B34D001DF13A00547B4C00593714003D583E007C013D00C1415800306F220010B65400FF557C0057
:40D2000091DD2A00C6543F00DB8A0000374CC600BFA9D500670458008CBCEE003BA41800AC3F1A001EFC13001E75F90033E61400A0F56E00527FF200174E1C00F5FBDB0025
:40D240007B9A170073367000B5BF5F000D23A200AA781D00BC85CE006623540074360900458C9D002D43BF0029B56A000F59160048EF1F00B8E5C6000A9D0B000DFB81008F
:40D280002D454900D4069A0095194F00353B1E005D1BCF002B74AA008D6A1200341CC800A2568D00BDA10300F813370090CCCD003B7F1000D1ADFC00489C2D00B8A0E7001E
:40D2C0008F7554000BF3DC00C5646900EF186D0089B9E500297647002411B00001F15B006FD0AF0037C87F0013BDC4001A6A690047C6E200EB9A7E005240D0005B44C10016
:40D30000BD472400D6393E00C249AB00EA09540091E3DE0003EC7E0083B0440011717C00E79F2F00F410BB00DF383100B4F7090031720F0084DDF7001E1D300068BEB1008B
:40D340003CBA3F002B3248005E48910027FAC100145608002FE4280027C78F00EDA1CE00B164A200C6F627003C7039003C9F3300ACC88E00156DD700BB60FC00124C8A004D
:40D38000C11E300053107C00ED5845003E786A0079AB96006112AA004166A500B9CC150020988D00D981AB0061BAB50061B5EC008B71FC00C9AEA500032D0100B97F8F00F0
:40D3C0004C071F00C31E55007DB11D00210B040097B0F700447E6200EC28B0007669C20088C78F00CCDAB100F8D35A009E930D00BB27350022D9260031457D00ABCB730097
:40D40000EFE2D00026C198003FD1ED00592E8900625DA100780C4100530FBE00CD659B0075BE3D00A6C10F003343A100E215BA00367BDE0010F07A0042637F004CB4E900E9
:40D44000AF1FBB00D965C9007892DC005B73C5005DF8DC00E12367006E5E0900AD04400057F45B00BAD25000FA897B00D9B9A9007C12E50046FF8000FDBA13000A9C1200CC
:40D48000911DD600BBA0DD008EB1B3007D4D2F00D4DCCA009050FD00F22A8F00C2E7AF002EB78E0002B0CA0041E3620023F84D00755E7900C863E0007EF87F00EE74BB0025
:40D4C0005B091500435E4B00506E7A007766D5002C388A0070E2BD0060DEDD006D887B00EF63DA00FDDBBD00BE07F900E5A3CC00CA8F3F008563A00004E114001ED3F20086
:40D500008A7DA5005C3BB4008076E20060F22300818AD5000FE35A00D72E8700DD5AD000E27B2A00100ED80094E04C000A058000FE3A0B00BFDF6B001E5514005F52BB00DD
:40D54000B38BF100DD84320075A10600DABB5300122F0D00362F05009EE9A800B0B98C0074BA1800705FFE00332EB200E31BCC00C37DE7008B51D800546381005AB34E00AB
:40D58000F1BDB900E88AA0009CFB1C00D13CA400709FFA00E4A04200335182007D43A10062394D00A0661400F401080080C0F40018079E00D6F1A000219D89006030F50035
:40D5C000D7FDB400FF30F6001EF0BD0086C91C005123CD006FA2200075A95000C79087005ECDE300F922F600E63DCC002038D60061EF8A000AF83000EFF1E30014FD3A0034
:40D60000D9DC6100248E2D001FC6EB0071768E00E54A9A008DE84C00AABCCF00D44A7800D493970014C8630043A309006DEEA800EF0FB000D5D3E300FC88ED001BF19000E6
:40D6400074E0CE00C5493200577E7500B8CAC000D2667900F2C92F00A60E6800B5007E0042C4BC00D00E6D0007E89B00297F5D00B73D7100D92D060088212F00EDBD3C0007
:40D68000B4695B00D184C500D512AA000167C200C42F8F00B34E99005D6695005FB51200D1F74400B9E5F10006B6AF0064D926004C775F004FE4DF006AF4FA007090CD00C1
:40D6C0007B772B007CD975007838FB0038FD60009EC5B400E5E661009D67270022A69F0083475C00946F6200BECA520077E4E00053B68700548F39002F4F7E0006BC100014
:40D7000080BF510054CF6F00984BA900BB528300C9140E0002E1A6008D79A800E603CB0061A48A003D5D02007902F300411DD000A2DD5F001344CB0035CD780084E74800E1
:40D740007DFA470076A98900A7BD000047966F003B6D6C00E4375300336DE800CFA8D900C62B170001E2BD000547A70019D3E9007768B5006004A900C99130009F6A9600FF
:40D78000751A0700320A6C00BC0BE400A8CA3F00710A0600A993EA00B29876001F90CF0005C19900688B3200F93189004A37120094A711006D1472003FF8D0007AF6F30077
:40D7C000F8860000F5F19D009C344100D0A21D000A0DA400E06261006EB4290068562F00306A5E0055C6FE00401297005A085D0052947D0086CC5C0049E65200C06B380044
:40D800001A8B2D00E73B070051465400F6C6790058459000F95D3000058DFA00D83A37001854D100081F9600D8F327009FD16B00318694008FDEF100CCE6A7006F650E009A
:40D840000ECECC00916EE20061861E00E8E3E000E1BC6800615C3A006A4FA4004F2B2600856CA300FA1B8F00C3DDED00D03EC600CC2940003F98EB00D54A1F0085E11B0027
:40D880004AC6A700F29D3F00C8C0A600E0CBE0007F734D00E8AF0300012D890062DA6F00F7B9DE00CF3631008138DB0004B27E00CA36B200E7A6280027149A0026D64200E9
:40D8C000CB1F1800A50CCE00BEF77D0027E3360070F5DA0062E96900F6D07200C8136F00135F4300A8FECF004FA0A000E3F9060094F3CC0068F9D600685855004CF7FA0049
:40D9000055C3E700C1E8490088A29700D7832700E54BEB007F7F5300220CFB005FA2D8001E0F7D0098ED260038BF5F002A418E005708F400392CA100728C41008F1BFA0066
:40D94000D66F5B0096D6BF007E351600C7B6A30089ECC7000C745400C18EB70090697000A2D196006D1FDB00AB5E1A009B1FEE0076469700A2823C005756A40042BE5A00DB
:40D98000D7888900C6453F00355F8400539C3D008F774C0032553D00E28CFB0008CC79009152A40009D41C002D404F005EBE59004E914D00358A2000DC1DD70000F50100A3
:40D9C0006AF28900D36DBC00FEA0DA003BE8AA00255EA900439FB600A11ED5000B9BB400115C0600D386F00043438100FE01D700161E92003CD06500D11AA8000369ED0093
:40DA00001BFCBC00A8EEA9008A5CD6006E37C400E4ABA70026FE3B00878E9B00BB5C6F003ECDE6002F780700E0119A0060F8140044ACC2008EC48B003175C6007615730055
:40DA4000DB866D007B5BDD00872BF700CC1A43000895D500B1774F00E5052A00EB3D3E00C3FEE10004DD97004C95D40065623200EB8B5A0057BFF500BC348A001812CA00DF
:40DA8000D169270054D96100E8F752009BDE6300BAE10600868B350021506200B8327B00C207C600D2C17D00EF848A0053C55700C4DD4800446CDF00B0AD6C002619C100FF
:40DAC0001C989700F221DE00D7D23A004F7AC8007C595700925A95000D20760023D60A0008851B003D9F1000F0A6CD00B53F8F00369CD0003E218600032ABC00DF098F00C2
:40DB00001A78AB00FF998E006E9F4800946D210009AC56004ABD14004F5900000E62BB00A3589E00293110000A978B00245D2200C5976400D82EE7002008FD00615330008A
:40DB40008555B600025206000A11590047498100699156009BBF9C0027757B001AB6EA00D943FA0042F3FC0090999500E473CC0086FB0A009055690084EB20007C5153006F
:40DB80004454BB00037A9200D5E2A000C564350035F7270017B3000026ECF700FFD2A500F5BBD70037138C002EDD9B00A254AE00698455007FC92800AF05E8003AEE920003
:40DBC000E130C600FCCAFA004E2BF80068FAEE00BD41D20083C93A002B9247008B2CFC00D72ED7003076A800BBE80E00CC977700456E6600C5D534004EE129008984A90016
:40DC0000A9B473008A005800F83BDF000ECF20007EB20F004FF73F00205EC3000F977100D15F73001962CE009E92160075A0C3004AE50700A55CDB00A978FA00E5DD6A00A4
:40DC4000ED303500E7B5A90068155D00B49549008E3935007E88EE0007F9F1003CC084009C5201005F99D20013BFD70036046700146B3B00449D6300221A8900FFBDC300FB
:40DC8000AFE47D001F444600F2061B001C6D4C00A9DEFB00C9EAF7005ED1D50070F49700265C0E00811E2700781E0D00D40A500013394C006078CF003FFBAF00A1A1DE0029
:40DCC0007878EB004A7906008B4F8700991E4E007F60000018990E00AE6CFD00286EEC0096FD5A00F21D74002954230068F865001C286600C4641900439C5C006FB28F0038
:40DD000021457800A771F400F6F8A9009D912100980FFC0053224700D4C21800EADD8800667D600088B85000C67221008044CF007A66F8002BD2C6005A90D500E0CD2200CF
:40DD4000534275005B4739005162010063877D000D293600BEFD21001D3BD3007187E400CAB57600C97A69002F0EBA001EA425009C74B500A8F0AB004D35C400E85DAA0098
:40DD8000FC35F600D2EBF800FAE57C0088BFAB004FEA3700DCC9850028B65A00098ADA00FE013800C53BC2009D0D160050F44000B29E6F000CD6C90018D3CE00CADB0800EE
:40DDC000AB846500427C8D00356E4800F3BA66007607C0008ACEAF0008CF84001E8CD3006FD7E20025944300462A4A00925A0D009537DA0061B0FE00B1BCF300E451C60043
:40DE00008F2A49008895ED00BAA5DB00AEF7AB005A2D0800BC91FB000C9A0700A20591005CA97B00B7F2EE00B3DC5400107B3000F1F104001C85E600977DBD00675C840056
:40DE4000E502A3003B88220046A5CD00D798A800E027E6009A321300E817610097809B003AA0540078FEAD0056B6BA00B4142C00520823005C19E000246F7600D57F4E00FE
:40DE8000A7BED80049C10400F7336100A8EDBE00F4BC81004DA26300475BB10061F4E20017FC5000CEC09100DEF2B9002A4E130077D302005DE63900D6521200ADA1C8007E
:40DEC000B14A4B006A38A1004FA57A00489BE900F00F8F000B89D800F1D3450053E70800E00A3B00043C2A00516F2300043F2400F3B4BC00862C8F00243A59008B89510081
:40DF000043CDB2003BA9AE009F620E007A515A00247B28003D093B007AC1D4003FD36A00494F280077DFA7007E17E2007A746D00630DE90041B41A00785445004C51700071
:40DF40001411E9004382AA00D926C9000269DC00D3CEFC0007C70C00FF50760022ED0000D968FD004D45BA00043C3300F5D7350081206D009CAE2D00FB96C500037A9B00D9
:40DF8000CE13FA0023C669004717970085863700F165E10077FECE00E348090076811800F02C0700959CD100A3C0D600336E310078506F005657A1002FA2BC006C717500AC
:40DFC0007A8907006D60570049CC0E0044DE7800459298006A4546005E471F008C21ED003166CC00029B6A0061B0FC00B24A83007100E800229881005ED367005777A500DF
:40E00000E1632800C28EF900485DA4008441C60041ABE70089303300363BD000FF01B400FC22FD0029A35400927D1D00C2210600BA8E3C00F56EEC0029D5F2009C4EB200F4
:40E04000B84A4C0053615900ED2C3800793E6500321B9500A11C1200027EFD00EAEE7F00A6D569007287CA0049ABFB00D7536C0036978900D835E700F4BA3B004576A90090
:40E080009BC77000B3506900B215110043135A00DDFCBF009A1E91008F70E500CA2EC300599FC800D65AE2008276DC009EDCE4001291BD007ECF080041B84000B217CE0091
:40E0C000DCA91300786AF50000BD9C00B2E65500F3C5CC00E14C4C00124B8100C195CF004A67EA0006887200DAB68A00AC6D1400B3FD07001662B600CB951F00B1DC3B005D
:40E10000B0DF8D009A5B7A0097E5F800C4F84D002D1B67003F08040013B92300B0C9D800672E920048282300FDECDD00CF77E3006899140053E7A9003E3D5000C2E1BC00D2
:40E140007FF3490092BC1700156090005263F1001850CC00CF2C81000B057A004A54CA00C2D40000A395FF0066D6F2007912920020A434004D5846009B78BE0080CE1F00F9
:40E1800083E9F400340DD500F71FE300EC0D1400E7FE5200F06F280066CA0F0094D3690038ACE30087779300D10D2600E1C10600B69CD200A0CAC300D83B46002A1BDE0045
:40E1C000E8262B00719A2C008A745A000117570010AC9800BCEE6E00337C1400818D4600EF3BB900EB791D004A576C00F922A20097AEE7002FB05600A7DE290061A08000A7
:40E20000330D6100A19942007B78AF00B39336001D8FCA00AED681004DC89E002C582D00A6ED6D008F7AA300F3789600DFF1E7003A02FC00AA1245003F4F93008FCE580051
:40E240002EB3A900B9AC8F00270E4000FBD20800653919000D0E1200C3CB0700D453B50038759D00891830009F488F0008163300F6415300FA546B00B9A97800180B05005A
:40E280007DB68700487D250078693B0021804300334A2C0091380E001DA252004C169B00EE7B7D00C7EB030020CDBB008F4821006C4134005BB035006C253500A6BB510058
:40E2C00019F635006C68A800A494960003A68200E7C7FA00423A290006C5E90068921B0068C0BD00CF460D001DE7B300BF9E050084977200B0C1A600B7338B00F45383004C
:40E3000024C120000F3B0200DD54D2009FBA590082194000B41F110063B25B004786250029764200C8439300BDEB7300EBC9860076A4D3002C510B000638DC000F0406003A
:40E34000C4F8CA007F7656001E127400E8CE9700B94C08003AA8A4003051C60090B2F500B01E8500D95D6A007ECB4F0097F7B700D5CA010079F859000FBE48005EB052001B
:40E3800091D809005B874D00997E6A000014FF00AA322E0096EB5200617BD900C826FC00FA3321001FAC59006FA89800CD0E4A0007BB3000647B6E0003E22C000F4774004C
:40E3C0004B12B700C1175200FEB80300C92DDE0071CE9D0086892D00EC11EC00555CA7009AD7F8005D077700BF75520041463200FD379600B385AF00B21BA100BF9D3A00C1
:40E400000DDE4700B6DF7F009D144800217B7600710F9E0017AE3E0013CEB3007D5BEC0037AC52008A89730099213700488E8A00EB143600BB51550014D5E800956E92000A
:40E44000D052E2007511A400B02F63001F0ECD006C34270009385400BDF058005069110001D52A00DDA991001CED790093A5B4006808CF006A318300260BCF0077EC53006F
:40E480006F193100F9639000D3B740003DD7F9005CE65400EFDE3F0036138C00FF6B970066A0E6004D7DD300E78BA700289C5700A265BC000B1BF60039E433004B6AE200E5
:40E4C0002ADC36000041C4004664C20057A13F0087AE8D00715E99000594080072C7EA0098BD8100C4FEEA0032F10200DCCD6100E4B423003D38B900FA241E00EAD90000B1
:40E5000018D6A500B55ADD002D8406008CF03900153202006FA39B007F4DF7009AF5AD00A9818100A2E3B9009EAF01004B738100A5FCF300D62D94000469E5001FEA0000FF
:40E540001A1832009D3FD7008E8C6700B0A60900011A1C00B2207400733E22002C68FD0046479A006A3E7D0059BAB40024C2480099E1E200BC0A6A00AC396100097AB3007A
:40E5800069924600BDEC640086C59200C90F8600AAA80400F43BE0007E0A3900B862F00001D37600329A8E00FAAA5F00BDB58600F1D13D005F6E580012DD2C006FCF4A003C
:40E5C000C783DC004C535C005E550E00792AF200E3856F0088DF67005831D000E28E5B00DA907400BA690100F0349D006DBACA00A7F1C300BD93D0006D6A9E00785A06005F
:40E60000E3C1D1003E06C7000DA45300F92702007D41970081F6310090437B004E3999003DEA8900E0EDBE0078197300DDE023001EB90E002378AD0029319000DA33350051
:40E640000019DD00306A8A00D1D02C0098650F004AC937001AD465003C645B009E4F9900AC5914003101DD001985C200467D7600FDE20A00144B0C00DDD6870035DE970090
:40E680009A76150042B93F00EB8EFA00C7507200932E1E00D80D000050288A008AA59700FFA4C90057C7AD0069550E00FAC02100A2F6A6005231EF009623EA0067EC7A0075
:40E6C000C6B9410085B2700034379900CD88D7003965CC00D4F9160052D4F400661BCC00C3350A00E946C000A017E9009C2C1A00E7897600D79CEC00A2203700F4FE5C00D0
:40E70000A35E63002F60DC003046A3006D14FE005390920001597B009042CC00FA793C00BCD6990097258100088C0500B91285005945D70021E758009BF4DC009BBD2500CD
:40E7400018CCCD0008ECE500DE596600219666005CCB6300D82EB000F863E900C5A6AA00E83F12006082FB006280D300B3BBB200A569E200BF52A9000435A500D9C4B200FA
:40E780001BF5F4003856270042E67100494A43000A44D300C430F2007440930014D1020012665000F04EE70079E6A600B0C470002BF30D00A5F21800FFF94300C28D0D00B5
:40E7C0007E4E6D0055FA2C00D328CD00AFE29100CEF64C002802D3000E9658003854DE00C832EA00677EF8008655B50088ECAF000AB8230048F18D006DEE710064AC8E007F
:40E80000BBA3D300A879BE006E800F009DB1CD005B9D76009CDAD6002613430079CF1600527C1700C4891A00200B2900A7C3090000A2C1008332F800F54B0D0023F0D000C9
:40E840002CB13100E5173800993E70002F87B0001506AD009229B80060DCD000CFA743007A3B360043A1ED006AD5FD008FBD4B00ACF48700C7E04900BF588E003D4A2200B5
:40E880005C9212002470D6005508660096EE9600B26DB90039AA2C00B0298000A55E6B0077AE9A003AD861004166070072F5EA0030A30500F6256700D8D94700BA7B670044
:40E8C00041F44F00C15E4100AA32E900E2AEEF00D0D74500C51A6A001A8D16005F19BA00EB4D560055F5B20015AE1100A3049D0011193C003821AD00CE364E00FAFA8100F7
:40E90000D05CD500B33C18004FD2DC00F921CA00DA73D900BF8201004BF04700B4BBF100DEC4CB00C2A60C00D7D4A600EE78CD000C49E0003B966100A90CD500DAF426005A
:40E9400098FAC5005B546000DB6C650004D64200BE4F810096B0C000669A2F00321E7300D350CC0012580300FA9B3A001361CA00314DD2001D9D5C006DE45500D424C600B0
:40E9800015C479001AF14A0080A49E00A47CF500017FFE006E83E100091A7100CDCC9400FB55F000A199D300132200009DED4C006BD1680049629A005E319A0031F9130021
:40E9C00010AB0F00A5392A00E67ECA005CA952009E4F9200A5D14600F4AC62006AF200002684670083667600E33DCA002C5A1F0015899F0018B54F00901F28003EB1C60043
:40EA00003BF97F002CFCAA0029CD79006BB7EB003628D800AED4BA0055DCA400C5146600BF2038005781E900BF85320003B8D800F1B0850016812E0004A93600B6D67F0095
:40EA4000259C12007484CD00D4F41100AD123400554F1200C6A6F800A5B2AB0022FDAC0062DEC600410A3900187018006535D300329D21002DDD15003A58B1002ABDD700A4
:40EA8000DBE7BF0018A858004611AC003615A6005BA59D00E87F250001FC7600E830B9001F24C1007089FC002D7D10008A6461000B77E60021B30200FCF6BB0010A5B90001
:40EAC000C44ABE00CD442900E0D523000E51390093683700707DC200B0E0DB0092495D0018509000CEF2BA0030A27E00964F9D006DC56200C01C170078BD1C00F3123000CB
:40EB0000DB338800AC6CFF0018989C00B5C5A3006D8AFB00472FB00059DDA500246358003FE9AE0034D58B006437D100AA31F4007C0CD1005650ED009907D100CB3F97004A
:40EB40004AAA17008689CC000670020038A7F90000850F006D98CF0024CB3A00582BF20059F4FD006668CC00DEBAB10003EC79006BC8BF0064754100D3F8FB00E0366C0070
:40EB8000AE6636005FE366004A595E00E2D5C500D1FEFB00F6F68600248A5E004449BF008D49B60047AEE70019D4ED0009D5A1004EC9BD00733B9100E6AC2F0048F7C600B8
:40EBC00026AB70007107D10059240E00ACC88D007B6FE8007F907E00575A9000DDA0BC00E03BC5002704DE00AB575800FD224100A2EE1400E9B9BE00073A5B006CAF8A003E
:40EC0000DFFB9F006B662600D437AE00A940AA007D7DF80070C2F8001F5413007243430031595400649026001821B900E3ED00003A1AB200B853950028E9EC008A524C00F9
:40EC4000E51F5600732F11009C25CC007EFAF90099E9E600E2EC7F008DC0FF00A771060065DA950025CC7D00331E9D00EEEE0A009AE42400BFD68500B06A8200BE601400CA
:40EC800026B4CF00D1642900ABE3860019DED70049BDB2003E06C200060301001E649E0041EF4F001602310083734D00A13A860021196000DA0E330029D70300EA4ECE0059
:40ECC00025739700A74093003D759300B6D26000E46D8A008A459100111D5400BA8F2900190F2C00CEAF4F00EAE8FB00D04A6D00A04AD80025F570003BD3DF0066168B005B
:40ED00001995CD005A174F00ED2C840058352800477DB0002A4BAA006086C800810574001B835E00B8955C008F684D001565250003442300485796005366A600CA8E3500F8
:40ED4000A2693700BC07970042530B00B3988600A85EA000917B1A00A96A71002ACFCD00DE9FE800253DB60090CF610041726F0094F8FD00E59C9D00381AEF0016B19A00C8
:40ED80003F63250016B3AD00CBA8160049D2D5003A6B6800AA2137003628A50027519A00B1D1D000479E900062BA8300D5DFC000EF74C10065A6930095F42C00812E570022
:40EDC0008A84D900B7AC98000353750074359100A8AEA200E70CC900471E1000B7761800F2E52B006CFB020027A74F009740DA0098FEE20016622900BC781E00E64EC7001F
:40EE00004BEF4B00E6362E009FE59F00B0D20A0038C0430003AC84006B518A001E4BE3006285DF008B4BB4005935E800567879003D6FB600EB36C5002A5BDF00F4B42300D0
:40EE40000DDBD6002FC9D70006CBDD00962E4700F61C6A00CC30FC007D53330019894600EE9D3500976B22001D36D200EB7349004B078A001E36540043C7FB003577BB004D
:40EE8000522E3900A05684000C200E00E80E77003C6141005F61BF00E2CB6100C53CFF00877BEB0087FA7300430D760020865C00D2B1F50062B05200D2199C004F308900F9
:40EEC0002114590075735000B1F439007D832100F9EDD200E4D6CA003A9B9D00A12F1C0076C6C50069345D0089CC9E00DDB8F50024A05B0074FC42007517FA00B11B2600F2
:40EF00008571D00032485B0004B13A00E0E3B10000ECD700BE75740052946600B87F9700F19B9D000A7A5B00C5F55100CC32FD00603E370024205800A99729003E7BB200FC
:40EF4000D7B670007AA8F100C485EB00D079C800FBEA19006142BD00F0BAD7001E49090060078F00754BAC00084837009AAFC200C90FDF0022B991000EBCE100E9ABB400E3
:40EF8000F5B664001BEDFD003A017F00E5D0DF00CCE2D2004334C6004F78E200154F5C0090061C0036ACB2006677F800BF2F1D0091811000D1045600C1E68300A381B9004F
:40EFC000305CAE000AE257000D392300525DB000F6900000C22E7900B6D39800DCBB2C0045C00A00BF824600574AA400376CC30007F5200053BA02008C9C330033A03D0022
:40F000009BCAB700D27C13003E110A0091452A00FCBFA600DED13D007E5E5B00236692007AC39800D549C80092322100D7ACC000DE7EFF009B322D0064DA4C00B7B8950095
:40F0400061662000378212001074A2006CF0540057586600CCAB8900FCB14600CD1B33002C04A4000D9929006C880000F14F32008491D9008EEED200E626F10071533700A8
:40F080004D2D1B00BBB3450049567100186E84006904EB00EAD992005B6C3100456075002B0D5300885AD7007BAD0500C76A96006E811400899A000017DCB800AEE0C000D8
:40F0C000D3ECBA00163DB400BD998700D68145001657010071021F001C1475009FA7F100738A750079703F00610801006815B8006C3D8E00EE125F00CED18000979DEE002B
:40F10000415AA80012024D007AF900006F84BE00BE4AC50078A39700081D28005CCDD100950873005793510016884500D5EB8E0087BA8500028B560074F843005A14790086
:40F14000C05A8600E6B7E900F336B4005B3F1D00557B6A00E6A867009B2A7B0031F07B000C4D330002354C00EC726A0003EB0300AA4D9900F06F49008EAD95000AE61900F1
:40F18000B1F1B7002A640F0070DCC300EC9BEE00C773C500A4DB85001C6C3E0007ED5F008FBAFC00EB35F300C65C2800DA7B1D00F2BC600064DBB400694727006954B1005F
:40F1C00027604E00CC154200FB3E64002FEA1100BC0A5400C8AF8A001F629A00AA2B0800F7081A009CD0350087C75100D9803900283B270021EC4B008BD84900A297AB00E0
:40F20000648F4600C78D660016FB2300B1F3230012E8E500BAA056000F90FA004E7450002DDAF300588E340060D1C100FD288400E251B60022765A00F612B300B19BB40061
:40F2400006C3A000F97EE500B3998900E3F46900D2D2EB000DC3CF0092577500F5AD630052AF6500E11AAD0045A4BF00250DEB00009A12003EA0DB0064180D00062FA70086
:40F28000B9D56E0019996900514C75002FB2E2001C8DF10091AF6D00F633C0005195DD00B7F7C300B0C7ED00A9535000D613CD002C5ECD00106F5300038748009BBF1A0029
:40F2C000DF5CB70049463600A824530053C04D006AD3010031817E009DA5520061CF5C00FCC5AF0071A410003BC624006A5903000743280079369500CB6D0600F71A98002D
:40F30000BC5A3300C5511600D13F8700608B5A00E744FE005A4E4500F098570002ED4800ACD6D7003AFCCA001FEC66006C80E10076668800F5A2AC00FE6BA300B56E0A00D9
:40F340002D0CEF00AF201C00C9CFD800C90DB4001F9FC20010D0CE00AB5F4900BE1DA000E29E17008D2ABA00B918B1001C6CF00050149E000121EE0020BF2300A6409100F7
:40F38000A7E4B600AC19EE000C9FA6006E0119002CAFF800B61281008645F60071DE530067D94E0010641800B268D600973C600060E1B900FE563A0045A8B50058B17C0015
:40F3C00042DC51006FBFD70042AF0200D8C5DC0080285D00F20DCB0098A28C001F8C2E00CEB0470062EC990083D58D00645DAC0048F47F009A3A3000F61FF200D0412300C7
:40F40000F5158A0047D84D00F2BF220039901E003506E200CB1F7C00B15F4C00DE89920035E2480056FD8100A9564B0049AFF300607F900035E2C000A4098800D42BD70081
:40F4400052A24500CCB0E7001FAACA00721B570024BAD800D1F9D800F3D67C00975D0700EE1B8E00F6E4B80081CD0C004D4BF400F82AC1007BE0CC00391DC100EA032A009A
:40F480009D8E7100543C0800772C0400AD08CE00F8738500F7B491002758BD008934F200DCC24600FF680D006CC6420089516300B1380800B61E9E006982C2001653200035
:40F4C000CC9FB6004C0D4100DF1908008B8BE200F97EEE00E77C84004199D400994F4300B4BCFB002F605600F53468004BAF5600583C3B00D51C23008B9D2500FD4BDA00B1
:40F5000069B3E6009455330041EBEA00D97EA900D4A0880073E57900D28B03003ABF830041EE21005CF77C00AC9550004464B200E6012E0051123100F6CD6700B0A3D600E8
:40F54000F2399700682230005F900500C33FD600745CD1002D76A000A1732C0044CB0C001D4B070089B94B00E7156E0055110C00F1C061004E8D980086BEED00147390005F
:40F58000FB2F29000189690087E5AE001410F900D042080005276E0031B41A00AEF9E10052D4260013123B0061B89F003186D0007B39F9007F6F1300F058CF00846FE90007
:40F5C0009C13A700358BEE00AA149C0091DE7E00193D3C0072926500A0EAF900539DBC00E8D4B1004C4664001081AA0057D0CE00ACC561009D9BE30085D2F2005F8C2300BF
:40F600008E094700E661B800BCE4E000C8F2DD00BFB2AE00C6A7FD008EB4F0009533A600E0F1280094F5830032678B0061F6EF00FEF2E400D73B5E0002DE51003D823B00CF
:40F64000CE8851009BD629001FDCE600F924B400C02C4700727CCA00D7879900F07775003F1CEA00E9903000C79C4500B5053500F5F7C10062D6F700E3452A00958CCC0039
:40F68000FDE27D00BB0D3F0085707600235BBF00D31D48000663DB005D7A9500F80EF400A2104300C8470200DBB44300EEC816009CF859001D7F5E0038D02600A06B940005
:40F6C00053E83F007873F0003A1C27007D9E5C00C703A0002899B600CB886C008B36C700E9A8EB00646D5A00BDBAE3007EA6C000B80F6B005CA4E7008DD3A40052AD0E008A
:40F70000F80C4F0014B3190064592900F913C200A7BE180013DB6C0092DCEB00F80DF000317E92006CA76B00FCBD9500D867A500F0787800DA6D20003EF10000CF06EB0096
:40F740004F76FE00F10F0C002CEE9F008CE27E008E086000F31F0400B71A720094BB9E0078806900EAC8DA000AE0C90048E51600D0DAE4009F892800D5FE8C00DA42440059
:40F7800000822100283E7C00EECE370067B3E000AB53120077A7D8000A1B0F00B5223B00A14F380086BC130091AA160051DC450025B74600ABE00F00B3B81E003E764A0008
:40F7C000324356004B2081001C48C700897B1B00A54AB3001ACCE800082DBF001175F800C4C38A00B842F300D9315500C3ACCD0064FF2E009CC542001AEF4F00104FD200D0
:40F80000E56F310027241E0059244500B1E2E600CC541B001FD15D008A9700003500DE0096107600ACE0F300AA194600B8E22F00233430001BCA4700BBB46B006499880064
:40F84000C5C67200D55C7400148CBA00C09C710061AEEA0052635100AEC57E002B2EE70075B1B6000B6E8B008E802200DF789800F4DBA100C4814500D7F8D200953EB4006E
:40F8800007BC300090CF5400BEDA7A005C8DD000B42F3100988139002E476400E872B4003354440063EF4F00E4B83300E7CBBB00ADF20600C6B30100DC26DA0054AF2400C0
:40F8C00017F36100A08E4C00F4444F005BB6C000410395000CE82F001D7AB900ED8657009209E100F23B3900E0F78F00F041E700E3230000EFFB0800736F9200EF51840025
:40F900002B6BC400918F560040E6E30045EF87000DF75100DB2B71000E7BBA00E6C57E00C1E4C500A631BE00231B9D00609A9E0093CBB000A2D44E0077E0FF00C8529500B2
:40F94000E7843700C02725001125800085819D0045EFA200F6B4A10063BE4D00B0F1DC00E6EC81006017B4007E2B1F007E4036005BFF6A0061128D003C8AEB007F68AC0032
:40F98000879BB1001E67050000DE450066C26900A4FFB70091D8A900FEAE5900D4959200CF5AC00082E5C100E7B6A30079A94C008F1BCC00BD9D6B005526FB0037A8D900A2
:40F9C000E9F8B7001DD6BE0019A07D004538B200BD43B900276EE0004D85CD003BA4D90038C16E0001372A00CCB86200BA793200FA1C4D0009B5110019634C0024479D00BE
:40FA00000E368E009B293600AE542E00B8B21D00FC591B00A6EB9300061920006C9306009C878D009ADDA900DC7ABD00D3F63D00D1137500AF2D4E00A001A7009F94C300C1
:40FA4000208B4D00DB78A3002B16F4001C3202003D190800C5A9AB00A74053006573D300A9390A00A965180033C8D400ECAEBB005CDF9B0026BDB3009F00E900B5B63600EC
:40FA8000B0F92D00DE0F810057E47C00B6DFCA00CF74A700F60F4E00C1F45A007B9D2800E9E3190081F72D00BB950A00DD63CC00B0832500C4A70D00E8FE33006B3669007D
:40FAC00028DAD80070660C00A74089008FD97E0016EC1400F7577E00A6A0D00061B8DF000EC3B800576F420044A86300B251C900D512C400EF9C4800B61A88002FCCCC00BB
:40FB00002D811F008BFD6C0096196600F884980064EDAD002FA6F600CAAB06006B3DF800E050CB00C95E8C00EB16EE003CB4AA00E2E8750036782400521C5B00AEB5D600AD
:40FB400046ED74003E0E9D0046ED8900A9E8B7001B00D800C9D2C0004CACD900805D0D0088181000BC650500C8E8520033F8BE008902F200DCF6AD00F94994003C07BE0054
:40FB8000634B560087D29300ED8F09004BA2FE00D1C2880030BEAC009347BE002FDCB8001AA39500386A54002E50FD0032A5D700425A15002AAFE000D3176B0033E5AF00DE
:40FBC000CA71F70070805E001F40990004766B00703A4900C6071100351A0A0044D1AA00077F5600E9718E00C26140002261B000FFF6DE00971A460001522F00A92BCA007B
:40FC0000FE88F300F6400400E29541000C226600E59A310035A40900C4460000E8667200D7BC6B009949AC0066BFB60025B4DF00CB3947005395400033A8DB0088E3E700CF
:40FC4000E79BC3004A2EA900C7566D0053765800BC8F62000F0E7000A7B3A500326B0C00AC299B0005DF470086A86700317003000C04FB004AB5E2009B98CE00300F410050
:40FC80004D5D6500F976A5001A800E00DEEE66003D0A14001E33F4002FB245008A8D20004B97D40039DDD20051CBB20015F6E000B6FC4500BAA2A200CA1D1D0043D746009A
:40FCC0000A30B100F8E81B00B1F629005353140047A74700BE64C800B43BB2008925B3001A7565003B51E7002AB1A3002638D100E0802B00CC4D1B000363C0000506E0008F
:40FD000063E05A0081FC7C0053118F005EB23D00223F9800A8D1AD00B1CA2900BC583C0098716200F0D2E1008AB43E00DA8C8B00E1AF7100DB6D1300CA892800D53E8400F1
:40FD400030A4E800C1A590002B403900A994C6006F6F6C0057CB3000DF65AE0003CE6500CB331E00F0A76D00E83B2500E0784000AF16F000158E2800D9F7790095551000A3
:40FD8000CD7A9C0008478D00A365AE000C62900088EEC5002BAF7000A6738E00269F0F00D5442C006584AD0047381E00B5BEF000D5634A005467290092B5FC006B91D1007F
:40FDC000CA321800A79E8F006C13A100EEBE36000852B800C9F25E00AE615D00AD07FE0057B17F005494E500B572A800380E870011D4C60045895B007864740079A006009D
:40FE000017FD09009CF16D004BAFE9009DCBB400083F79001CD15B0092A87B004FC42F00E643240051CC40006F362D000F23D500BC739F008AADC40025B70B004E6C33008D
:40FE40009CED8000245EDC00473F4E00AE9F190050692600B96D0A00D879EE007D0F2400B22E7500B6249000E8958A00EB204400110C2400D479F5001914A40051AFF10089
:40FE8000AB2D73007742B00018AFB500B16A3000C59C0F0009C8A000FDCA7200472DB400FBC43300A4A16200167A9C008A98F10037C508001F8F1500E33FBD009E798C0064
:40FEC00040B88800FBEFD800A275F1005CC87900FBA77400372B0B0080DA7300A7911E0064BF1700716DDA00882F9C009ECF600056D8FC004B8C66009116F900DE37FE0049
:40FF0000870492007DC901001962EF00FF64D10057213400ADFCF2001E068F000F09D900D006440018BF3200E3A3750029313B0027C4D200EEC84200841C6E00F349B6006C
:40FF400039234900B713BE00795B3900DA298C00FA6A4F008DC2E100749C3900BD2848005C00850069475500FCD89600BBE39D00CEB0B500CEF1550021A7BA0071CD5E006F
:40FF80002382BE006776670088C09A001852000083AC0200CF3EAF00E5472B008D31D9001BE77400593A4900BD4B3A0041CB2C0020D239004717DC00B9CCFB00B6E290009A
:40FFC00087C63100C0861000810921001AB4DC005359F300EFBAAF0069476B0078305700F1C52D00CACF9200B9F52B00D7AF83002115D800BF02EB00B18F6700ACCFA80053
:020000040001F9
:400000007758D000578F5A00B4D9870006C31700EADFB6000FEA9E005A4E6A00B871A80041FE3C0048764D00E5686200D0EFA000FDE30900FDC6160076355D00C1747800E9
:40004000FE6919007ED088000BA5A7000C97FE00E7528200034FFF0062BBEC005307F400566881008FF656008E6BBA00DC727E0054A3BB003475F50054E1250000B6510085
:40008000AAEBBD00F8465600DC6C7800110F8300E2224B00F00DD700C4053400DCAD1A009B3CD200657BA600A698A5001C706C00B293AE0065D0960035092700FB46DA00EC
:4000C000A06352002D4A9F008812BE00D63EB0004B3E1500F188A5009CB59500A3D14500BFB22600C38E8C001F486F0054470B0005551100E66CFA00FC69E80051ACA2008B
:4001000074CB330074C99E000E582C00479B8F00A8B81300292B570035AF5200AD092400F2B7EE0001373B00D46A23000EEBB400281E7F000E273500DB6FEC002BB3730073
:40014000AC09E700283D0100041A340097FBAB00885CC900C2321900D858D500706CDD009DFDF30010891C00D9F4F5001C64D2008B7DBE00DF804C005053010066F067004E
:40018000BA7CAA002FFFB50074D43F00B75B660066767600897BD100EA836800A8659400F8C66F00813402005A1CD30066178D007B67DC0013B18000B2F38F004BCC6A00F2
:4001C0008120F200A2349B00FB57B60059222400EEE83400B57EA600ECE9B400D2E9EA007E32BE007E65F60069C4D50097D4DF00FFA817000CF88A00F6DCC50037E039007D
:400200008F488300AC4A6500DBBC2A004E827400A94B0600D07FDC00A998B3003F1180001DD1020000F7CE00B20C1400A346B5008C3D2F00BC321D0055BA28005FBDE400BC
:40024000478BD3001BFAE300327D8E001DFAEE001BC4F9007BAB4A00A9B49600588D6100C13D48001A6A640072E5F900E8F1080087171B00D19C0800024158008CE2310057
:4002800073D28600B1037700A316F80020C4F500EC21C400593262008813EF0089FC720019EAA900C61D390004051600C0CAD700CDF3E700EE4B3E00DFCD110078222B0097
:4002C0007BF7A700BA4F190077B7C500ECF4AE00390966006761230011FC66007B412F006AC36D00DF42FA009393960007B869005C0DF70027358700CE618E0060D7110070
:40030000F708A7000780970012CCBA00C1251C00BABE800007F30D00128423002ECDAE004B902000B53BC600A10EC4003642F700C72A6200B640960033A9FD006F9F640041
:40034000AB698100E7706B00C0861F005952BB003B135D006220FC002E7D1A00B84D7D0004F18000A3EA4500ED390700A3E6DF00F113730055637700229CAB0031829700B6
:4003800083DC5F005344170066133D00AEB02C003411BF0063CD1E009DB5CF00BA171800609587002EE9250054D3E400DD1AB50067FE34005293AD00BBF89600A21BF000A5
:4003C0001269EA00289F1D00E59E9B00A7EF5A005E6E39004FDE08000034CE0045D5AA0041F28000AE524B0088D6200096C53D0087F4400004E4230050E42200B4CC5500A1
:40040000714DC70030FECD002F37D700FE2F66001E7F6000EA8AC000332FC70074FB990029FBD2004A80DA00FF881900111F3A0096E5B900B1B7100078E2C100C2C35A00C0
:4004400056FC04004C98D100BD132100F1627F00C18D8600D9E1C000C275C6000749F700C1E5D500AE62CC00A5036A00767DEC00BD8970004F3CB300C04A72007A73F60081
:40048000703B9A003E2F6A0062017C00462C3700D1A9B30049187800CEB14400154F630053644600008F2800E5AA1B001D4C17003F0B8600E6EF7C00F1EF1E008F965A008C
:4004C0002A821E0085D505004AAAC00008C0D400B396AE009BB99B009561C2006435FE0025789E00BA9BFF006FC68800F3BD8D0000914100A355710089304E00C8BDE0001E
:400500004D23DC002CACBF006C717F009B1AAE0097128800860B35005F37B900AABD9B0006E4320018898300C493DA001E806C00013F6700D5CF6C004122F800D7B54E006A
:4005400054E67F00D2D59700BE1E6400915E36002DD3A100B0D3380018F72B00BB868F00C1266100290225002B1BAD00CA056600B636E70077E743001FE91C00DF97D50016
:400580005D70950008F200001BF5F200EC16A000F7B7AB00EF1238009FC8A0000CEC7C00D508DB0061EDF800CE246C000E155F00899674006B234400B74ACB00A3BCAE0012
:4005C000563C1600CC85640087CA82006F3F2700260D3C00C19A8300B7E1C500AF868D002172A7004AFA670027EACB006C7F1B00D17A620044ABB600C6BE9200A41DFF009B
:400600000AC545001CE4AD0086B30D00F25F7700B20BFC00868A8800E0AF5600F35C6600637CE10059F41000A6F83E00159C4600567E820074212700A1243600681C160069
:400640009BC9E500B295AB00E7956C00180E0600901AED00D16B2100A92F8000455F21008D084C004F8BC9008D17720047D9B800742E79003C821600008E7D00EF8121001D
:400680009AD781007EF3EC001952EA00B223620016730300095D9600BAE29800183ED4007FE264007923F8007910BA0080C6E8005D0FB0006E93A100230E2E008D2BD90001
:4006C00022AA240081D73C00CE07DA00BC6C7900E85957007C763C0073E64900785ADE000F012200E9A9C00011030A006A77AC0006AD4300ED44DB00422FB2000BD48E004D
:40070000C66395004621B8008B9FD20074D4EA00832A86003B421700BBC679006420E3009B9A8C006719DA0024DD1B0002CDE7006F0C8A00B2061A008B4C900049DA9200A6
:40074000F8A946008CDD9400A102D000077FE300DC2F3D005ED1030089ED6200197D42007E515C00DB0990001EBACC009AF3970080E28D00C9E51C002DD78000F03953006F
:4007800042CCE40027FB6D00788F5C00763EE00058285E002F224C003689B600CAD485008CCED2009DC82600FAE4B9007C5FD500F8C314000AAFB8003F63BD00FF90B500CD
:4007C000BF0B060097F8CC00F709CA00519EAB00470C0E0077E9E30067DD3B0093A614002CC8AD00934B3700F539A300FD39B400FA678400056F000011954C009690C70051
:40080000DBBC2300A36D130042A05F007A87D300A8181800BC0A46002DE10600C44A0100DA5B43003D237400C11BF500867B1D003AE5A300F314BC003EEC5300FEB9EB00E0
:400840000857AD00683E9500F001F20018ABD300D55B00003E69E70034032B00F8B4AF00E63DB900D1794800E9A35A00B14B230012639700BB42C000495F8E007F27D10054
:400880005420280027C79600967ADE00A6BA4F00C81238005DE3010063C4010068C290006867EF0094F6D600C461020016902600903DB100FB18DA002C6411000E822F006A
:4008C000253D7500D4ABEB00E78F2400F09A7900999D6F001B580500619FE900A0827C0024B1CC000FA63D00A63EF200D6D1A500FBB6D200D7DEE2002285070006619400FE
:40090000EAC51E005460580043FC1900FDEA9A0049430200855655006657C5006ED83200C5743500511ECA00B22DA700FC791E00E87A20002CDE3B0004DB0600C145420099
:40094000CF6F1B000DF07A0005C9B9008CCB0F00C3A53100E6D0CA00D8B135005EA8EF00FC2D8F00493D0E0063AA6500BCDDF900B7D11500E0407500843A0C005186D300F8
:40098000BF74AE001BE57F00B2A02F00978C8200455F7100C84B1900D59939007EA55500D1F1E900B08189001A16CC00379E7500C2D0B7005F5337001B3AF4004363BB00CA
:4009C000521415001E49C3000AAAE6009C032300AA9FFA00B530F5005AB44B00A07B93000434F400ADEA5C00343F0D00B920C70087189000B54C4D00B3EE9800B5A79200EF
:400A0000612C220065DEAF00C7D6A50002408D008803C800F2736F0000E3740047486D00A7568A00EBBC4D00A3264900D2224A00C76B3800995AAE00D3DCCA00FE65F100E7
:400A4000B44CF100C6C443004212A20005D6610088660300D7E1150077407300FC6BE000FB50DD0029DD6500169CDE007D38B8009079FA00F5984B0001C3F100C23EEA004D
:400A800023344A0025BB9800A943F70033879800D0E3B10019C661003B24CC00C1BC9000BC4E7200193E1E0095CC8D0081F29300C3DF9900ED23C50065245200C69B9C003F
:400AC000404D82005400FF001DBE730053C335004AB1BA00CC5A61005F8EFD0015277A00A2A29C00D6EB7F00432F6100DB096F00EA0068008C2A410072033900EE30FC00C8
:400B000067A42900E3CE710012EB7E00B0BC780016933A0048AC48006879EA004FBBEC003F768600C830080047095900F7E62D00777283000E9B8400D41FF70075FDDF005E
:400B40000DCF7100DD7A0D005E2B6000DF039A00B66EE000F7D660002A63CA0073455D00F5805700DAFAB900E5F1D2006583AE00CC2F8A0070929500FBDD1A007376DA005A
:400B8000D44A6100923F1100DA98D200CF4B8000EE3145009FEE85000020310019E71900D543C200486F7F003342E200BCAD220063FACE00561B8100E8E83800312E290077
:400BC000F6057C00FEAF2E002C28A600AD2AB100929ED2000F94C700F8E4C4006BFAC900925A190097CEE100C36DE400C166EC0011C0D400F37D25009474FF00157E610040
:400C000029F1EC00C8FD7100F1CD4300C557E0008E93190089ACD100C7CD7000F29BCC00BF0875001F7FC800878E67007F360900BF4F7000D025720051C1240097E45C0010
:400C4000CD2B24008BB7CE0075E5EB004EEA2A005ED48C001CFB9B00CF03F4007B68F300849BB400BBDAF200C417170090A711007A5D7B007E118E00BB168C007127E600B7
:400C8000211B4400F7FA1B0006B5320072B895000679D000FA0E6E0052930B00E6A2E5005B3B0C00B9E9AC00813D5A0088E316008084D5003D30D80078C3B600D36A3B00CA
:400CC000ADD5AC008FBCD90048621D00A40DFB00310B4400AB16B30058DD2100A90D8F009544EF007D22C800759BF5008C269700676B8000FDC66C00261776005AFB560044
:400D00003B5B6D00EF33E10000097300C0309D009EFC19009519AE00A04F6D0010B5C300E09C6A0073737400B35415006955AE00422A6D0074402C003823670044A665001F
:400D400033EDE800E58F8100880A4A0075EEBA0060259E00424045007AF3D200F696A8007E75D40095BCFC007CB70300FFC65900EE21E000F0E4160044D56F00C0FF160082
:400D80008A34E0003C697B008BF25800D52A43001B363D009C081100E3756A005602D5009B1F9C00F920A600CFD3580074063900ED3C85008343B700A4EDC700BBA6F8008E
:400DC000DC89F2000A217A0014FCF70091BAA800F6755300CAE0FC00B6184700E7497F00DAA1A4006773E400D17BF600F0263D006FAD1B002F1A37007BA03500B3C50600DE
:400E00009B02DD00120A0B00B45E500003F0AA002D637D007A5290009ACDA500C9E5F5002FCFDE00A4A17900F0CB9A0099CD6400A08A45000DADAC00A9F9F800A6707B0041
:400E400008DF0F00D6A35D00198005007856B60038AB9900DF6420003070A80057D6F10068E1FC00AA610500B834A800074547007042480067FB8200C1091D0057667F00C2
:400E8000002C1E00E0FF300054B28D0071DCEA00467FAC0045C05900FA71E0005B0E2A00867B430065496700B82BB20050106B00E7F64600AAD87A00F2785E009D22A20061
:400EC0007EBC0B00683845002BF9E400CC69A600CFC9CC00943523004595DA003707DF003974F10028886000F15E5D00E2EA540049F6CA009A7ECC00FA12F100EE7BB9003E
:400F00002D903500E92E270083D27300E64E9A0088349A005AF1710019D295007BF635004DCE22005A1DC400E2A1B800579D7C000D53FE004DB17500B85D3700E7A6A7003F
:400F4000EF486600E8A21F00449FAC006D287900F6511B00DE7CB6003C95A100D46D600095651800E880F30093005E0091E1EF00D4B71D0025A27C00844475005DB5980078
:400F80006D7CA600E0CC2A002C709E00EFF54800948162004721B5003EDB23001E6B8E0090CC37008DA6C0000E49C9001D2D300056334F0044902D00035D5C00EA33290084
:400FC000C4F40A00DA4086009C2F7100402D07006C0D9A00368E1300AAE6F900C8C7EA003F29D900DD2EB3009FC4B70030458B0052092700D53CB30064EC4D00C23A2700D4
:4010000077D68E00CBD7D6000D942000BD2406002D1DE60083B6C300828E7600999AED00E56D6E00E5D582007CC897006F424700BCB6A600A9B0FF0020DC2E00CBE5420088
:4010400096DD74003047D40004A23B0033D10C006F2FCA00FD2EE400F644D900257CB200167781003ACD1D000B101C0017E69400F6F32400627B180055E54400CDCDC40098
:40108000F02B1C0011021300FBCC5800C69FB700F330770020DE8C008359A1001AC7AF00B8B26000E6C723007826DF00D48496001FC58000BD910F00B53F4B00DBDCB700F4
:4010C0001D338900FD05FE0012C00A00A71DB10062F0A000CF47D700AA30A100784CA8008085E30047C36E00A33EBA00BD1F3D00DB56AF00D8D24300B1459F00B75C5D001A
:4011000075D066000AD4920051AE1800463289000AB48D0029EEF800EB7C31008E067900D9C3210082D060001BE67D004B553500808E1F00DC1B7000F3FA9000F1B97B0085
:4011400031ACB600E900DD0092169D0063FA8000775F4800A5B0CC00241B35003FAF320051B34600B8034F0021CF0B0013CD1200716F1E003F78B9007D8FA5004CC33B0077
:40118000645FCD0013DE08007828F40083F6A100072D0E00A4F459007BB91A0013C1D400C2FCC800BBBAFB0056B96300D00FE100D2C4E8004843C7009F770A00DFA5A8008B
:4011C000A1CC400020ACC500D460880075439C00C9DB890084ED8E00553FA000C3901D00A74656009DF47400A48A0D00985A3400B6E96000B4122700BCE0A4006C3DF00063
:4012000039A5CB00BBA44100461817002BFD0D00E8B00A00A1457A008AB8960045A72C00F6B57E0074D43B00D2D57100C14F600072AB0100E383DA00E597550006BEA900F9
:401240002D2802004D4D1B0052056000EDF3AF0081985500A14C9A00EE488B0036670A0063CB780019EC3E002901C8002FAEA800C18E6B005A3E96002C86FA0023FCCC00E0
:401280009E1F4E00DEF9E000B51B21008C021C00C52A1F00DED60200D2B57000BE5FED002A06500090F022003552C3007534250001DAEC0008D5B800BC589E00C5AB6800EC
:4012C00052B1AF0029BC2200BEB167000B12E500BCA042007C5FBF00E1AD6A008229F200E2A00400F4877700CD11D900894247002B47D6001605C700ED4BF0004EE8F100D6
:40130000D13616008B7F3F0078823200A664640059613700092F8D00C78B8200A7B231005599670008BC6B003F2CA6004CE59F0001182A00C8513600AEBB1900A0F5E300A8
:401340000C89B10097743000DF64930051079A008FB43300CB9D580011B9C1005FEA28005F195F000F96E100E5377600834123008CB2C8003651DF00F160EC00920A610076
:40138000D653D600448121008A6ABB00719F67004BBCDD00BC832100BCF1680061EC740096DAAF00A55C4100E7ACD400DD08D200F87878004FCF510021022F00C7432600B0
:4013C0006995A500C4DE7600E4201100FEA8B2006E19E400EF80FA001289B10003C93F008C5A550010EB7600AC83DC002DEDDD0049DCE60010E32700BBA17100CF941D007A
:4014000016A90800E1D0780027E25A00F2B901004D56C5007CF24800152D1600D0A48B0019149A002D5B5100971F2A0044ADB100F9472800ED334400A69B8800E43D24003C
:40144000FC847500176CF6004FF6BD00272E5E0060FAD60041289B00F5069100CA4CED0041EA2D00A9F6890095864B004454E200EADBCF00B7DE2600DB27B400CCE09500E0
:401480008D37650065EA6100EF39FA00FDBA0F00CBD97500270E1900BCE6830080DEEA004C8B3D00AC216B00AEAD4000999B0B00EC62770002E39C0032887900024CD100D9
:4014C0007D55E000BBE0A50041619A00F4F29C009729DF00C3122E00F6003000A9C3EB00A9533F0061170600D344E800A7280400601EEB000B7D7F00A8C55C003A65CB00EF
:40150000CAE10B00E6FDAA00E98A4F00F0F1F000F7FE55005E6DF1002505580012E85A006546D8002C97A400F7D1F90028D534005A577000234E70004D227C009C2D5C000B
:40154000BF0D7400B4E7D400E4AB00006530E00009202100621B0F00764E37004967A3002B43520003EC2F000DD96000D6FDC9006BE5C8006DB846005F96C700E0B44C00B5
:401580007302F700E562E200EAD1E30015942800B9771100FF05A800CC537D0059DBE000AEEC4600C5A90200C84EC700F7D559005478E30037272A0053B32000C79B770002
:4015C000A2F52C00A0E6220020682E00590C020030A3EC008F33BD000384A50025A70E0069CAA800A14DF00047AFBF007883840060AC6000A0835600A8F293004F13250099
:40160000A6A87C000376F600E931BF0093369D005F4B6B00C85F190089E76C00A5B1B3009718D1004EAA98003D9799007335CA00D9159B0071E5BA00B7B4D4008E428200DF
:401640007A43E5004BC6FA001158F60074374D007C999A005057AC00BF7A110057A0A000597AAD003904240021145C006D576100D4108D0054B8570035C3AC00C6382B004B
:40168000E703ED00CCCB6800E1967E00B8EE9000E76953006A0ACC00EEC49500537E2D0099B54300F1AD1B004FAE8200CE979F00AC444C00343ADC005DA3BC003B539F00C5
:4016C000CDB5CA00975BF200B6AC7700759D8D000955F3007AE02900724D9A0016250E005AE90F007ED486006ADD4B00F7052D0053C59800C049FD007AA175000EB07F0064
:40170000329B460022375300553146007EF7BA00E84C9B0080254C000F0B680054B0FF00EB0AD70031160F0081D16A00CD215C008A8C7000E7C8AC006A4BC700B6569F007A
:401740003E1693004BDBB200FCD59500E0BE4E006B333900A979EA00AE8ADC0041F35500DFB02000D9550D0051D6810040BAD7003B07A1005E275900C80A3A00B6FD3B00BA
:401780001D1FD80037E02A00C130FF00B4D65600BAA891004A5F6A00001BD6009DF3B900DAEE6F007438CA00071A1800ECDEBD0055F87A000789C600919FB70057D32D00FC
:4017C00087CDFC00F4DB870028BFE40016E4C400CD9C44000143AD00B7E02B007A06B10090B07500541B4F00897A4F00120ED700A65A08004E845B002C4E2D002079DE001A
:401800001BD95600286401008B040500B292DA00684990004B54970041951F00463405002D251900EC2B54006A84CA004044B000BC1CF100FCF19C0017D95C005AB3520075
:40184000E45EF6004E8EB3002A79EF005A696B00E32DDC005DF8280056D98D007022180067E00E0063171C0003CA1A00964FAD00EFB23A0065E1610052896D0089E83C0037
:40188000DCB00D00A3371300F43BC1001F418700629D2600C154B40063C27C0066D77600FA28A1007F68F70009BD6D0027F4DC007C80BF00D8B933005FFF9D00E200AE00B4
:4018C0006BF0FC008A29EE000A6B5400759EA900866B1200FDC89D006BB0A600859C4B00A8548200A7107000D8E99A007CB761000A074100D3FBEF004C9D400005F74F00C2
:40190000FC3FD7009747C300FFDD2D002148EA002EEE4E00E9C52800A5A0980044759100E53B5300F6822E00BD21BE00F79F720020C60B00EEB92F000B05B6002D96DF0045
:40194000EFE5FE00E5820A0042A5B600634D6300943C9A002A741500BB604E0000635800B395CD00AD20B20022935D00DAEFDF00C86B5E00E88B8500E6993D00EF53580006
:40198000B23EBD00D81F420068BD4100A9505F0045878100D7EAEB005FCC0D00B5819100539F2600B91892004F383F0040716D00BCC54A00414D00000925D900414418002F
:4019C000EFDC700087606800610CF000546656003358900050E4560036E7B30022DF5C007AE40000D62B220000330E00FECA7C002102B100E98DC600923A410045568E00D2
:401A000016E4AD00258BEF00435804007758AA00C862C7004FB6A800BBC12500D8A22D000955180072FDD900131ED9006DF8FB008DB78200A0E9BE00C6BAC100687D78008F
:401A4000A8E091007609A2008881D30059674B00DE071100CAA1AA00B45EBB001AD2ED00C14A6300C6E5E500F44EA8006D1EF700B00D4200F388D90007D0F800A269B60047
:401A8000FCE5820003B56000406C7700CBBD6A005603C10034289C00CA58910024C73F006E00BA005C842B00AFCAFC00FFFC4F006FD7B000C47B520063A0B20078590200A6
:401AC000B5684D0010B5280066BA69009374480096FF6800AC07120045450400581F20008ACF2F00FF6FBF00BF11A7007E1E0600E28FFD00DF346900331AAF00C9D8030078
:401B00002074CF006B38D600861D6F00DFF728009705D100B1201700DE8498008B536000641ACB003A6B0B007B67BD00F0811800AA729E00CE9DA000B62BF20089CCB80066
:401B4000228B8E0078B64B0078639C0035B923007B110A0004B64600E345500014EFBD0007AA320017BC4600B520F400EEB7F600C5506300B72D7B004FF5E10047E73D0094
:401B8000C1905A001DA3E3004FA6EB00D4998C00082A050077A3E200E92853008F31AC0051865600E6049C00B23C14001458B60035EEF8000539E300A5F5550051D10500D2
:401BC000E20A16007BE9000020263C001BAF47004549DA006F2B5000F8C711000F640D001E12C2006AD2E40091965300A1B49100DE50C500792EDC007687EE0002EC330056
:401C0000A08175001EB17100C1D2CE00C6FF1200CA2A08007A079E001EBA8C0085F8E4003929C800D7260D00CCB2070055D4CC0034FBAE00D6BBC100174FA30033936100A9
:401C40002DD9EC00D9C02200606B7500F23C7B00D951BD0041073B0046E09E00B101E200C287D300F67AB200C6630F0071686C0002A55F00C18B00000D6CAB00CB2C87005D
:401C80009765E800E8AC17000FDAF200970149002A4B7F008E8AF7008CA500007C7681009EF4A700B6FD4200E3224200DBC06700F5D4410064AA4D00B8B89A0049CE6900CC
:401CC0003D8588000AECF2004884CB0099B5060087F26000FCA40E00BE591E0007157300319F920073056F00325CEF00B563B400CFE70A00AD97E00027D44800A470360079
:401D0000835DB2009B340400ECA643000BC13A006B554800D5C30200BE0EFF0015A88D0097BABA0016281200A8D41000077A6A002ED509005BC14A009FE04D00FE09120083
:401D40004D961A0051AB1E00DEBC43006C78730050A18000FF350400B3AD6A00EF0FFC0007B8E10010F7EB0033F0310019DF9000F1BE08000EE715005FD6080019E99900A4
:401D8000B1F5E600AD56C000F2543900FE400100296773004DC44900F0F17A00E7C87600FD7DF300AA3E92000FC06E0046EB280083A66C006F93210083102200DAD1D100D3
:401DC000F1466B0044D6A600AD2EA5002FA65D00773D0D000FAFCF006B7DC700FC81D9006A41C8008D7AF100DFA6B500ACBD960010B7FA00661295005E844900BEE90E002A
:401E00002352C200BA229A00A475CD00F7D5EA0088075B007D829D003BF272009C7F9C0061EC6E00DE7CF7008342600020192E0096AF7D009CB7460068A48300F8EAA00079
:401E400032CBA300A17169002B5A9F002EB24000DA6C9C00EFC4820053C8E9000467B40040B6B20008D4D8000BA74A004EB00C00671F79005856AE00E5DD04005A3FB000FD
:401E800024DB850069CD0200A5BFEE002EBEE3008108B1009340E100304A84004897F400951D8D008D12FC00F1C6DC00E0CA55003CF0A1006617BB00C55124003E5F0A0034
:401EC000E795120062B58500B4ADDE006AECB700F57D5700578D49008AA21C00201F2C00AA0E410011C4FE009EE9230080DEEB005CA106002595DE00B094FA00094C620074
:401F00004A966A0040024C0004C28E00D269C8003DABBF005E152600A379A700C874B500AE68DF00B148AA0076D84800DBB3A9000451E900FF3A5100A68A390057179F00DB
:401F40008CED3C007A2FCC00F5421600487159008A5730000821D60061C5D40021C6DA00A55A0100F6237F006D0919002FC0A30071F60800D0109500C51ACA00A1D6490007
:401F800024D648005BF5F800713F9C008F842100F413EC00F5EB1900C42F6800675DBC0047A9DD00A7228900980C690046D447006A729400428E740063EF8A009E20430032
:401FC00028A97700B8AEAF00E6F80800734AD1000300EC0096A41C00E92D300058B04F007DFBE80006349F0061BB060076082500A670FA00AC4D2800F52D3F00D24ADA00A8
:40200000FC94FE00EF75BF0029C0C300F68E4F005298ED006D9F9D00976D3B0055A1EF00FFD85B006DF9790052A7F8000A266B0015503A002AC7A900C7A397003069FE005E
:40204000ED193B00E504BA002CBC890007045E00ECF16000347E5D00D9D05A0083594A00F12A4B00827DD000904D5F00CCE63900742B020006B1B400C1EE2800CA25CA0035
:402080007C8D45003DF52A00360B5C004481F200F4EFEE0021F5FE002FD5E600417EC0002C9A7E004F106700AE6A5C0054831100A9C24D0037507300CA6E39004DCE9000A0
:4020C00002ED5800CA59730041704600B7ACAF0080F03000593FBE00A097B3000A13B700F74F3E006DCBE8003B855B00F1179C0088EEE40092122A0003408300DFAA660006
:402100004CEB0300815BBC002FE5B600F50736007D14EE00483E6C00ABCBD900208F30007BE1D600E6E4F400E5DB7B00CD9F2D00D99E1C003BF52700B2979B006FB8400039
:402140006078C6005C659700AB2ED8000E28E50045C56E009560ED0033D3AB00EF0EEF006E5909000BBD8200C0C9C90090649A004DBC6F001A67A100F811EE001EF96100A3
:402180002C4EEF00FE622100BD4FF300FBF5CC00A94F0D00C0200300CDF6D40093623300EA43B500DD675900B230E500C410590067FE7500B62327007C21BC00149BCD00B1
:4021C000AC3FC7009B0F82002FAA5000FD531C008219AF0072D3EA00624D0F0061F7ED0047F52500363A7600E746BD007694A6004AA83800B056D400511EB100D3B5F10072
:402200004303010039230E00CD81FD00AF01E300D62FEA00C6C83A0013D8D500652F9F009D72BB00F9F4F1007FF5CC00964B8D009A77400014DBEC00D2CBED0073053900A8
:40224000B90DE300B39BA5005BC471002D891100345A2C00B4AAA5005629B7003FF6A600FE49EE0080A6650031B448003C8ED2002A62B7006FEBA500B93C590076994E0027
:40228000CEFC1300B69AC60050C346000F5F9D00261D190043830C00408C7B0067CC9D0061496F00C19BEC00AAB35C007FF3FB0087B10200D2C1E100580B4C0077239B0069
:4022C0008574E2005ABE9D00D500A900E1C0BE0040849C009BC80600E0C03400A5300D001152D100CA752F0013A12E00BAEC2100A38B4F001FEE17000991DD00D2A7CC004A
:40230000EC64D1003B6367003B1DF7000B69AF00D611A00087A32B00000BE3007A0EB200D8B01700094FDC00505B1F00F4CF900055F4010031418700EAD7CD0027FA2E00F1
:402340003ABEF700E0DA6A00BF1AB50034282700F7175700B2652D00A590E800FE31CC00BEFB2D00FF707600067C6A002E1A25002B422600642F3C00E0DECB0091E93600B9
:4023800015D0FB00ED2885005D27AF0092E22900170C3600410BB500DA9D6300CC5F3C008C64FA00703CA500C7A3B100207F5800B70C300018677D00EAF73A00612DF30060
:4023C0001E816A0018643A009C491200DCFD8000EF4955000BC3C80088D2C6008D1A6A005503A0005972810015F60400227CD8002FF84100C33B15008A744E00FA51CB00D4
:40240000758A0D0003133A00018607000D11E0004B6485006B6789007C151C00C8DA1F005B9BC3001A6EDA00023F8700C3C284004CCD320043328200EBE0F000AAA8F2008A
:40244000A53311005D65D200FE3C9F00A58035002FE8D5005C5AC800ED155D00C8026200631C560053FFFC003E469700978B8600EF3CF900488EC900E2259B00EA05DC00A1
:4024800042BCEB0053539100F0AC9600C7E3810081481200BCE4F1004DE83B0017CE7C00439F060069A48A00057830003E266C00AAA85800601855007CAE9F006874020048
:4024C000016F67006E2746004A559B008F01120037A9ED009483A400AC715600DE81CC00AB789D006F264500046C6A00F2643C00DCDE9C00DA5802001C5B1C005A763800FD
:402500005B38B00037FF0900FED6C300403938003E1D4800993347008D20DC00AC7C8300D8A3A00059FC0700CD018A00CC245B0067713400DF17AC000225AF004CF4D50034
:402540001EFE1F00F32955007CB095006A3BCE00DEE7BC00C640D5002A9D5300006A5300FE1F9400C9236100E6E55400987D0B00DEFF99000C7DC300E783CD0063511B0043
:4025800090B70500BB0867004EBE4D000388DD0051378000B8D52E00CE67A0004C6019001BEFB200EA6C8E00836CF40000999900BE35C500C0C07B00C86FD3009C520D001A
:4025C00012982F000354DF00A784CC007028B00001EB5900AA8CC9000E5A8E00DCA7CA001F3DAD00DD19BF003AC01E008AE79400CED7100082E91F00DA0BD40019C92F0022
:402600008DDAF90039336400C9C5F700C3EA590086EDD10085368800A2A86000BD3898003A61B500E18F44000BD7830064750E009D35D100D1273800D0AADE00203AF90053
:40264000BD48C5003FA41200026A1000EFB0190066047600818E2400A83951003215AB00E33E3800563354000BD81100BF4494001B5B2A00C6ED6300327BBC0095AB080008
:4026800071E0A500CB604500C73E4700DC2BEE002752F7007E29BE00756CEE00AA3C2E004ECB37008676000031136500391F2F0075D7E800B6C843001335C70031A49F00C7
:4026C000341E4B00279C43005AB08200111373005BFB7300A9C0EE00B825B80075158C0098B0F900EFCE6E0021297E0057306400D4EC5500C0AE4D00853685005EC0C60036
:40270000F8A51400998200008AC44900BD55CC00261FF70022144500E4EBB400A5B23600AD81D200068E070049F3D60060348E0095AEBE00C8DB4F008DBD2800B38AC70059
:40274000140CDB0011C4EE005FF9ED00263FEC007A0656004046570045780C005886E300E6E1D2000CC9C7006CDFD0001586C800A56308001452E500614D8700EC069600FD
:402780001AC1460096E2B200F7596800ABE5B600B186FF0026195C001B3ADC000F6834003BDDD7008168A4005751A000D5599800C1A89B008247CD00E7F7C700425896002A
:4027C000B8E33B0080E8D600042B1700637CED0017563500AADAF600AA6C28009DDE8200573441007680D40061E709006026490069E62D00CB23E40067459900936190008F
:4028000036C2FD0054FF0F0010A75800D152B500FF817B00EC770900834CEF006BC84600A68934000C94FB00DC098300358F6A0052A5F9001D680A00BDE8D100EB491300EC
:40284000AC60D200C45C360019BE2300D31D59000CA0FA005480C700D63742008D068B00CCF99C0032D72B00C5A37B005C20F600DD9A0100BD1DC9000A588B00404B750041
:402880008E20DF001BA20900E07E4900FD77BC008329E100B892C500BD939D00119DC400AFDE3C0070B2BC00E80C0200761C2200C080F2005170D8001BE1CF0030B72B00FA
:4028C0007D70290069A137007159D10084B14300AF89A000F0903000D38802004FB7910084E94B00F51D0500A91451009704830094CC5400011DD60065D732005409100074
:4029000072F539001EB52B0062BB7700D652EB00C0587400B0833C00709C1D001E7DDE00AA54BE0091065E0087B32100BC55BA0085D77F006B11210082768000594B5900F1
:402940005C8E880017A814001948D000D30113003F19AE008AFB8A00CD7E0600D8C620008563D5008C8FB600C8BBCA008C01F900F3A41000A5B2BA00DE580F001CEFEF007E
:402980001C5B37007EFDF8006F6C7C0027557A002798AC00454AA0006068AF005A29520022DC2200B8B5F900DA5D4C004686E300CF956C00485EF6008EFE5B0070A328007D
:4029C000ED64F20040EDA500699ACA00A5CD1D0022C7EF004A908A00E97FC50077842A00C0794E00AE812600A0E7030034906C006D495D0099A7C900F1498800EDF06C001B
:402A000061DFF900163F1900F00AA200C375610078371D00337D390059A8C600B9B37500B716B9002B1547001FF7070078EC2B00B98D0100F1E29800B78282004D70DB009F
:402A4000EE0AF5008338D300E7AAB400D688E6008889290032300B00207E93007A73D000C9E1B300F132AC003F991000B5962B00F5B3CA001BA90900E6368F0002D48B00E8
:402A8000025693003A16110011083600090F8C0028467E00E69A5600ED2D1700ECEAC30001F95F001D31D100E4A68B002A50E900BD6AD600BCCCAE003DB99C006E6EEB00CF
:402AC0002369F10088B4A0004F4ED800C48D1900CB80FA00A6EBE900A4407E006BE95600B1D0C500A276C90077E6DA00EA43E600E392350099285B006D776400A0C12D00C6
:402B00006F454A009E2AA200A43AF8004747800086CB8100197E590001218500090F7800403E4F003F5D8300233BEE008A3DA800D4D12600692E4700B8883B005945B10036
:402B400078213900CB15CE008590D900A2CA08000FFFFB00F6EB7400C8BF4900C470EC0038BC8D003C9D2C008BBA97004D8283006DD5BE00B36DF4009C0AD2004C80CA004F
:402B80009020B4009097B900D9FCCC0003EF7F008A566B004B6AFB0024BA2E00CB60D2003CDED100CDB34700811D58001892680048CED200E33F6F003D1F5200BBA2FF007E
:402BC00039FD8B00893FA700EF4220008ABCF100787C7800C7BF6F00B83CC00087F53A00D645F3006CEBC2004E125A0085D98D002C6417008C1D7F00BE86F100D5858A009E
:402C0000E746D900B90D590011DA9500F304D5004C869D00E9EDF700E60F830095B16400DA9E4C002783E700CBC53A00B7F688008F38EC00730F73009D78B300A350BD0051
:402C4000EC569D0081C1B7007D4DD100BBB5E400FC109B000AA8E400CC91970002395E000E6B9400AE83E000083F19008F8F6000E488560028AEB00092615E00381F1800BF
:402C80009B093A009F3F83001FBE1300E14F2F006E623A00AB04DF008F6182001078BA00D45211007DA84100587F6000C9AE97008239E6002030770037CE190083C99800EE
:402CC0003CBDCE00C74DC7008040C6001AD9B000C4D69E008E4FC100C6EDF40098EAF300249E9000C02B1000F9BC7C00065C97001FA2FC005CDE770082EC8000E74D1A00F6
:402D000046BB250010123B009FCBBE001A0469003FE6A10045535F00297D76007A29A900D680BC0031EE2F00EAA99E0092D851000E40E800A1C816007942470063034F0084
:402D40005091B500B54C86003E3DC00035836F006C96440093B4BD004C89AD00C9600300072E9A007EB23800BB38C8006049D600B29A5300E7057A003F429200147D27009B
:402D800067EE53000840A4007BBA1F008B865F003B35670033EB3700EACFCD00AD65EF009DD8870023370A00789CEE00498E6500632612002E9BC600CF9D6D00E999940051
:402DC0004E57D800C9EF6D006DCA28001FC00800A986B1003C362D007DFECB005D7DD200208185008AE20D008F6679002FAD8C00D406D600D182290037BE4E001CD5DF00C6
:402E000057A72C000146C200547A8900952935003F955D0016432400D3E50500B42ECE00182A27004F5142004396300026267C00833F51008207B90036C1D90008628500CA
:402E400022F924002041C500A39ED100811A37004E791F00F3E32D000BC804001B5237002E6E7800FEE390008350C5007DA943003E341F00571C7F00433C740093F9970086
:402E8000D6952A006919D3008CC5F400D8294B00A4F86400CE5120007DACE200A55C2D0091267C007A33190080F9A600DAAA730055E994003304BB004D84D300F24A590013
:402EC000216068003E7DF0008CE6A70074202200B8C963003E995500D72C550052D6520083BA6900A420CE0031812C003AD7C8002754DF0066CBA200C09EAB0034E85800F4
:402F000035ADF100BDB0F200B3924D0049A6B800726E7C00C34289002B8B830029EBBE00A0DEF30082D9150032F7A8001E82DA0053F92B0086A3DB003D1B8A00222A580004
:402F4000CF2E760083028B0060466A004C4BFF0023C8AA0053C22600F1150F008AEED000A59F83005FFBF7002ED1F10083362400309D2500285503003FF87000E59C1C0060
:402F8000EE7ED300CC883300FEE10D00532CCF005141760030F7B00020F849006219E700275F5A00F4823C003F019800CA0FFE00367555005E6474003CCF24002300CB00DB
:402FC0002806410080666200FAA38B00C356BB005214E50013764E00AA6134002813B3005EEB6300A4F099007D28E700089C63004840AE00E0CC6700637B1400F4B940003B
:403000004527F80081245E005DBF8B008E83E7002DEC0300FB9A200045D1F600C89571006323E500948923004432AB00BF15F1007DDE6F001F8FA800057F9200C9CD75000D
:403040008E3B4900F287F500DD3734002E6E4A00F22AE70040895B0078B82F00D4C7630032FC820078940D00B914090061AF98006DE6BB001C716E00C3EA2800BC1807001E
:40308000BDF9EA00337C9C009A04A200472B5500FFDC000087E47200E5EFF2002AA325002B144500AF374E007434CE00141C1700DC2075003DB67F0072ED0F002F451F0055
:4030C000BA634500FDFEAD00BE656F005130AF00384B28000E19CE00342C6000B0490900CA926A002E406F003B5049004ACD54001282A300629E7200C80E260064BCEC000F
:403100009EE46E0019094B00D5C21C003ED19800CA5C79008EDD880098D65000A9083F006F195E006F80030073AE070067B4C20065EEEF003C4069009CEC3B002AE6EB00D6
:4031400047C2F30022C71B008E8DBD008FE5CA002C4815007822EF00F7BF1000E8710700D2EEE30050DBB800A12716007245AC002C69B20092036D002ADA54002B9ED600FA
:40318000EC7ED200935B2600CAC70900ADBA3E00F945C200D5C7D800F02255003FCEAD007CF26900FBFED000E9FC0B00E1788B002062F8002059D800A0292200F0E194005C
:4031C000AB26840027FC9600AD44F2008F689500530370002E95E00015D09D006D7CC7001EF92C00735B80002AE46D00FB713100D410CA004E8F5400CDAC9500673A5F0021
:403200001C892C004356AF006ACA9D002A543D00B40974008931B7006151AC00DE7D0E00BDE79C000A6C2B0029A5BA00DD874800DB1F1700F8BA8D006BB84A00B098640002
:40324000FE705C00915EDE005F5E0C00B4D27700C218870005EB900046B9B600D876D20015A44E00A170FA002F7D2A0015B32C000E40DC007A09D100898DA100BB0DAB00B7
:40328000E5776900CB3D3900D828D1007FBB9C004C128A00247B8800F5E3AA00E2DCEB0094EF0D004BD178005176900076FAC700E1F3AE0061CA1800454CAC00E4179300E5
:4032C000D5EBE500B8FAE100EDEE9600786556007F658500E239780025B8FC0016A74A0064DF7C0037D639002BFB5000B9D797001DD6C100D01CA500F60C420065268000E0
:403300003BA54000D5243800F10A5500CDA81D00FED3BF00F93CF5004F7A150036A0BA00876A09003A68A30046C622008A2ABE00E8860E00671B2E0071A7F80029A95300F2
:40334000BF4043008135E0001856AC00F806DA00BE277E00890A4300A79B9D00E3EEA3004C4F1900839015004CD12B00A570C900D40C91008A74310089FCFF009020A3007E
:40338000EFFABD0010432B00A0C25D0091712500D013D1003ABF6B005017B60021F9E50052C3A200FBC192003C004700A697B9009A481200918F820062B770002BB83F0010
:4033C000CC84C000302E570025E29900992B26003E655F006070140098E02B000D15BD00C36E8D00C199D50030D63900BD886600F42DC700A8FA360075373B0011FCB600D5
:403400008D26CB00D921CB00E6BF2000BA2B8E00C56B9C000FCF50006A031F006E07A0008A000700A34F0B00FAAEC400D79786006D741F00E4015500C542B6006B56900040
:40344000E5BB0300B0E52400EEE7F6000797E10037A12600A93AEB00B9066700499F840006E87F00C4F919006FBE510096AADC00F35A7600FF528B00D6500400B6566F0027
:40348000ED573A00150D3000227686009B4AAE00F665520002465600D3E64A00AEA1B8003003DD0082F5FD00778619005FF88B00107434002824A5005A68FF00E096E200F8
:4034C00015E2F2005B5C1200B2759000CEA70A000B54940095ADE10046DC860033E7790093F3A5008E217700A2CD4C0025D91F00B2CE2700F7DF8B0000050E00E2AB620060
:4035000059545A00A54BE300F8A9E500F0689000478687003F2DAB0052E0D4000207BC00D4D73F00096BB800D2F0750079691400024CBB00E3A896000F03B00091D3440036
:40354000ABD740004DA47500B836AA007BEE9F00F1F2BF0046929300C5664300D6B62F000AA15D005369F7009FF6B100F4F3F300F120A600EE47D600F0E9FD007EE6A800CE
:403580003F184300B5242E00313E4700B9DBDF00C1FB34003FAFBD0071E401005861A200A0445400C86AD000768CAE00B5C6C80009D5FF0022C1EB00612BF800838E630025
:4035C000507CBC00ADE22300723ED70040936500B6BE86002A416C007CD6BB00E0C29E0032C12300B2D0D8009C946900167B9800C43B40000E994800FB5E800051ABE80097
:40360000073B2F00B811DD007053A6000FC9FF00906FDA000A857100ECEB4B0097502A0008C2A30045A619004E09B100D7AB150096B00200A62D6B00934E15009FB0A300A9
:403640009A05A600CB3A4800D020DF00C6714200882E6E005319B6000684700080560700113CE000F4CB2A00054AC500E8146F00B7667B009A427B00F2A10A007972EA005D
:4036800098B05E00B2E7F70011FAE800D1F0B40081831D00BB2CE40011EE11002727F300FB1EBE00B0172700878BC40016D45600EA23EC006EE8C3002D53EF004BB984004B
:4036C000FDBA840070615500A9BB310002F003008C8C730061F9A20045F8A60049D7C8004132720081667800F3810C007B16D400745D6300E522A90074A19C0015AD90007D
:40370000A81A8D00FBDFFC00AD110B0064143000379EDD00C86C2A00F58A7200684DC400590518003F144A009E8C5700E8132200ECC70900A1637500A67450009030420027
:40374000FC573B0059DCB4009705F100ADC4EF005799CA00D217F900148B3B003CDEBA00E57EA20070F76200193B2B00918832000353CB00C6115200F6B75C008F10ED0024
:403780008556370043E39400192E5600EE939600EA586100E2BF2C00AC13E100B60C420064B561001650B60030ECA000DAD56F00FC086100962260005AF346006FFE040084
:4037C000B564870068E48B00BCEC8B00370D5E00542A0500EDD94D00A07C0C00D03029004302FE001AD9C300AFC52700D838F8008789A900543EC1008739810042C1190091
:40380000C7B99B00FC897200BCBAA0008F8D2B006F2C2900BD316400380C0600CC0A1F004850BD004A6D0200C4256D00C03702008ACA77001C09B700E4EE7600ECECC900D7
:40384000139C160007C4AB00099EC5008D31C900588AD000500F2D0023F48A00455DC1005B9DA0002E252B004513C900A8DE0C002FA8D700BDFB15006A50C90014A68600D1
:403880001096370032BDDD00CA3C7900287A5A005E311E00E6E9A90092AF65003F03F400EDAA8700A6F87300ADF34D00C949E10026E51B00EBCD0500188664004DA72100DA
:4038C0005F638300856CAC007B4844003D138F007C97E4001293A800FDCC1200BFF53F007734C60016F37300D0B7DC00B48DA0002715200014676600636396003501580096
:4039000023CB2600B052F600A38A6D000DD91700ACACC1008CDF4F00D17F59009A639700C2A74F0025559C00C09B7B00498E0800C055C0003D787F00891DFE006E739B0028
:40394000C8481500B2A4AF00184BA00075C6F100D0ECDA00EB257F003C472800FCCD640055A77F00B52C0900F629F9005A50BA00AE4B6600432064003715A400B882F400CC
:4039800073233400355D97003C58A9001E5F5C000DB29E00EF69E200FD9380002CA3C2008BE38A00F1DD0700A9DF2C006AE8A7000D1A6400DB15BA00CC230600E9702E009B
:4039C000033FD5001B234200F8476A00644E2D003C3F60009C432D00C340E300C1B02F004B320E00B400CF0039F7500052B67000102D6500C945A80040FF16007D1FF200FA
:403A000048656B00F396850090C74B00AC867500E1B95E00B0838B00F1E3BA00BADEEE00534B2C009F95AA0088675500DB1E8F004F86D500F5BB6B00B08118007D1A29000B
:403A400068090C001CF6C600D8F2F8000995C90074168B009BEE7A00014B21001DC00500298CC60025123800C6FB8400E6D0B2009D091F001B1B3B0002BAC5004AE7AC0036
:403A8000D9BA55002050410004BF1400539F120084836000D53AD100AC7CAD00D2D69C00EB78C900985504000E1EFE003464D800014486006B335A002E24F9008DD6B90051
:403AC000AE353D00240F5A005AF3C700D695B900394C0A000C63E700EBCC1100483B4B009A10010000C86B004254D1002C872E006B1CF0003167D50042EC9A000FAD5B007D
:403B0000E6A66E0028C78800CC96A700A4705A00741AF400ADD51E0011895D00E3D23C00A2D67500DFD44B00632477006EDDB0006D89F100E56CFE000ECDB60097811700B9
:403B4000D9CF9100DBDBA30044A9990053AA7000C92F690033401800BD47A90050AA9000C3F8A1001BE7BA00578FDB0035973900D5ECAF004B089C00507CDB0031D7B00001
:403B80006CAA8B006188A6005720D00074C410002BA65F00D0B10A00BC8BB200CF353A00B2489400F3488F009F9D6B0056C87D0086041400DCDF0F00967DCC00645C530060
:403BC000ACB5F000DBFD020045EE6100421E63001698EE006384890033A2C000B86BC600F3A1F00029008E00B469EA003C3D42001898BA000E64130043CEF200B899410038
:403C00001A0C3300C4678B00EFD8D20063EC4C000E871C00CEB97500D713490068F32B000A6B9F00EBD3FF00C6977200BBE1B600259671007FA81800EF3AFA00B8E5890035
:403C40009E8D12007B924100B003C10075C522009A8E5E0058406900534871007C4E9C008F5BD1003A97F9007145BB008F468500544BDA00F904B000E0FCDE00439F41009D
:403C800068736C00DE8F8C00D2A4C900169ADB00A93599002C2D4A00B4792C004B734200EA52F200C45D0000CD2A8100BAA00F00E8C97700B739D40016170C008FF0BA00F9
:403CC000E872F200ECAAE200996B4C00BAC4EB00423061001B818A00F95217001957C50022481B00AA653E008E10810033F3980097D074001ECCD400566DE900AEC90F003D
:403D0000AD352800DBEC9600554137001778080005CCEA00BECE5000EEAC98003EB9A5000AAFFF007F35A8007CDBEE007A626200875C1200B638A2003CD31F00A37C0700E3
:403D4000FAE2020004D9C900187ECF0086249100AC4BC400DDE229004286F7003CA7C200A69348005211DF006206D800D641EB00435A8F005C6965006F81FE005206330044
:403D80007228C800183A0B000A463100351DE200B4B86700C6F2A900A3752000A1204E00F2ED4300270E8700808475008DC7A00065C45100D1DDA600D0E7CA003F4C0200ED
:403DC000A009AC00BF6B0C00D27AE500AC301C006D0B4D0024D8DE00DA7A5500A67217004C055C00EA1CA00021B679005D82630077DEC900241992002DA31B0084C1F000A6
:403E00000B89820095DEAE00B8D0D40028643A000BB685001A745800748D0100D60FA80057124E00FCCBD100452C24004A5329000435F70091643C00C02F5000C0066400FA
:403E40000B2FC800329FB7004BA2C400850AED000148D300245970006E192C00D1568B000D71A600DBB58500F620AE00A3731000BA595F00E9A4A80025B3F1009852A100FF
:403E800032D90A00D11903000273FE006F7DE10010419D00CF8386000EF775007A980900F5BEDA005912EF003093080020E82B0047AA7C0051843400A56C720094879700D5
:403EC00062EFF300C59C7600427D05004E5F3F00BB704800D2448E004DB1B2001009FA00DFB1B60085FF6A0031177E00882B4A00295A3700AE32CA00C1668700383E490055
:403F0000B79BD30099FE97004B19B2003F998A00B06534006D919800A6BDA90035925400191FC900F4A06B006C5F3100394FE100C19E3D00751F2000143C42007494D90088
:403F400030F269000C5CD00021BA090072C4A30024F9D6002EA83200206753003C2301005188F10028E20500B0F4E800BBA97F00E2C2B200B2A95E00E7D288000251500051
:403F8000FBB04900C01D490084ACEF00A51BF700D8303C006D83C4004E85B900736FF800EC9A6C00A18DF600A5BA43004D4CBD005B33E6002F902E009147C600C8C38A0091
:403FC00083FD26007A8EDF007D43110055D25B00564C7B006F81C200BCD96600ABC8AB0045CCFA00B21BD800F239A2000EDDE30056F14800F363D0003FD2C800B74E180003
:40400000202C1000C54B9C007421BF00A9FF0A00DE157700C3AE9100694ED8000F284100316EF90032CA9500CF59E4002B1E6F00167B4800C96C0E000A25B000D18A360086
:404040005DD3B10066DFB80036816900D6430800494D6900AEB8CF00184727000AB888001D75940025764C006AF45500B64BA100D99A7D00281A84009E987A005962E100B9
:4040800051F07F007CF6C60088C8870009776300B68BAB00695C25008D004B0075344D008BD25000D95213000CDD3F00227A9B006A1C7900303C5C00C0ECF000EC37A40036
:4040C000D5E0BA00A05D0700EC5817002D1BED000E29C2006932310010C1E80024053D003901F40041985400BE43F200D3DC33002F31CB0008DF280014C452008A80030038
:404100002B389000C410AE00F2D81C00EE1F6000CB0D2C003A103E004F983A00881D2100DE09B500CA8461009C520300A0A7F600B5880D00423BA500557903008EBB4900FC
:40414000C855BF00EAF09F009B0C40006E528C00F914C1008644C400CBACC500FA5D53005FF7300092513A008D18D100AE86AF002EE20C00980235009456E600D393F00068
:404180009467DF009101D000472CAD00FDAB2A0012683400C6E03700BAE16B0087701100BF3BE700CD8F0B00F0B54F00DC4F2100C58420008507EE002DFD56002BAF9600DD
:4041C000A36B680074061300E5274600BB8D6C00D5931B000A0BEE00622E570026C4C400FA4D1200B57795003F814400BE502A0071996D0044C0AA0080822D003C6D19002F
:404200005A0EB100D4D5EB00722BD200C279530015ADD0003DDC500009D4E20018843300DC3FA70024C46F008717B000C512A1007F592F0061EF5400DB02C900B70F9B00BA
:404240000E216400B2B6AF00592B3D00272F8D00801B1A0056F3660045B70800E5098F0010719100CEBA1D000E75CA005AC4460029F908006BE80500936D7B0064E07A00E8
:4042800027E03B0088F97100D21B7500DCDC6100187487004D244600BBE10400C7348D001B635D00DF4427005564C7008C7DA9004BC4DC00CE1D5A0043C3E500EF290D00C6
:4042C000C74D73000D98E400020D20008C7BE700CECDFC0068EB1200E968E5008BD3F700C6899900EEB75000732C9D008BEE3D0073FC7900F0FBC0000C545B00FEACB30090
:40430000F71838007A7647008A8257003285C1007EE62200E6A77800017FBB002AF486007C6CDD003BAC790089A9E600DFEADD00472D42000E996500B6A8AD0088FB8800FF
:404340002DC466001E8F5A000E5BA8006FFD8A004230AF00360390007AA9020007891F00A5562D0094ADF600DEB708003514D700F1FCC1001CFB6A005A2073002421A800F5
:404380006D780E00C4061A00BF79960062B8E80071B62500D6C06500167EF500CFF1C800A2171000FC860F005F906E008AFC7B0073145E00C7F62500122126004B438D000B
:4043C000CA7E68004EF438009F21E4003877D300FDAB340015AB2B002B5A5D0072277400116E8D00B10B9400CB192D00915BF100BD8AE10099B437005DC750001E0F6000C0
:404400005EADC0001AC3C60008DDCD00F337F000F956BF0061F43400EC5ACF007C2CE200EBF97E0006D5E300AAEF450008E43000092E04005C969F00D5092C0056479600E9
:40444000F68E3F00EC5F9600E40E56007D1CC4004C8D5E00A8387200BEF10900A692A000C82EBB00F5E069000FF16D008B4CEA00A66FCD006CAB9100966C39001F7EF70064
:40448000AA298F00090A6300ABEF9D003E2937003B148B006F817100D4A7F200A6217500C4D18C00D2DD52000D89C80032DDED00EDD1E0003899A800C3880600767CFA009B
:4044C0001D7255008F83A7009C2A030039552200F6E85700D10B2C001FF9380007D6EC00246512009E7A7700C75804005DB35D00B493860081E75700E4BC7C00D0510500C8
:404500005916BF009B1A9D00424FC400301A140012B49400F175D500B8C50B00711B2100E0781D00A3A9E400632C5B00DF6D5400E9F5410035E85000B58EC0000652C000A8
:404540005F50F500E8C899003AC89200AD8DF800C8A3B800C9A141001548BC00356BBF0097284200E0835D00C3CCF90033776A00C7BFF20044FAA20032FC1A001376890033
:40458000B2D6D8009E64C30083BCA100E4C98A00770971001675A700D43BC0001BA9BE002170ED004A2D4E00D6040C003D999900CA99B900F25DE60031627300559E3A002F
:4045C0006B058F006F724200C0D1E400979921000BF5F200B7DF7C00CCF68200F19426004F498300AAE9B300EB85830037803F00EAC32900534907003C43AF00EBB3490008
:404600000BC25200D2BF7C00778BAF0081AB3D003BA3A30063174A0072A79D001444400049CAEE00D055E50040D74400A07C0700E5715B00206B38005303C900C251DE0094
:404640005EA0520034E91E00133183002BFB500054C6F2003593ED000E887500D1439D0058F24900DF087900970C7100214A9D0037CD2B00DF97EA0094E0780099AC7F00A7
:40468000742D7800EF475800A68D990098E7BF00FA1E3900FE48B600B67ABD009485440004CEF30024016000542BCC005C98B3009816E2005DC4DA00B1164B006E4FC70055
:4046C000E4B7760051559000908D9F005C6DD80098FA6700C959A000EB82050021B1C900DC426B00259DF20062FC30008311D700629D5C000462D000C3859E006421A90073
:4047000009492E0014DE81003A6B5400990AB70000BA980070580200332DA600F00D6A00DEB00C009119D700FC33C30022C3D500CCB92B00D9E3E8001D34CD0077310F00BA
:4047400043CD21008F0DA600A63BB0006629A000DCDDCB0055BD38000FABDB00712F010090818C00D0D7170032DC860070CE41002DE96B00AB924200CE938C00BD978F00C4
:404780009C9CFD005F324E006FA0C400AD1DAC00A612800018FB2F009EF1FF001205890071226C003C163800222D96009DA1EE00690E530018DDFD00E89528007B32CB0081
:4047C0005C7B6F00C735060076518100350BC900F09EDA00BBE1A70030F2CA0049AF3300AE2B92009DD5F800E9728F000B89BF007FEF7000C949F1001C789900407B8C00F7
:40480000E6B26C000A1DDA00376590002B7509007351FA00243521003050F200252053007E47FF002364C400164F64008D5A3B00AAB5B5004ED2F000E8AE0400F435760005
:4048400099710D004A7FAE00A68CC800C7153400D4077100A4E28C002C15FD00287B9F00D101C000AD52B900F491FE00D66BF700D2CC8500B94EEC00575E1D0058E0F300AA
:40488000E190A60053E236005EB7E60084AF2600037F860056B69F00D51C0300A732E60003436E003FDDD000A5BAA30083A572003E7D1100DCA934002D014A00D2AA1300F4
:4048C0002DBCD500D2B2E30049CC1E006B74480089D36100A674AC00A99778000A834500FD1A660097C7D10042B7F10010A89000D8446A000585EE0059855200CBB72A0074
:40490000F563D1008972EF00EFBE11004D57C200AFED6D0031DC6500271BE90056831700B3BD0400130A7800601A6200E4C996000E6BE2007E4A1300BF59C200051053000A
:4049400013674B00CB211900A8A9F700315572001716D200DCFDDE006DB05F0040261A00CEF6B700A8909400B1446F006EB55C0068FBA0006FF88E00C4DC3F00883E330081
:404980000F77120073D52D0095593500BB974D00179D350013140C006E1F100059A2FA00D66E48002DC671004A2EBA0095B125003A52530054208E00D8D2690050182A0067
:4049C00067DEB500E1A73F0097954000D029B30043969C0013AE9A0061E5A90042C9030043AC9A0079081800D2F1A100B30BE000ADDCD6000FC68E009BAB5A00EE161B006C
:404A0000F7259F00699E8F00DF4BAD001FE5E200063232008562B00010380D00BFC88F004FE2B900FA8BBE00133C4A002D0F6300E3F18E00E4509700197ED000D4AC29005A
:404A4000DB49F500C2E7C800B44E02006C43CE0042FA0900A525C6009AF2C200A46A23000F2BEC007029E5005B6C8C00BD49C300A47AA300E5ECE0000559EE0081E14700B0
:404A8000852762003F6E3300778D70006386C70033CAE400B793A40036309B0058CE7200BC7FE30005C4E70066E74A00C17B6D003A73E30073A4BC00925F0F00033930009F
:404AC0006E4A700099A314008877C8008CF75700E75389006C4909000D37FF0019BB620096FA6300BB3FFC009B508800ED4A890080283A00165E950075C12B00364A21009A
:404B00001EF9100001537F00DE7D18007EF5A200EAEA390045B8C90056CC27004408660051989700D992AC00BF1591008653FB0003673B000986EB00711C970045220900A2
:404B40006EF765000DC2EA00E3C22100CB3D1B006FD082008025F6002F5CB300A35A25005762C7004CFFA9000968E100FCF757004A68AC001D557F0053F7A900D8EA3400C5
:404B80006DDD5200E9CC9A00FC988600AECBC400E0EECF00DD25AC008E7B5D00574289008705E900894CD5007CBB0100EB1535009B9E4B009B2EE500D13BAF00D332D3008F
:404BC000B37CA000AB1C8A00EFC88C00F714070095A4A40067A3A30039F182000E9C3D00CAB02E001BED87009B4ECC002F6DF800E9EAA500D33ECF0016F80700AFE9670037
:404C000039330200B692DC0063A51C002753060056813100BCEB46002A7612006CDF9500F806320023F0E300127890007AB82800190DE800380D5B00DDAACD000B60700040
:404C4000AFF7280038E9B000120BF2006EC89600AFB4400059481D003E540C00C4B5CC007427400076A4AF00636511007D81940031D6AD0051A321007B60BC00AF3A2800F6
:404C8000CC57EA000CB37C0062CAC10037C76400CAB8F0009F534A007D69D0000FF30F00FCC91900C6157F008728C8001278A2002C937C0011B801005E7925003E27900017
:404CC000F0D674001FD03A009EE10B00EBDF6E00897EDF002D1F8D008D883A00DBACCB00B31F8900BBA39200B48427004A00F000B8E94D0086C7AF008ACFC600A135CF009D
:404D00006A604300B482970000E6AE00A6D5F9002917BA00D89EB60013A1BD00B8EDA2003A6E5E0066BBE2005F35D40037DF9800CCFC6F00D2738700784983002AC0430020
:404D4000897C2200DCE0890000977400C83100003D1A1F00394AD3002DBA3A00B7B21C00DFC87D005CB664000762D0002AB14800E8F71C008BA8C80097FFC200562CA100EA
:404D80008755DC0007A38C00CFE4800076016900E5455400AB5466005964A9008C7C3A001E0C26003AC19D006EE9850022147700AEC934002E5F1300F3FA0A007382DF00E0
:404DC0007D11310031E2AD003F7AA100CA25B100422D620087CD2D00AE926C00398E770085BCEE008DF1A0000B7FD70028471300E02B8600E8ADA9001A2ADE00350C950007
:404E00008FD9B800C8A5D100BDED670090AA83008076FE00FEB70E004A0D3800D62B59000BD40200ACC9F10065022500A32A4B00899E45007E1C0C00584F3500716868008C
:404E4000792A4F0000783E003777F5004B32B100677571005A5A8900C657CE0062F478009338E700BE3A3D00DBB0D4006AE21B00CE343B007B8B7300C46CDA00092F7A0057
:404E80000BEE9700EEACBF0098F34600A318E0008D42AD00B8CD37006532F500D49411007D955F0071B43900F565E000AB14C80015EFFF001ED5A20056F1F100150BCD0013
:404EC00070BC9D00FE53120003FC3000FB5077000B6BEB0062C242000C1AD0001EAA20000F587300F7915D00F50C8100DF064700BBDFEA00E2B80300CA8FFF00B5922000A3
:404F0000AF1BA50094DF0800C601B100163F8A00594E4E00EF5A100036F268005E3EDD00B2F04400A2290900E528B70096B03900A47B3D00D38D4500DFA1C500BFAC4A00E1
:404F40001BA5F40077C5730097A5D4003555D8009BAB6800A3536500D6DEAF00B20D9F001F6238001B2A4D003F26B800CA3E5B00E69B1D001F01E60079FC1E00484C3500C7
:404F800026BFF800434C1E00B867B2009BB5940007E50900FAC2F6004E7239001ADBA100E1139E008CBCBD00D8021A00E60E0400AE72DC0099C0CC002997F3009A8D4000BE
:404FC0006B657F00EB045C0060D191009FA84A003908CC000CDB5300BB3FC700A2519D00D2A199004018A000DE9E7D007BF5BA0019068F0062D70C002051D000AE71BE00F4
:40500000B101F50018B59500B8864900FF8E8E00BA2C6B00D3FC2D00CFE64C007F554D00C280D100F9F69A0090EB9400CCEAC20005CB2800D1AC9A00A18B8200A4C83100D9
:405040009D69D200D883DF009170D200B58408009453EB007D3DEC00FE01C900780A8E00C4E515005096B900317DF600720ED600D6485F008AD04600F7612D0091441600D6
:405080005AD797004F46F600FCEC660036B96E002B61E000E3659F00944B6700F643A000EE397E00A09ABA007D588E00E5303800D3CBB90058D14400B05D8F0007958400B7
:4050C000E29B1B008AF6FA0052265B00DB75B90037768F00D8FB710050250200ADF8F600E8DB3900139FFB00BB15C6008D0C1900E7A7CE0067321800E2B369004E602E0058
:40510000BE9D5100D1F4CE00C3C640002B7BD7009D33BF008D010400A3F1B100E54E4B0018B15200594AE200A7D94C009072550019545F002542F1009A06BE0019E82A0096
:40514000DEA02A001E933C005BEECA0033975E009F1551004216BE0061262F0046389300330D010033BF5C005850A300ADDFFE005A9E330039729800C3907B009032A70074
:40518000DFE037002AAB6A00ADD94800955C7E00AFA3EB00314823008E452F0060DE590029C33D00B5FC1500FDD7DA00F3095900B3581800009F5D007F192500DD19D8006F
:4051C0008D96D400968B05004A2718001A26EA008EDDE3001FA65600EC94880065D7CD0093DCD100918B7500F8A2F300D213020080A24500D630B100DFEB38009957BF0051
:405200002BD0B40067A6C900C05C4600B114CF00EBE9BB00B7A08B00490E0F00A2695400E086790007EE8E00FA339500FA76E600F70A33008613A1001F7F1B0083F7B600EC
:4052400039CF1900B9891D00824ED0005078B300FCD78F00D1A11E001921E90087B55F0021348B0023460D00DCAAAD00EFABFA0043A18A008B550F002B333A00663C6200CD
:40528000A8BE380017ABA1006EE2BF00BD1CD900AD204C007CE7DF00BAE3720093458C005301E900EE935D00796CAD00CBA6FF00EEF67100F31AFB00EB2F2C00FB49450015
:4052C000093F59008D060900CE5E2000F3CD2A00B7E0210018E6E40018CF96008A3BF300F8CFF900EC9A6100F9B24C005CD24600B3135E0028257E00ABF25E00CC47BF009E
:40530000B7C893008C38E000A7F729007F26FB00CC1A7E00A1C001008A5344008EDB6C000FA8420084ED24000FD3C9009F217B004411CF00165F1A00A64B2C00ADD56C0062
:4053400089614A0044C82B008A4D4F0084A2C500EB046F00B602B0006B298200F7B8DE00929BF4007A3F3100FE6BDB00FE67DD0093C65D00C6EBF5003BF72900634816003F
:40538000E8721E00A249BD00E31C3200C478C600DD5A8200F43A1F005572E8003F140D006A193200A5A62B006597E6006100A80016227700BAC51D0065D1C900A8443C00FD
:4053C0003BEBBD0045BC2C004DBFA400E345D500A97D2F00CD41B100217F3B001804F4003658400090EDC9007EC998002BFD69000F57E100DA5DCC00E5D3B300A500BF0054
:40540000C1ED7A00CFB52500CB6EB10074DDA4008E4EB40077001E0095CA0300DCBA1B00B8049A0022E33300E5E1010008653D0097CB38003CA09100C586360095E44D0037
:40544000F3AF7200E97E2E0079173800E3904C00690082005C2F2200D3D6FA00E77FC2008391D000AC52F100CB411F00A3BE5C00F0637000470E320022763900C9E77300A0
:40548000A6BF8B00005619006750E4000F32040054BC43002DEC890021D52C00F361A800855DEE00E0045F0014D94100C2562B008CCD89002D4F5C00DEF813003C254200D0
:4054C00039C22A00DD8FB300AD2907001A1203002BEAAD008E2F0000CE477900A965FE00C029D100ED5A7600F5EE720086374D00C8E57A009EE7F20066790600246DE40075
:405500009F80CE00F13923005535B300E354F10065EBFD00F192A700CBC01E00C06AB5004D849C000EDA6E002AF40A0050440700C20C1F0067CEC300920EF100C3380400D2
:40554000980EC2009DCCBC0036ECF400C5268800C73FF9003E55350047F31D00E53A0200214DB6006FCE2100ABAF5D005B44A6008D3FF100F38082003FA2DF000B40E000BB
:40558000B8C81700B81EFC001151CA0063A2340067B4BC00DD2F9600413B740009522600453DD80040C95C00B5E10D0003B23D003BB6DB000D6DF500822B92003A24A8005F
:4055C00022CB8E00B0F8810072E06F00FD476F00D3455E0038A8D700D3C1DA006328920030F93100073D6800F07E7800884E4F00CF490D0015A14700347C54000A87E30030
:4056000085454500DD3E6200243A47008322490051267100AECB1E0016435700D8340E003B27D80077AF7200B7664C0065DD7C00FDA55C00FC91DA009287D300DE2F160095
:405640002624100062952700710DB1003520DB00E7B6D500E3A94E00E08AE300806824003E8C3A0031DCFD00F3A7F2008658A70084A167006C75AB00E4E79B005F087A0030
:4056800058FC8D003BCBBA003E0131002F082C0096B03600381691004451F40029F1CA00745F2100FC819800E24FB90008113B00CD85EE00F348CA00168F2800C4BED900FA
:4056C000E37A0000BA769F009A87D700519BA700CD2B98009AFFCC00CAE38D00254B820070EBDB00878259007180DD00B62AE3007B05A900BB6B6C00DD54510046B7A800C7
:405700006B92F0005F9C95009161C100F04B9D0089BB4700CE431300288FEF009AB306008B6A670029803200A9773100E47560005358FE005AFCC600E819280058C1D5009C
:40574000AD2F2000D71F3A00ECA8A6006D449C00F16B7D001EC5670087FC200037FC7D0025A1B700112212006722A300B4EBBC00A677300074547B009DFF9800EFA5B900A6
:40578000437E4600A5B76D00E95AE0007832AC00C2B71900EDE69B007C4DC900D214D40027ABEC003D718500FE217A005090B500D7777F00D8978200944EFD00D406490075
:4057C0004BC0E800368EBB003C49B800F28FF80072947500FC219B00FCE40300BE557B00AE4BF30066208600262DEE00FD2CF800FEE6A900DEF12D0078F00100F8C9F400DC
:405800003A855C008541CB0045D4F1004E60EB005E42610082E61A006A5C2800773A4500368A970070527700177F9F003F1715005481CD000175CE008CC46A00204ECE00A6
:40584000184DB400F841CF0044AC2E0009561600895A1900D2010800CA4983007410CE009F184200413FDE006FBE32008A11EB00F9CCCF004CDCF5002F99E5005A717700D9
:40588000177EFC0008097200E897030007E0D800C65854002CE05100B38ED0002A82B200649823009909610035BE0A00253863000DC19D00B9C0E9001A363F00A1DCB900E4
:4058C000FF0024003C4CAC00115AAD00EDDB0F00F43DFC004CD145009CA93900CA4FA1005BE0C300F3F5E20016381E0004F1C5007D5F27000E932A00657C0D00000C2000C5
:40590000D572C8001BD86800BC93800038296000215A4E0071A5A10043307B00C0837000A94D2800117A4B003D122400847F6F00D1821B00CF99630006670E00E70B950038
:405940004817440056B955005F02500067050900092AE3001594EA005F41E100744BD9001CE48400B3EFB80015BF2F000B9BE700CF2A590012503400BC8216008F371C00AC
:40598000900A99001C8ED30085CB8000BCBFCA0080766F00FD37E200B9FCFC002788BC007CC37500F792BD00284FA700FD6AD800E2E54F00B9C7550079F21A00EE90A200A4
:4059C0008C8FB90075C81C007CC581006E89B200E4F7E000A95863000BEF4F00836D87007A1D6500E3AD0400A1FB1D003B542600B8A73500AB820E00030B8600978BD500D8
:405A000079A5B7005F19EB0073649900CBA0E600A152B40019926C00F8207C00C335FF00EA4A9B0045E133006A60C000FAB1C400992BEE00B07E8400AD470D0086291400DB
:405A400010DA6A0051E79B00C7D50B000167A800C70F8B0032F4BA00A6E96F0009FC1C00B025580017E98C00D7F2F1007B7DF100874F530029F362007FB8B00074BFA70024
:405A8000C9165000859CD5008FC16500A4A2E5003B9D6A00490DD400632C8D009BF9390006CF9C00690563001340D800A6D828002DCF2700FA6963000761D7008C23820020
:405AC00067356800ADAB710050EE180034EECB00A4086F007B459A00CE7D820070DBD700164CD80090437800B2A17E00C3B501004E5E8E005520DB00AA8DC8001E5ECC0092
:405B0000B665AA0067EF21006DC06700EB944A009446DD003BAD3D0000278F0039D88100D98D9F00D8F97C007FB6E400F5FFF7007E9D740037D90300FCE5C1008DD5840028
:405B4000A4C94D00CBDA28008139CA00D2E85F0001CD9C00F65CFB00E55F5F000BCCBE00522BC700A7194E005A48DF00A6562C00CD100F009F41760069ED53007BE1D200FE
:405B800033E886001CDF54008CF7C50085F35800C2E16E00F5B9570010EC2B00AB00D400A4E94500CE5853009E447900302D01008DB0530056CF9100F121FB00AC6AA10013
:405BC0007270C90025B9CF007D094400DA2FA0009CB21500748FF00006556000F7FF450006ECB900055846007C4EE3005A8D94005011FF0085C5D50057D599003E0AB700D5
:405C00006921B200E197D500DB20C100FC0F49006FCFF300F10347003439CA00F10ABF0016286C00781DC6007AEA8C00565A02007AE79800D94DB300224FD4007027E30036
:405C4000C8BD6200891936007B2E9800421B2300C42757007E6C270075615100196FEE004F9A8B00AFE58D0087E39E006BA0AC004F999800F063D800FC10AA00275D31004A
:405C80007C225200FFB744003FD43C002E182B0060C99A002A803A0031B91C0019B5F600CF84410056021400B285080066D96C0023B671006586570075434D0040D41B001F
:405CC000E32D3000FF8A2500317D1B00FDE6A600A6BE850064351700C95D1F00430ABD00C7B805007AC87400D85DDE00B2976D009AC06400401A500040C8670083AD08006A
:405D000008501100E44CB90030034600266B8E003CDF2900281DC500FD20070098F2E800B601AF00D6603C002C12480081533700FEBBAB004DD8E1005E5FFA001204950060
:405D4000E29278001EFF7A006097640086FB4A00104E8800F1A53F008AB19D00EE2A4F00E05ACF004F3DA80059A402004AD15200AC3698006AA6B400464F4400E782DC007B
:405D8000D2C6DC0097C2950070B61200D783D500B2326F008B6F7F00FCD992002D59E80014EEA900D778F2005A31B900BF2B4600818E8F00C432150005C79E0086D77B002E
:405DC000B9634E0055376600450CEC00DC01EC003DA74E0006F066009C133E00B31966005043EF00EAFB0C0067C50000BA860A00C201EC009B0EA700A58BA50059AE1B00B5
:405E0000D9853D00F859C9006CE64E0096E01200A519960031AB780094B263007F6DA70015097C0000542900C22B1600C429DD00EC1CD60078E61D00ED896800201D8F00BA
:405E40001020E8007BCA5D007D2340002CB23900EEB9D600D7CF02009B11DB00E36C0800D0395E009EBF3E00A47CEB00F05A3A0037AC1800021C0D008995C600F6536D001D
:405E8000583602002C8E0E00362B9600FE713B00E5BC7800E6919300DF539B009B81B100999DB900C56EEF00FE53150087EDF50049DC0000420B3F0015F3EE0020B72E00A0
:405EC00095972C00AB55600058922D008E824A008587BF002F9DEB00745B4100B30F3900C498A10074722400FB9A7900D8160200B6D3E300D32AE10046524E009F491300BC
:405F0000F6F4DF0021FDE500627B1C00FDCA80009367A8006D94B500B23CDF00D0A90000863F2E005C831B00272FD4001B42FF0019600A000F39AD006F6BA9008BA23500E7
:405F40006AFA060072CFE5004F63C300BB0E4600A80B9600A59E030020B40800A3E22000C50152001AFE2000C4920400B096190040912700E3804200502DBB003F1FE900D8
:405F8000E9AB3E00F1916A0099D4AA0043F419001DB96500416443003A161100BECFEB001F666200C05C0800739B2B004BFECF00E7BF0D00D70DB500250D620016049900D1
:405FC000383C130048538C00A7854E008CD091008BC67100B618D90086A0520091F0FE004329E8001398AF00F26BF6007353E3000841F600AAA8E400D1F6DD0016F96300F7
:40600000EFEE1200E3296500CBAEC70096ADD800B39BF9003E7982006DDC9A000112010046C4FB00E7BC8700D3F355009369980030B66A00DEF26D008B2D560067EC500012
:406040007D21070071329400ECB66C008EC42500CC78E70016DBD30079688300A47D930086E94800BE95CC0063E41900C9E02200FF1BF900CB267F0090C51B00B924D50012
:4060800011633D009481A8003F5FCB00FC637F00BE9ADE00C90EAF0096FB77001F7BEB00DA6E6F0034FAD200DF47E700CD541800882A9A00AF17C600DBF57F00527B4900A8
:4060C000503162005969D200F0350F009DCCA00015D70B00C290CD00421E9600A8B42200AD898B00A113DF0035CC7400C14F6D00F8E364004659D200C3ADE5007B01630038
:40610000CB03F300DE7CA3004AF9D7004CDCCE00916CC60085E81600785CBF0034210700F804C7003066E700F1EDA700DAC1CA0005B4EB004DC733002C668C00268DBB00BB
:40614000096552004AA57E000A302700A4784000E41E7700AFD9D300FCD1F900446F73003A5F2F0085CEC90051B03800C9B74700C2EF5800A3D26D00561B9600C2890A004A
:406180005BBEF90031C5AF00F3504A0005E0830053249A00FF263E0032099100B64E0B00CC237100FAEF62000408A300E0BA5E00A783AE00FB3FAE004106FA00A12393003A
:4061C0005437F8008704F3009B558300DFFD0E00B0E1DF004CD03D0012BBDA009D89D20064793D006F882C0038F231008E924B00D70D1B0050C02B00BAD8BC00C1B2F500E6
:406200007B712A008847B100D9FD1A0015AE7000F6A68B00AF42070094518400A2376500664B740074A24F00D265C600BF0CF2007336CD00C7FA430014D6E800DEA83B008E
:40624000162D9F00FAB17F008CD3E900A8D4A600DB6B25008F98DA0085521700E4F3A5004384F100BEEDDA00E898AF00E2B36600CBD5EF000EBAC200A5B3D80053EE0400DD
:406280004B671E00546F320021DB0D00079CAE00149BB400C3E43E00836F700072F4A10023566D0074FA480015D90100D5A50300B79B2A00B76DF900A4B769002D6D3F00D0
:4062C0005E25C80053AED500D1569D00F6A76A00D45D410008D121005B31AF00D4EF63001128AD0015B92A005AA48A008472800048E54900A81D100031BE4E001B07A800B7
:4063000006BBC80002278D0075DCD8009CE6A400BF77320004D2B4003369B300CACD8A00F0D62900818576000229F90098D92D007488840016B5A3004D300B004CB98D0038
:4063400005BC280037620D002211C6008BFB0800E50EE20096C3F400D4FBE500391DA800B7408B00C84A0F00FF70CA0054319400C6403D0077AB87007B3FD1002D912700E2
:40638000733AD200C0BE9F00FCDE9100268B30003DDE3F00DC2B6300BD14160047E92C00FBCE8900FD53EA00FF2BF400894A0C0024F0B500F7686B0042F41300C2FE860043
:4063C000E9A08C008DA5EF00F318310003905E0004B92B00C172AD00C2663D004C5595003FD66500C09665003AF0D80019C45D00C5D59000B257DA003A680400F3F4D500F7
:40640000C024CC008C71B600E9374400F1F43F00D211F400C2AFE500A7C7C200572AF000CD080400954DFC0003AA740059CB790049B1240081C0130035248100276E170036
:40644000070B3A0060D54F00B5E17C008A38B600A934C700B7F6AA00DC581A00A93879006F884C009A732D005B6A02000DA8570060F931007399CA006D835D006AC04D00AB
:406480006153AC00A7814200B63EC400C40A580021EE0600F4F2CD00E5F07E00CA137B005DAF62000BB70900EE9CB200AF7A2A007C747B00F4068700BE020C0072F30800D4
:4064C0003914AB0008452D00E9F9620087844B00BD1B90002D405100AC5392004806ED0007528600E7F8E200BFE5AF006BE9A5006A990C007840D4008E09400012E6EE005A
:40650000854A6C0011453D00F2D1B900344E10007F254000EA90A30096150900AF3C1100C4F69C00D390B900FD2D1E00B99A40006FAE3F007FF95A0094378600DAD3B6009F
:40654000C4FF1200F48CE600FA10C60033746800694BC0009AA26B003FED8F0027418C00A0A2760062DDED00613C2C002E95F300941EFF00DB57BB0060BB430089D5240056
:406580006328CB00D8A719005EAFC500CCCFEB00FD7C96003EF5A200402F9200EEC2F200AE2B78003196700077611700956E570071C62C00EF279A00ED407700F1656F00C1
:4065C0001167D7005585AB000EF6570050F44D006CDC1C009A277000E0B20E0059148D00E8895D00DB899000A05CD200EF0A7100F448E7008C72A700F7EFF2004F59E60084
:406600007A25E800E6723000BEA3B5001FA7680028E52E00B78FCC006E65FC00EDD7D0003678D8000F4A6D00417845007ED45300E3C02C00A57A8E008FF2BB0049B774003C
:40664000918EE600DB95E90031975500798D210096E13800CAF8D300230B0100D7CF7A00C98AA700CA50AB000C2E380088FB5B00DBE45F00E2B25300B8E0C8004962BC000A
:4066800059A12D00AC7DE700DAE504002D7EE800E669FE000352A5004B352B004D337F00C9067900382D0C003D76B600F4BCE500CAA2DA002265F80067DA5900198AD300D0
:4066C00081057F00D60BBD0026694200DE99EA0032405000B55DD900E70DED00FA422000EF31A1005F1A70001813D60019ECE5006F08E6003CF7E500CA7305001EF47C0001
:40670000FBCEF4007E6C76009AEEED00FBDDE100BE4364001B7108002F849C001FF5B80096593F0038A5A50008106400621D4200C071B5008147810066C3F700B4F66200B2
:40674000E6719300913427005F38150046569100C6FDA700B2E1CE00FE3A7000D1BFBD00070C2A00BCB12B0038E44400DCE9AB00EEB51B005DAA650051C53900A377F20080
:40678000FD0BE500D5C98D0044F8E4000AD56E003E1C3D003FF63900D3710600ABB31D00A5EDA500FF9E0C00D37FD8002BFB8B00349F500044BCFF00607D89009D6729001A
:4067C000D27E2C00F342090081775A0036BA8F0043F3A9006A977C00754653004DB34C007572280049729900CCE21B00DF001E00ADA369006A8C350012F4C50028A29E0018
:406800003AF62200C12002001E6F90007FFC370047291800C8DA0400C9F2960077A1C20006810100BA8E980063C52000E1B82D0050F74A003B45A000E6015B005C34C8003A
:40684000D8B93A005E81F2008273CF0063835300041FA000C0884A001E7B7F003400F1006CE00300CDC567004BB05C0016764F000E5C4600CEB2C000F53D8600E8684A0031
:4068800043156700C5B837008EB22B00107A1A0023B3B400F954CD002ADDBF005C896600F26EC200AB1D1E00D32CE40081ABDF000B408A0013DECD000AD00E003E75E3009A
:4068C0003B9AC800133CE500911734006A8CFF007460A90086565B003D651200F6588900961D38009C08E500DFC49500A966740002C6B700B9ED72008578FE002C877900CA
:40690000BFB41700328A5000C51E77001334F000A3005100DD7FD300A0631000C492FC0049C6E7002B8BC20043E33500CD0046003C9C5300CA421400D9AC8100DA062B0070
:40694000716451009800A300B5F5C400A66ACA00B2EE0B00B800660073A8A40030311100C9CCE600904E0A00A48FF2000C9C9B002A033C001D1BD200E8028A00DF5D4F0037
:4069800063C1750031CA6F00602B780023655A00E14F6A00B103C10041FB78008F1A13003A40F400B4355100999FC40016D92900125D6F007A639A00D35EE0002D27D70023
:4069C000B6AFA50028C4C00034F66F006631D800A1942500C38A0F00E59D3400BC3194007E7D170040558E0078CF1200C6B0D700624EAD00D1FD9B00BEBDF7007BC95B003A
:406A000075D3A2005E1A7000058009006E6E5C00172F0600920C3C00CD52C000E6F7E100D25004001B61B00082174E0028018B00300EDB006AD00300CE4B2000E422590020
:406A40006BCFE1009DC4E000EECD13003C136100BCC86600E0F8560070020C007C931C009DAEE1009130B8004A5EBF009BC311000653DF00C57A44007470200029B9B300AC
:406A80005E0691002F8DA400DCEEE100AE99190071BB0D00C67C1B006C87400054FCC5000E5D9700E5447300DC25200090DCAB00DEE92A0004C77100046F5C00786D800061
:406AC000E1C0CD00698880002171D1002A6E7A000E0E0C00A46F1300C38FAD00496EE900B5ACBA00681AFD00E5074B005B078100315B8F00FC7C43004B93DA0027228D003D
